:020000040800F2
:100000000002002029050008C5040008810400083A
:10001000D5040008E5040008F5040008000000000D
:10002000000000000000000000000000450400087F
:100030000505000800000000290400081505000857
:100040008901000889010008890100088901000868
:10005000890100088901000899160008991600080E
:1000600099160008991600089916000889010008D9
:100070008901000889010008890100088901000838
:100080008901000889010008890100088901000828
:1000900089010008890100088901000899160008F3
:1000A0008901000889010008890100088901000808
:1000B0003118000889010008890100088901000839
:1000C00089010008890100088901000889010008E8
:1000D0008901000889010008491200084F12000830
:1000E00099160008890100088901000889010008A3
:1000F00089010008890100088901000889010008B8
:1001000089010008890100083718000889010008E2
:100110008901000889010008890100088901000897
:100120008901000889010008890100088901000887
:100130008901000889010008890100088901000877
:100140008901000889010008890100088901000867
:100150008901000889010008890100088901000857
:100160008901000889010008890100088901000847
:1001700089010008890100088901000800000000C9
:10018000000000008901000800F0C4B900F004BBC1
:100190007047000070B50C46064600F061F9094B47
:1001A000094A1D682919914202D8084A914204D28D
:1001B0000C2333604FF0FF3500E0196000F058F970
:1001C000284670BD0002002000000220B459002023
:1001D0001946104600F0ECBA1946104600F0F0BA85
:1001E000132303604FF0FF307047132303604FF079
:1001F000FF307047132303604FF0FF307047022930
:100200004FF0000303608CBF002001207047000006
:10021000114B70B500241C60104B114D18682E68EE
:1002200000F09CF80F4B53F820301B68A3F1080234
:1002300096420FD026B13179092904BF0A213171C4
:10024000092103F8041C33F9021C074B2A601980AA
:10025000012070BD204670BDD8020020AC030020F4
:10026000E0020020E8020020DC020020082930B56E
:10027000037919D9082B32D842791A4B53F82250F6
:1002800000F108042DB12D68856053F822502C60D0
:1002900000E0846043F82240134C4279012303FAC2
:1002A00002F22368134319E0082B18D945790D4B46
:1002B00053F825203AB11468A2420BBF00222468EB
:1002C00043F825201460427953F822303BB9064C9C
:1002D000012303FA02F2236823EA02032360017177
:1002E00030BD00BFE8020020AC03002008B50A4B77
:1002F0001B681A79082A02D95B7983420AD900F06F
:10030000BAF818B1054B01221A6008BDBDE80840D3
:1003100000F082B808BD00BFE0020020D802002033
:1003200008B500F09DF8094B094A1B88094D1BB21E
:10033000002442F82340084A286813682146013BFC
:100340001360FFF793FF2C6000F062F8DC020020DE
:1003500028030020E0020020E40200200023C2075E
:1003600002D440080133FAE718467047134423F0DB
:10037000030310B54FF077321C1F43F8042C6207BB
:1003800042BF4FF0883243F8082CA3F108044FF025
:10039000807304E909000F4B44F80C3C002344F837
:1003A000103C032344F8143C2246022344F8183C32
:1003B000012344F81C3C42F8201D0B2342F8043D65
:1003C000013B032BFAD120466FF0020340F8443D75
:1003D00010BD00BF21030008064B0749074A1868F3
:1003E000884203D1934201D20433F8E70348C01A8C
:1003F000704700BF00000020FEE7FEE7000200207B
:10040000EFF30880704700000048704700000020AC
:1004100000F02AF801DFFEE7024A536843F08053F8
:100420005360704700ED00E0EFF3098020E9F00F22
:1004300040F804ED02490968086000F003F8000084
:10044000E0020020FFF7E4FE04480068016801C9EB
:10045000B1E8F00F81F3098800470000E0020020B6
:10046000EFF3108072B6704762B6EFF310807047FA
:1004700080F310887047EFF30580C0B2704700002A
:100480000D490E4A0E4B6846904203D8984201D956
:10049000002102E009468D460121042072460242F5
:1004A00002D1EFF3088001E0EFF309802DE9F00FAE
:1004B0006B4600F06FF800BF000200200000022031
:1004C0006005002008B50249042000F08DFB00BF44
:1004D000040A010808B50249062000F085FB00BFA8
:1004E000100A010808B50249072000F07DFB00BF93
:1004F000230A010808B50249082000F075FB00BF77
:10050000350A010808B50249092000F06DFB00BF5B
:10051000490A010808B502490A2000F065FB00BF3E
:100520005B0A01087047704708B5FFF7FBFF6A4692
:10053000114B1249934202D243F8041BFAE7104AC6
:10054000104B11498B4204D252F8040F43F8040BAC
:10055000F8E70E4B0E4A0021934202D243F8041BE7
:10056000FAE7FFF7E0FF00F01FFB0EF01DFBBDE810
:10057000084000F073BB00BF00000020FEE7FEE76C
:10058000743D010800020020D8020020D80200209B
:10059000B45900202DE9F04F9A46494B8FB093464D
:1005A0009A6B03925A6B04929F6ADA6A05921A6BED
:1005B000DB6B0793434B06921A68434B9A420446FF
:1005C000884602D041480EF085FDB8F1000F05D0F5
:1005D0003F4800250EF07EFD2E4626E094E80E00F2
:1005E000E068D4F81C9008902069099060690A902E
:1005F00019F4007F3748A6690D930CBF04F120055C
:1006000004F124050C920B910EF064FD089B0093FD
:100610000BA90EC930480EF0D3FCCDF8009033463C
:100620000A9A09992D480EF0CBFC2D480EF052FD88
:1006300039462C480EF0C4FC05992B480EF0C0FC3E
:1006400006992A480EF0BCFC079929480EF0B8FC20
:100650003A0403D5039927480EF0B2FC3B0603D5B4
:10066000049925480EF0ACFC24480EF033FD5946A1
:1006700023480EF0A5FCB8F1000F1BD121480EF065
:1006800029FD314620480EF09BFC69461F4BC91AD4
:1006900003D549421E480EF093FC20468268C36889
:1006A00001698C4641698E46AD46514691E8F00F8E
:1006B0004168006801BE1749052000F095FA00BFA7
:1006C00000ED00E000000020FEE7FEE7690A0108F7
:1006D0007F0A0108AE0A0108C90A0108060B0108D1
:1006E000440B01084D0B01085D0B01086D0B01085F
:1006F0007D0B01088D0B01089D0B0108AD0B010856
:10070000B20B0108C40B0108F50B010858010020C9
:100710001D0C01084A0C010810B568B1012815D15B
:10072000174A136823F003031360136843F400733C
:1007300043F0010313601BE0114B1A6842F00E02F4
:100740001A605A6842F480725A6011E00D4A1369C7
:1007500023F0040313610024FFF782FEBFF34F8FE1
:1007600030BFFFF785FE54B1BDE8104000F010BC6B
:10077000044A136943F0040313610124ECE710BD3C
:100780000070004000ED00E008B5FFF769FE0020B2
:10079000BDE80840FFF7C0BF034B044A4FF4E13106
:1007A000002000F0C7BC00BF04020020270E000894
:1007B0000A460146014800F041BB00BF0402002088
:1007C00010B50A460C460146002000F019FD2046EF
:1007D00010BD002000F0D6BF034B1968024611B9C6
:1007E000084600F0AFBF7047F403002010B5094A77
:1007F00013685BB19C6881688C4202D21A461B6800
:10080000F7E703D15C6841688C42F7D90360106058
:1008100010BD00BF00040020F0B51F4E1F4D33680F
:100820001F4C013333601F4B00201A6818602B687F
:10083000226019460746B64641B1DEF800C08E6810
:10084000664503D80F4601200968F5E700B1296025
:1008500007B9F0BD00213960E2B133B15168586881
:10086000814294BF1146194600E0114608461268BD
:100870001B680AB903600BE00BB9026008E0556819
:100880005E68B54294BF15461D4605602846EEE7F2
:100890002160F0BD2360F0BDF803002000040020BB
:1008A000FC030020F00300202DE9F0412E4F2F4CD7
:1008B00001233B6023683BB9FFF7AEFFFFF789FFD9
:1008C0000130FBD0002502E0FFF783FF05464FF023
:1008D0000008236823B9FFF77CFF854214D91AE08A
:1008E0005E68FFF776FF854208D923685E68FFF7E8
:1008F00070FFA8422CD3B042F7D329E08642F4D946
:10090000361A132EE7D8F0E7236843B9FFF761FFE3
:10091000854206460BD9FFF77FFF0025D9E75E68C1
:10092000FFF757FF063E14308642D2D309E010F19C
:10093000140F04D3FFF74DFF8642FBD9EBE74FF0CE
:10094000FF3600233B603046BDE8F041FFF744BF6F
:1009500023681A682260C3F80480C3F80880DA6844
:1009600018699047B5E700BFF4030020FC0300209E
:10097000144B1A6882420AD112681A6012B1506888
:10098000063801E04FF0FF30FFF726BF13461A6824
:1009900022B19042FAD102681A6070470A4A13687D
:1009A0001BB1984203D01A46F9E7084A05E00368EC
:1009B000136070479842FAD01A461368002BF9D199
:1009C000704700BFFC030020F0030020000400205B
:1009D00008B500231846054A054900F0E5FE4FF02A
:1009E000FF30BDE80840FFF7F7BE00BFA9080008C8
:1009F00040420F0070B5084EFFF7EBFE3468054625
:100A0000FFF7E7FE8542F7D800222346141843F18A
:100A100000052046294670BDF8030020F8B50446BD
:100A20000D46FFF7D6FE002385420646236010D30D
:100A3000A5F10A0383420CD20A35FFF7CAFE8542AC
:100A4000FBD3FFF7C6FE8542FBD8E36820699847D1
:100A50003EE0FFF705FD63680746002B34D1A3682D
:100A6000002B31D11B4B65601A681B68B54238BF3B
:100A70000132A260A2689A4203D92046FFF7B6FE6F
:100A80001EE0B54202D9144B19460EE0134A136812
:100A900023B159688D4201D31A46F8E723601460E8
:100AA0000EE05068854203D313461A68002AF8D135
:100AB00022601C600B689C4202D1A81FFFF78CFECD
:100AC0003846FFF7D5FC03E02046FFF751FFC9E7A2
:100AD0000020F8BDF8030020FC030020F0030020F4
:100AE00038B50446FFF7BCFC6368054633B9A36814
:100AF00023B92846BDE83840FFF7BABC2046FFF7C7
:100B000037FFF6E7C36870B504460D46C3B1FFF77B
:100B1000E7FF092D0CD8FFF75CFE0646FFF759FEEC
:100B2000801B8542FAD8E3682069BDE87040184709
:100B3000FFF74FFE29182046BDE87040FFF76EBF53
:100B400070BD00002DE9F04704460E4690461AB9E4
:100B5000BDE8F047FFF7D6BFFFF782FC63680746A2
:100B6000E3B9A368D3B9DFF83CA0FFF732FEDAF8A7
:100B700000508146FFF72DFE8145F6D8304408EB42
:100B80000502864288BF01326060A2602046FFF7FE
:100B90002DFE3846BDE8F047FFF76ABC2046FFF758
:100BA000E7FEE0E7F803002008B50121094800F05E
:100BB0009BFC0121084800F097FC0121074800F048
:100BC00093FC0121064800F08FFCBDE8084000F0CE
:100BD00021B900BF0D0C02400C0C02400E0C02406B
:100BE0000F0C02407047000008B50F4B1A680C4606
:100BF0009AB9012203281A6003D171460B480EF0FE
:100C0000DFF921460A480EF0DBF900F04FF90948F8
:100C10000EF0D6F908480EF0D3F9FFF721FCFFF7E4
:100C2000E1FFFFF7B1FD00BF040400206F0C0108D5
:100C3000730C01089B0C01088F0C010808B500F02B
:100C400085FF03480EF0BCF900F0E6FE002008BD69
:100C50009D0C010808B500F00BF9FCE71FB5FFF784
:100C6000FFFB0E4B0E481B68029300240D4B0093B4
:100C70000F220C234FF48071019400F055F80A4BB9
:100C80000A481B6802930A4B009307220C234FF477
:100C9000C061019400F048F8FFF7BAFB1802002089
:100CA00008040020550C00081C0200200805002044
:100CB0003D0C000808B5FFF7D3FB094B1B681A79F8
:100CC000082A07D95A79074B53F8221011B109683D
:100CD00043F82210FFF7CCFBBDE80840FFF79CBBB0
:100CE000E0020020E802002038B50B79082B03D978
:100CF00008490320FFF778FF4C7901F108020368E7
:100D00002BB113F8035CAC4201D31846F7E78B60B4
:100D1000026038BD5D0C0108031F53F8042F9A428E
:100D2000FBD0181A704700000F2A2DE9F74F05462F
:100D30008B4691469A462AD810F003031BBFC3F195
:100D40000403ED180B46CB1A303B23F003031AF0D3
:100D5000080F05EB030405D02A46A24203D2126015
:100D60000432FAE72D600193FFF77AFB2749019BD4
:100D70008046012251F8227016B25FB10132212A59
:100D8000F8D14046FFF774FB6FF08A003BE06FF04C
:100D9000150038E01D490C9841F822402A46E680AB
:100DA0000D99FFF7E3FA0E9B194AA3624FF0FF3348
:100DB000E3611368206001331AF0010F6562C4F823
:100DC0002CB084F805902771A760E7602761676100
:100DD000A7612762136004D001212046FFF746FA7D
:100DE0000DE00A212046FFF741FA1AF0040F06D160
:100DF0004046FFF73DFB4846FFF778FA02E04046E1
:100E0000FFF736FB304603B0BDE8F08F2803002023
:100E1000E402002008B501F009F900F0B9F8BDE8D6
:100E2000084000F01CB838B50446043000F01BFD43
:100E30000546204600F0FAFE284638BDF8B50446BF
:100E40000E461746051D3A463146284600F0F6FC88
:100E500020B90121204600F0B9FEF4E7F8BD08B53D
:100E6000002000F01BFA0120BDE8084000F016BA8F
:100E7000F8B50D4B1E68C6F307221D4622B9F4B221
:100E8000003418BF012400E00224FFF7E9FA2B68C0
:100E90009E42074602D12046FFF73EFC3846BDE899
:100EA000F840FFF7E5BA00BF200200202DE9F04F1F
:100EB0002C4B2D4A1B882D492D482E4EDFF8CCB0E7
:100EC0008BB00DF1280906F1800A29F8043D0EF0D7
:100ED00077F8FFF781FA0546FFF796FA0446FFF721
:100EE0008FFA2A46009023464FF4007122480EF0F4
:100EF00067F825EAE5754FF4007856F8044B14B30B
:100F00002779E26A5BF82730606A0793904406927B
:100F1000FFF702FF069AB4F90610079B101A226821
:100F20000592626A04920390E26A029262790192E7
:100F3000082FD4BF4F4609F1010700970544A26A64
:100F40000E480EF03DF8B245D7D10D4B02958DE815
:100F500008010C4A0C4819460EF032F80BB0BDE8F7
:100F6000F08F00BFF50C0108240D01082A0D0108BF
:100F70002F0D01082C030020770D0108C10D010879
:100F8000FD0D0108FF0D0108030E0108F80C010812
:100F900038B5FFF765FA1B4C0023E360054600F007
:100FA00037F84FF41443A360A268164B12F00C0FED
:100FB000FAD1154A40F20571116081221A601A684F
:100FC00042F480321A601A6812F4003F0D4AFAD0D7
:100FD0000E4B5360136843F0807313601168094B24
:100FE0008901FBD59A6842F002029A609A6802F081
:100FF0000C02082AFAD100F017F82846BDE838405C
:10100000FFF736BA00380240003C0240042A40078D
:10101000044B1A6842F001021A601A689207FCD564
:10102000704700BF00380240044B9A6812F00C0F62
:101030001EBF1A6822F001021A6070470038024091
:10104000034B044A00280CBF10461846704700BFE7
:1010500000BD010580DE800204281CD8DFE800F016
:1010600003080D1217000D4B1A6C1143196412E09E
:101070000A4A536C194351640DE0084A136B194333
:10108000116308E0054A536B1943516303E0034AB7
:10109000936B19439163BFF34F8F70470038024041
:1010A000042821D8DFE800F003090F151B000F4AC0
:1010B000136C23EA0101116470470C4A536C23EA54
:1010C000010151647047094A136B23EA010111635E
:1010D0007047064A536B23EA010151637047034A84
:1010E000936B23EA01019163704700BF003802400F
:1010F00038B514230C4A4343D4582568AA0608D5AA
:101100000A4B616803EBC002C9B253F83030506833
:1011100098472B0748BF6368054B1B681BB1BDE8A8
:101120003840FFF7C7BD38BD7C0E0108080B002012
:10113000D802002001282DE9F04780460D461746C9
:1011400003D92B490320FFF74FFDDFF8B090294A60
:10115000142404FB009442F83070E66802EBC002ED
:1011600001215360304600F0BFF9304600F080FAAC
:101170003046617C00F054FA4E464FB1D4F80890E6
:101180000021484600F0B0F9217C484600F048FABA
:10119000142303FB08F806EB080999F812A0D9F804
:1011A00004105046FFF758FF56F808400023E3604C
:1011B000504623616361FFF743FFB0FBF5F080B257
:1011C000A06077B199F8133001215AB203F01F03E0
:1011D00001FA03F35209084941F8223042F22C0384
:1011E00001E042F20803E3600020BDE8F08700BFA1
:1011F0005D0C0108080B002000E100E07C0E0108F6
:10120000012838B505D80E4C14230A4403FB0043CB
:1012100009E00C490320FFF7E7FC25682D06FCD503
:1012200011F8015B65608A4201D01C68F5E7142360
:101230005843034B1A5813685B06FCD538BD00BFF2
:101240007C0E01085D0C01080020FFF751BF012052
:10125000FFF74EBFF8B5104C04EB4014012167684E
:10126000384600F041F9A6680021304600F03CF90C
:10127000E5680121284600F037F9247D38462146EB
:1012800000F0CEF92146304600F0CAF92146284642
:10129000BDE8F84000F0C4B9B00E010801282DE9FE
:1012A000F041044603D910490320FFF79DFC0F4B82
:1012B000DFF83C80002543F820506401FFF7CAFFA7
:1012C00008EB04031E7F9F6930463946FFF7C4FED2
:1012D00058F8043039461D603046DD615D60BDE878
:1012E000F041FFF7DDBE00BF5D0C0108180B0020C8
:1012F000B00E0108012870B50C4621D84A1C22D036
:1013000021F0FF0313F5807F11D114F0FF041AD1EF
:101310000E4B03EB40152E69731C14D0012130468F
:1013200000F0E2F8297D304600F07AF906E001216C
:10133000204600F0D9F8204600F09AF9002070BD50
:101340004FF0FF3070BD6FF0010070BDB00E0108AE
:10135000042B2DE9F84304460E461546984603D95A
:1013600017490320FFF740FC1648DFF8609067013B
:10137000012100EB840000F029FC09EB07031C7F2E
:1013800099692046FFF768FE0F4B59F8071004EBE8
:1013900084041C4416F5807F14F8082045EAC20531
:1013A00045F004050D6015BF0B684B6843F44073AE
:1013B00043F0040314BF0B604B600020BDE8F883CA
:1013C0005D0C0108180B0020A40E0108B00E0108E6
:1013D0000B4A430110B50446D018D3588169007FE9
:1013E00000221A605A6822F004025A60FFF758FE81
:1013F000044800EB8400BDE8104000F017BC00BFBB
:10140000B00E0108180B00202DE9F843089E099F33
:10141000884691461D4623B91EB931490320FFF77E
:10142000E3FB304B400118F5807F1C58236843F0E4
:101430004003236005D0B8F1FF3F02D0404600F0E2
:1014400020F9A6B92F44AF4206D0A3689E07FCD569
:1014500015F8013B2373F6E7A3689807FCD5A3684A
:101460001906FCD4A368DA0720D5E368FAE70DB1C2
:10147000002319E030463744B84217D0A3689B07D1
:10148000FCD52573A368DE07FCD5237B00F8013B60
:10149000F2E7A2689007FCD5EA5C2273A268D10744
:1014A000FCD5227BF2540133BB42F2D1A3689A07E8
:1014B000FCD5A3681B06FCD4B9F1000F0ED1B8F11E
:1014C000FF3F0BD0236818F5807F23F04003236093
:1014D00004D04046BDE8F84300F0CAB8BDE8F88340
:1014E0005D0C0108B00E0108F8B50D460126C0F3E9
:1014F000832120F00F0400F00F0706FA01F102200B
:10150000FFF7AAFD07FA06F00323216883406FEA7C
:10151000030C01EA0C012160216805F0030E0EFAAC
:1015200000FE4EEA01012160E2680CEA0202E2607C
:10153000E168C5F3810282400A43E2606268BE400E
:1015400022EA060666606268C5F30015BD401543D1
:101550006560A2681343A3600020F8BD2DE9F04147
:1015600000F00F0415462B4A42F8343002EBC40257
:10157000069B536006468846C0F383274FF480419C
:101580000120FFF769FD41463046FFF7ADFF042C0F
:10159000214B03DCA11D01228A4003E0092C03DC5E
:1015A0004FF400021A6002E04FF480725A601B4B45
:1015B0000120996800FA04F2D243114099609968B9
:1015C00005EA000E0EFA04FE4EEA01019960D968A0
:1015D0000A40DA60C540DA68A54004F00C0404F162
:1015E000804404F59C341543DD6006F00302A568D1
:1015F00092000F21914025EA0101A160A168974066
:10160000B0400F43A76058611A681043186000206B
:10161000BDE8F081200B002000E100E0003C01402B
:1016200020F00F0300F00F02F0B51E6857000325ED
:10163000BD4026EA05051D601D680224072A04FA3C
:1016400007F444EA050494BF002201221C6003EB66
:10165000820300F007001C6A80000F22824024EA07
:1016600002021A621A6A814041EA02001862F0BD61
:1016700020F00F02012300F00F0003FA00F0906148
:10168000704720F00F0200F00F001030012303FA22
:1016900000F0906170470000104B2DE9F0415E6949
:1016A0001A680F4F164000244FF001081D4608FA33
:1016B00004F31E4206D06B6107EBC40357F83420D5
:1016C000586890470134102CF1D1064B1B681BB1B0
:1016D000BDE8F041FFF7EEBABDE8F081003C014003
:1016E000200B0020D80200202DE9F843124ADFF831
:1016F000508003010746D5582E69EB6800241E4030
:1017000008EBC0090223A3401E4209D0EA68D9F8B9
:10171000040022EA0303EB60214658F8373098476B
:101720000134042CEED1054B1B681BB1BDE8F84316
:10173000FFF7C0BABDE8F883F00E0108D802002018
:10174000A00B0020032910B516D80D4B00011C1862
:101750001B586068024001F10C0003EB80004260FE
:101760001869022202FA01F120EA01021A61DA681C
:101770001143D960002010BD4FF0FF3010BD00BFF5
:10178000F00E01080001024B1B58586A704700BF59
:10179000F00E0108034B00011A58136843F00103CF
:1017A00013607047F00E010801282DE9F843054643
:1017B000884630D81A4E1B490401371941F83020A9
:1017C00097F80C9001EBC00148464B60B968FFF7F1
:1017D00043FC36597B680024346048467460F362E9
:1017E000FFF72EFC104B7A7B13F809305843B0FBFF
:1017F000F8F3013BB36251B2012302F01F0273619F
:1018000049099340094A284642F82130FFF7C2FFB0
:101810002046BDE8F8834FF0FF30BDE8F88300BFF5
:10182000F00E0108A00B0020100F010800E100E0FD
:101830000020FFF759BF0120FFF756BF70B51346D0
:101840007BB18568C468A5420BD084680668651CB6
:1018500085604568013D2C40013B345D01F8014B3A
:10186000EEE7D01A70BDC368426830B584681B1BB0
:10187000934208D0C3680468013A5D1C1340C560F8
:10188000E154002030BD4FF0FF3030BD10B5154998
:10189000154840F2D243CB82002388B01A4606F0A6
:1018A00003FE002818DB02AC00944FF0FF337C22CB
:1018B0000E490D4806F05CFE002809DB23467C2219
:1018C0000A49094806F0C2FE0028ECDA084800E0A0
:1018D00008480DF0FFFBE6E707480DF0FBFB002092
:1018E00008B010BD24020020B00B00209A18002080
:1018F000380F01084C0F0108200F010830B589B0DE
:101900001822002102A80DF053FA0423029340F29A
:10191000D243ADF81E30BA238DF80C30AD238DF8CC
:101920000D30A5238DF80E3055238DF80F30172379
:101930008DF81A3036238DF81B3000250020FFF774
:1019400021FF184C1849206002AB0322174806F00B
:101950007DFE002802DA16480DF0BCFB0095154B01
:10196000154912487C2206F003FE002806DA74307E
:101970000CBF124812480DF0ADFB0DE00020FFF740
:1019800001FF21680F4B1860401A4FF47A7190FBE9
:10199000F1F10D480DF014FB002106480AF0CCF8D7
:1019A000CCE700BF540C00205E0F0108B00B0020F4
:1019B000610F010840420F009A180020770F0108BC
:1019C000800F01084C0C0020980F010884B030B53E
:1019D0008BB00FAC84E80E0000231A462146054662
:1019E00003F010FC58B928222146684607F0C0F9D8
:1019F0002A46014606480DF0E3FA012003E00548B7
:101A00000DF0DEFA00200BB0BDE8304004B07047A6
:101A1000A50F0108D70F010810B50821ACB03E484A
:101A200000F0F0FA08AC3D480DF054FB1022002104
:101A300020460DF0BDF9102200210CA80DF0B8F9D8
:101A400005A802F0CDFEBA238DF82030AD238DF825
:101A50002130A5238DF8223055238DF8233008231B
:101A60000093002206AB0221BDF9140002F0A4FC91
:101A70000028A4BF9DF818308DF82E304FF080025A
:101A8000A4BF9DF819308DF82F3021460CA80DF019
:101A9000F5F8002340222146BDF9140001F03CF87E
:101AA0009DF82E30172B2BD19DF82F30022B15D1FE
:101AB0000B9B009394E80E000120FFF787FF184B63
:101AC000029300230193174B009308231A464FF407
:101AD000C0611548FFF728F9144B0FE0362B0FD1E2
:101AE000134B029300230193124B00930622082309
:101AF0004FF4C0611048FFF717F9104B188002E04F
:101B00000F480DF0E7FA0F480DF0E4FA80220CA917
:101B10000D4807F03DFA00BF58120020FB0F0108E6
:101B200022100108FD1800089A12002098120020C7
:101B3000351001088D180008580C0020500C0020AA
:101B40004810010853100108140F010808B50020BF
:101B500007F0C4F9FEF73CFF03F06EF804F04EFE08
:101B600000F03EFC06F018FF00F006F801F05AF90C
:101B7000BDE8084003F0A2B913B50E4C0E490F485A
:101B80000AF046F80D49204602F06AFD002806DA00
:101B90000B48002102B0BDE810400DF011BA0094CE
:101BA000084B094802224FF4806102F0EFFD02B0B9
:101BB00010BD00BF701D002074100108181D00200A
:101BC0008C100108C61001081619002070B50546D2
:101BD0000C46FEF745FC2B6806462BB94FF0FF3349
:101BE0002B60FEF745FC18E0CCB10F4B1C680221BE
:101BF0002046FEF73BFB2B68013305D104F10803B7
:101C00002B600023A36003E021462846FFF76CF811
:101C10003046FEF72DFCFEF7FFFB012070BDFEF7FE
:101C200027FC204670BD00BFE002002070B50446CE
:101C3000FEF716FC256806461DB16B1C05D1002376
:101C40002360BDE87040FEF713BC28460A2150F817
:101C500008392360FEF70AFB236813B94FF0FF33FE
:101C6000236015F8034C3046FEF702FC2046BDE821
:101C70007040FEF73BBB0000F8B505460E46FEF788
:101C8000EFFB364B364A1B881BB2074652F823201F
:101C9000D2F820E0BEF1000F1AD054699369A34234
:101CA00016D9631C5361D3691C4046B9136933B913
:101CB000631C04D13846FEF7DBFB2046F8BD002C40
:101CC0000ADB0EEBC40393E8030085E8030004E09D
:101CD0004FF0FF34002EE9D0D560166976B3336833
:101CE0001361002C0CDB95695169D369691A8B4229
:101CF000A9BF691C4FF0FF351D4091610EEBC50572
:101D0000736893E8030085E8030016F8043C052B8C
:101D100009D0002373600A21A6F10800FEF7A6FA95
:101D200016F8034C00E00F243846FEF7A1FB0E2CFA
:101D300002D82046FEF7DAFA0120F8BD002C09DAB5
:101D400010460321FEF792FA3846FEF791FBFEF7A4
:101D500063FBF1E73846FEF78BFBEDE7DC02002082
:101D60002803002010B583694469C2691C1BA24284
:101D700001DA002010BD5C1C13408461F9D4026AB2
:101D800003C902EBC30383E80300012010BD000078
:101D90002DE9F8431E46264B53F82150254B1B884E
:101DA0000380074691462DB93046FEF761FB4FF0A0
:101DB000FF3439E02B79032B28D01F4B01462846EE
:101DC000D3F80080FFF7CEFF044638B13046FEF767
:101DD0004FFB98F80430052B25D122E0B9F1000F14
:101DE00003D13046FEF744FB1EE098F80430C8F8F3
:101DF0000C70052B0CBF052104214046FEF736FA76
:101E0000414605F11000FEF76FFF07E003C8EB68DD
:101E100083E803000A212846FEF728FA3046FEF739
:101E200027FBFEF7F9FA01242046BDE8F88300BF3E
:101E300028030020DC020020E002002038B5044620
:101E4000FEF70EFB074B1B882380074B21460546F8
:101E50001868FFF787FF04462846FEF709FB20466F
:101E600038BD00BFDC020020E002002008B50F4BA7
:101E700053F82130B3B1212202801A79032A0BD101
:101E800003C8DA6882E8030018460A21FEF7EEF973
:101E9000074B0120186008BD01461846BDE8084000
:101EA000FFF760BF4FF0FF3008BD00BF28030020E0
:101EB000D802002070B504460D46FEF7DCFA28B1C2
:101EC00029462046BDE87040FFF7D0BF094B1B886C
:101ED0001BB29D4204D12046BDE87040FFF7AEBF63
:101EE000FEF7BEFA2946034601222046BDE87040AF
:101EF000FFF74EBFDC02002070B504460D46FEF72A
:101F0000BAFA064628B129462046BDE87040FFF7D8
:101F1000ADBF0A4B1B881BB29D4204D12046BDE8D1
:101F20007040FFF78BBFFEF79BFA32460346294607
:101F30002046BDE87040FFF72BBF00BFDC02002049
:101F40002DE9F041124F3B881BB2934206460C46E6
:101F5000154603D10F490320FEF746FEFEF780FA2F
:101F60003A880D4B12B2804653F82270052138464C
:101F7000FEF77CF996E80300FC60434684E8030022
:101F8000012229462046BDE8F041FFF701BF00BF0E
:101F9000DC0200205D0C01082803002070B5044617
:101FA0000D46FEF75DFAB4F90020114B53F82240BC
:101FB00006461CB90F490320FEF716FE2379052BB0
:101FC00004D0FEF755FA4FF0FF3070BD95E80300DE
:101FD000E36883E803000A212046FEF747F96479A5
:101FE0003046FEF745FA2046FEF780F9012070BD25
:101FF000280300205D0C01080021FFF73DBE0121F0
:10200000FFF73ABE08B5074B4A1E1B68114018621D
:1020100003D005490320FEF7E7FD59619961DA61B4
:1020200008BD00BFE00200205D0C01080F4BD3F893
:10203000882042F47002C3F888200D4A9A6010226A
:1020400083F822200021DA7701F1604000F5614039
:102050000131522980F80023F6D11A6942F01002AA
:102060001A615A6942F400725A61704700ED00E04B
:1020700000000008034600201BB1DA685B681044CA
:10208000FAE7704710B50822094904460CF0C4FD70
:1020900048B12378FF2B08D1607800F00F00831E31
:1020A0005842584110BD012010BD002010BD00BF96
:1020B00028110108002102F0CDBE38B5CBB20021B5
:1020C00014460246084602F0A1FB054618B9204610
:1020D000FFF7F0FF0FE094F9103001330AD1A36845
:1020E00082681B7903F03F0321462046137102F0FA
:1020F00071FC04466C60284638BD00002DE9F047AD
:102100008C680746104688461546FFF7B3FFA3794B
:1021100040BAFF2BA0800AD12B7C023BDBB2022B02
:1021200003D8214AD35CFF2B00D13B23A371E37971
:1021300043B90FB9402304E0384600F0CFFC90F8D3
:10214000CA31E37104F108061022184930460CF038
:1021500063FD8246D0B904F118091549102248469A
:102160000CF05AFD014630B9102230460CF020FE2A
:102170000123E3750AE049465246384600F088FDDF
:10218000014618B1102230460CF078FD4146284631
:1021900002F0DAFB002804DA831C08BF0020BDE847
:1021A000F0870020BDE8F087D5100108381101083C
:1021B000881101088B6870B558800C46054600F000
:1021C0008DFC014618B919490320FEF70DFD66681C
:1021D0003046FFF74FFFB1F8C831984204D9204686
:1021E000BDE87040FFF766BFD1F81C320133C1F87B
:1021F0001C323046FFF73EFFD1F824321844B1F8C4
:10220000C631C1F82402DB0708D5234640F202227A
:102210000749012002F07CF830B9E0E72146284662
:1022200002F0AFF80028DADD70BD00BF5D0C0108D8
:102230000000FFFF2DE9F04F85B090F91030013319
:1022400000AF044689460AD18368B3F9026002F000
:102250000FFE00286AD043680446984601E0804695
:102260000026404602F004FE054600285ED04445A4
:10227000836818BF60601A461B7ED0F8048008BFD0
:102280000446FF2B2BD186B907F1080002F0A8FA0B
:1022900000284BD0002122460846B7F90860FFF716
:1022A0000CFF0446002800F09380B9F1000F06D01F
:1022B000424629463046FFF721FF002836DBA26858
:1022C000137943F040031371304600F05FFE43681A
:1022D0000133436021463046FFF76CFF78E0134638
:1022E000183310223C4918469B460CF095FC40B12F
:1022F0005946002E39D1381D00F06EFC06460028E4
:1023000038D0B9F1000F06D0424629463046FFF7D3
:10231000F5FE00280ADB2846FFF7ACFE0021024646
:102320000223084602F0A4FC064608B9204619E03C
:1023300083689846EA68A96840460CF09FFCEB6801
:102340006D6842461A449046002DF3D12046FFF7AF
:10235000B1FE224B3146B3F9000002F01FF800280D
:1023600036DC3046FFF7A6FE32E0304600F00CFCCB
:102370000028C6D107F11001082301F80D3D3246AF
:102380005B4607F1080005F0E1FCEA46064640B16D
:10239000B9F1000F09D042462946FFF7AFFE0028E9
:1023A00003DA2046FFF786FE11E02246F97807F1AE
:1023B0000800FFF782FE044648B1304600F0E6FD13
:1023C00003680133036021463046FFF7F3FED5462C
:1023D0001437BD46BDE8F08F88110108B41D0020F8
:1023E0001FB50F4CB4F9003063B90E4A01930E4B80
:1023F00002920093042208234FF480610B48FEF7F9
:1024000093FC20800A480B4B0360012303711423C3
:1024100083600AF02AFEB4F9000004B010BD00BFCA
:10242000B41D0020D0100108D9260008B61D0020D8
:10243000801D0020B8210020292B2DE9F84381467A
:102440000F4614461D4606D03A2B06D0112B0CBF62
:102450000423002302E0022300E00323292D3B7420
:1024600001D03A2D03D1A74259D1012605E0A74258
:1024700002D063689F4252D100267B6893F9100016
:10248000022805D016B30121204602F0D1FC1DE040
:10249000294602F03DFA18B986F0010836B101E08C
:1024A0004FF000080121204602F0C2FC234640F212
:1024B00001221E4997F9100001F02AFF10B92046A9
:1024C000FFF7F8FDB8F1000FDCD00AE0234640F238
:1024D00001222946022001F01BFF10B92046FFF718
:1024E000E9FD06B3292D07D03A2D18D121464846DB
:1024F000BDE8F8430AF020BF00232374616839B1B6
:1025000091F91030022B03D1204602F063FAF5E76F
:10251000022323742046BDE8F84300F00BB80449B9
:102520000320FEF761FBBDE8F88300BF0000FFFF5A
:102530005D0C01082DE9F047044618B964490320F1
:10254000FEF752FB4FF0FF3102F00FFA0546A0B143
:102550008368B3F90260002EF0D0304600F016FD1B
:1025600043690133014643612046FFF783FDEA6872
:102570008B699B1A1844886100E006462746254669
:1025800095F91030022B08D1EB68282B05D1AB68E8
:102590001B7803F0F003602B08D0D5F804802F4699
:1025A000B8F1000F6ED04546EAE73C46D5F8088002
:1025B000E368B8F8041049BA89B2994203D22046B8
:1025C00002F0DEFB0FE022460023D068034492F9BC
:1025D0001000022803D1283B994204D95DE05268DB
:1025E000002AF2D1F7E708F11809102239494846C4
:1025F0000CF012FB002855D04846FFF743FD494632
:1026000000B136B9002000F0E7FA002E08BF0646F8
:1026100002E0304600F0B8FAB0FA80F04009002835
:1026200040D008F10800FFF72DFDB0BB4846FFF78A
:1026300029FD90BB98F80730013BDBB288F80730E2
:102640005BB3284602F014FC38B34FF0FF3120464C
:1026500002F08BF9014610B1204602F0BBF9214689
:102660000025084602F004FC18B92846FFF722FDB1
:1026700013E04168456005460029F2D1BDE8F04706
:10268000FFF7D8BDA3681B7803F0F003602B04D1DB
:10269000204602F0EDFB074668B92046BDE8F0474A
:1026A000FFF708BD98F80630224639463046BDE8A7
:1026B000F047FFF7C1BE0222282102F0F3FA87F8A3
:1026C0001080054600287FF470AF3846E6E700BF6B
:1026D0005D0C01088811010810B5102298B00DEBAF
:1026E000020000210CF064FB504B0593504B082175
:1026F0001B88ADF81C3008A8FFF784FC04A9022051
:1027000002F0BAF840F20523ADF80A30002468461A
:10271000FFF775FCBDF802306FF400721344222BF2
:10272000F5D801A252F823F0B5270008BD2700080C
:10273000C7270008C72700080F2700080F27000831
:102740000F2700080F2700080F2700080F27000891
:102750000F2700080F2700080F2700080F27000881
:102760000F270008D72700080F270008E3270008D5
:102770000F2700080F2700081B2800080F27000854
:10278000EB2700080F2700080F2700080F27000875
:102790000F2700080F2700080F2700080F27000841
:1027A0000F270008F3270008FB270008032800086C
:1027B000132800080198FFF7BDFEA8E70121019842
:1027C000FFF738FDA3E76FF0850302A9684603937E
:1027D000FFF7E4FB9BE7019A537E23F0080353764F
:1027E00095E7019800F044FF91E7019800F0CEFFD3
:1027F0008DE7019805F024FA89E7019805F076FA4B
:1028000085E7019B587C00F00F0004F063F8047426
:102810007DE7019805F0D0FC79E7019A002319467D
:10282000B2F91A0001F012FB71E700BF0000FFFFD0
:10283000DC0200200121FFF7C9B92DE9F84300F5BA
:10284000E075074628468846FFF7F4FF00244FF05E
:10285000380909FB04764146304606F022FA38B1C1
:102860001022002130460CF0A3FA0023337402E05A
:102870000134082CEDD12846BDE8F843FFF7D6B95E
:1028800008B5102203490CF0C7F9B0FA80F04009EE
:1028900008BD00BF3811010810B5082209490446D7
:1028A0000CF0BAF948B12378FF2B08D1607800F01A
:1028B0000F00831E5842584110BD012010BD00205A
:1028C00010BD00BF281101082DE9FF47002605466D
:1028D0008846924699463446AF194146384606F036
:1028E000E0F900287FD13846FFF7CAFF10B1002C6D
:1028F00008BF3C463836B6F5E07FEDD12746002CC0
:1029000071D01022414620460CF0B8F9237884F8A3
:1029100011A0FF2B84F8109016D0B5F8C631DA0755
:1029200012D501F0E1F8814670B105F5E076304648
:10293000FFF77CF9B5F9C4014B464A46214601F040
:1029400083F93046FFF776FF98F80030FF2B04D16B
:10295000237C43F00103237441E04046FFF79CFFD2
:102960008146C8B9B5F8C62102F00602062A17D179
:1029700005F5E0763046FFF759F9B5F8C631DB07C3
:1029800006D54B464A464946B5F9C40101F05EFA00
:102990003046FFF74FFF03E0237C63F07F0323748F
:1029A000B5F8C63103F00303012B18D040F2FF2223
:1029B0000023CDE900234FF080730293FF238DF8AD
:1029C0000C3098F80D308DF80D30B8F80E30ADF8A9
:1029D0000E308022002369462846FFF775FF40F23B
:1029E000112363866463384604B0BDE8F08703882A
:1029F0005BBA23F03F031B041B0C4FF6C0629342EB
:102A000009D00378FF2B08D1407800F00F0005288B
:102A100018BF0E207047052070470E2070472DE923
:102A2000F0470025804691461F460C462E464FF043
:102A3000010A3FB13A780AFA05F31A421AD0237C08
:102A4000DB0717D42046FFF71BFF98B949462046FD
:102A500006F03CF937B999F80030FF2B02D0637CBF
:102A6000834207D8B04205D9B8F1000F01D0C8F8A9
:102A7000004006460135082D04F13804D9D130460E
:102A8000BDE8F08770B5134CB4F9C451A8420646AE
:102A90001ED0EDB904F5E070FFF7CCFE4FF4A06353
:102AA000A4F8C831402384F8CA31A4F8C4612B4685
:102AB000A4F8C651802208492046FFF705FF04F517
:102AC000E070FFF7B3F82046BDE8704000F06CBE40
:102AD00070BD00BF3824002058110108034BB3F922
:102AE000C42182420CBF18460020704738240020C1
:102AF000B0F8C631DA0707D511B143F0020301E09F
:102B000023F00203A0F8C6317047B0F8C631DB07E6
:102B100001D505F011BB70472DE9F0410D46174670
:102B20009846FFF7DBFF044610B90020BDE8F081AE
:102B30000029FAD00846FFF7A3FE0028F5D1802F20
:102B4000F3DC04F5E0763046FFF774FE43463A4680
:102B500029462046FFF7B8FE04463046FFF766F8E0
:102B60002046BDE8F081000010B520B90548B0F955
:102B7000C43133B101E0FFF7B1FFBDE81040FFF70A
:102B80005CBE10BD382400202DE9F8438946FFF7CC
:102B9000A5FF0446E8B100F5E0763046FFF74AFEAF
:102BA000002504EB05084946404606F07AF807463A
:102BB00028B13046FFF73AF84046BDE8F88338358B
:102BC000B5F5E07FEDD13046FFF730F83846BDE887
:102BD000F883BDE8F883000038B5084C0546B4F921
:102BE000C4011DB9FFF7D0FF20B938BDFFF7CCFFF6
:102BF000286008B1B4F9C40138BD00BF38240020F2
:102C00002DE9F34102AD00260E4C45F8046D8846CF
:102C1000074604F5E070FFF70DFE334642462146B5
:102C20002846FFF7FCFE20B1019B3B60B4F9C4418C
:102C300000E004460448FEF7F9FF204602B0BDE874
:102C4000F08100BF38240020F82500202DE9F34151
:102C500002AC0027884644F8047DFFF73FFF00F5EB
:102C6000E07506462846FFF7E5FD20463B4642460E
:102C70003146FFF7D4FE044628461CB1FEF7D6FFC6
:102C8000019802E0FEF7D2FF204602B0BDE8F081D5
:102C90002DE9F04F87B00F461546FFF71FFF00F5EF
:102CA000E073804618460193FFF7C4FD012200211E
:102CB00002A80CF07DF84646C3464FF0FF3A0024C8
:102CC0004FF001099BF80020FF2A12D05846FFF769
:102CD000D7FD70B945B99DF8081009FA04F20A4306
:102CE0008DF80820A24604E05846FFF7D5FD0028DD
:102CF000F1D10134082C0BF1380BE3D1BAF1FF3FCD
:102D000000F0878004AD2246002128460CF050F8E0
:102D10003B78FF2B04D197F8019009F00F0309E0ED
:102D20003846FFF7B9FD20B93846FFF760FE00903E
:102D300001E0022300934FF000094C469DF8081073
:102D4000012303FA04F2114232D039463046B34629
:102D500005F0A7FF002855D13046FFF79DFD18B9B3
:102D60003046FFF744FE00E00220009B834208D17A
:102D70002A5D0432D2B22A554A4588BF4FF0040971
:102D80000AE009D92A5D0232D2B24A4513462A55D1
:102D900038BF4B465FFA83F9B2694AB12A5D013206
:102DA000D2B24A4513462A5538BF4B465FFA83F9DB
:102DB0000134082C06F13806C0D10122002102A8F6
:102DC0000BF0F6FF00209DF80820014601246E5C00
:102DD0004E4504BF04FA01F0024301F1010104BFB2
:102DE000D2B201200829F2D108B18DF8082006A836
:102DF000002340F80C3D3A4602AB4146FFF70FFE78
:102E0000DDF80CB0BBF1000F05D1382202FB0A8BB4
:102E100001E04FF0000B0198FEF708FF584607B09D
:102E2000BDE8F08F2DE9F04F8DB005A801F0D8FC7A
:102E30000026544F03900DF11205B146039B9E42AC
:102E400000F09D8035F9020FFFF748FE0446002888
:102E500000F0918000F5E07A5046FFF7EBFC01238B
:102E6000B5F90000009300220DF1130317218DF82E
:102E7000139001F0A1FA86302CD09DF91330012B6C
:102E800028D108230DF13008ADF818304FF6FF7344
:102E900028F8103DB7F8C631B5F9000043F0030338
:102EA0004FF0020BA7F8C631002206AB0521CDF882
:102EB00000B001F0A7FAB5F90000CDF800B011217B
:102EC0004346002201F078FABDF82010B5F9000061
:102ED00005F0BEFA4FF00808B5F90000CDF8008003
:102EE00006AB0022414601F067FA00280FDB42469C
:102EF00006A90AA80BF0C2FE4246234908A80BF017
:102F0000BDFE0023402208A92046FFF7DDFC022376
:102F1000B5F90000009300220DF11603112101F014
:102F20004BFA002806DBBDF81630B3F5A06F28BFBA
:102F3000A4F8C83100231A462421B5F90000CDF8C1
:102F4000009001F039FAB4F8C6310028CCBF43F044
:102F5000800323F08003A4F8C6315046FEF766FED6
:102F600001212046FFF7C4FDB4F8C631DB0702D5C6
:102F7000204604F02DFE013607F50C775EE70DB014
:102F8000BDE8F08F382400202811010808B5FFF7AC
:102F9000A5FD00F5057008BD2DE9F34107468846FB
:102FA00016461C460AF08CFB054640B903230093E5
:102FB0003246A3B2414638460AF014FB20E0437E75
:102FC00003F00703012B01D103210DE0027EA3B220
:102FD0009A4200F110070CD031462C762246384632
:102FE0000BF04CFE0321284602B0BDE8F04100F092
:102FF0008FBE2246394630460BF00EFE0028EBD13C
:1030000002B0BDE8F08100002DE9F04F1D46D379F4
:1030100091B0FF2B8046069116461A9F40F0B4806F
:103020006B78002B40F0B080172F40F2AD802B7AE8
:10303000FF2B00F0A98002F10809554910224846EB
:103040000BF0EAFD70B105F108014046FFF79CFD69
:103050000590002800F098800023183F1C46194670
:103060009A461BE00D224B4906F118000BF0D4FDE7
:10307000002800F08980E6E70AF1180205EB020B50
:10308000AA5C012A0DD0212A08BF5C469BF80120CA
:103090000AEBC20A1FFA8AFAA7EBC207002FEBDC81
:1030A0000BE008AB2A780698009331465B4601F0A6
:1030B0000DF8031E68DB5946E8E740460793069182
:1030C000FFF70CFD0699079B18B933490320FDF75C
:1030D0008BFD08AA002942D0002C40D0B0F8C611C0
:1030E00001F0030103293AD12978029301924B465A
:1030F0000A4600943146404604F018FF002304F1CC
:1031000008020F21074604F0F7FE054617B9102202
:10311000494620E0237A83F002038DF82830637A51
:103120008DF82930A37A8DF82A30E37A8DF82B3088
:10313000237B8DF82C30637B8DF82D30A37B8DF8AD
:103140002E300822E37B8DF82F300AA90EA80BF051
:1031500095FD124908220CA80BF090FD09E04946A4
:103160004046FFF719FF102249460CA80BF086FDD8
:103170000025337E0095A3F1FF0253425341059988
:103180000CAA404600F0D4FC11B0BDE8F08F00BF9F
:1031900038110108681101085D0C010828110108A7
:1031A0002DE9F04F89B003F108099246059149468F
:1031B0001D468046129E0AF083FA9AF80730FF2BCC
:1031C00040F0B5806C78002C40F0B180172E40F2B2
:1031D000AE802B7AFF2B00F0AA80002800F0A78099
:1031E000183E2746002E27DD07F1180305EB030BD9
:1031F000EB5C022B0DD0212B16D1002302930193FF
:103200002A78CDF800B04B465146404604F08EFE79
:103210000AE006AB00932A7805985B46514600F019
:103220009CFF041EC0F283809BF8013007EBC307AC
:10323000BFB2A6EBC306D5E74FF0FF31059801F00A
:1032400094FB08B1876800E00746494640460AF00B
:1032500037FA064600286AD0437E03F00703022BA4
:1032600012D127B13B7813B17B78002B31D106A95D
:10327000A6F81A803476224606F110000BF0FEFC08
:103280002B79590616D512E01FB13B780BB17B782C
:1032900013BB002C49D1377E003718BF01272B798B
:1032A0009A062AD44FB3A4BB2B795B0601D507211C
:1032B00001E01FB10321304600F02AFD95F90430EA
:1032C000002B737EB4BF43F0080323F0080373762A
:1032D0002DE0002CCBD12AE02CB3337E9C4209D0C8
:1032E000224606A906F110000BF096FCB0FA80F019
:1032F000400900E000200746D1E7002CD4D0A6F812
:103300001A803476224606A906F110000BF0B6FCAE
:10331000CAE7737E03F00703072B08D10321304669
:1033200000F0F6FC03E02746B9E70027B7E709B04D
:10333000BDE8F08F2DE9F04F87B0154698468146DD
:103340000291109FFFF7CAFBB0F8C6319A070646F4
:1033500069D5EB79FF2B66D198F80140002C62D13A
:10336000072F60D905F10803083F0DF1100A0393F8
:10337000002F1FDD04F1080308EB030B18F80330DE
:10338000012B0FD198F800200298CDF800A05B46E1
:10339000294600F09BFE031E45DB52460399484632
:1033A000FFF7FAFD9BF8013004EBC304A4B2A7EBCE
:1033B000C307DDE7B6F8C63113F0040F05F10805C1
:1033C00028D013F0010F194B194C18BF1C4605F0FB
:1033D0008BFD06F5FC7780463846FDF781FBB6F895
:1033E000C631DB0716D5294648460AF069F988B187
:1033F000B8FBF4F140F21523A6F80E320D4BC6F8D7
:103400001002B3F9003006F5037204FB118138464F
:1034100008F0BCFB294648460AF052F918B1437E31
:1034200023F00803437607B0BDE8F08F80841E00C8
:1034300020A10700B41D00202DE9F04F89B092466D
:10344000059181461E46FFF749FB0AF1080B054628
:103450000822844958460BF0DFFB002840F0FF802B
:103460009AF80830FF2B00F0FA809AF80730FF2B0B
:1034700040F0F5807378002B40F0F180129B0F2B09
:1034800040F2ED80594648460AF01AF9074650B90D
:103490000B23009302460346594648460AF0A2F819
:1034A000074668B9DBE0437E190706D5F28852BAB1
:1034B00092B212B923F0080301E043F008037B76CF
:1034C000F3889CB264B15CBA674B68491B88A4B2AC
:1034D0001BB207F13002614307F11C0008F056FBF4
:1034E00033790BB185F8CA31B5F8C631C3F30D0293
:1034F000A5F8C62173791B0203F440431343A5F8D2
:10350000C631B068A8B1D5F8D03190FA80F89845A6
:103510000FD005F0E9FC0A22B0FBF2F303FB120026
:10352000053008FB00F0C5F8D081B0FBF2F0C5F81B
:10353000D401F36813B11BBAC5F8D83105F5E070B2
:10354000FEF774FB129B103B03930023029304933A
:10355000039B002B58DD029B103306EB0308F35C42
:10356000052B1CD004D8012B0DD0032B1ED03FE01F
:10357000222B2AD0232B3BD14346129A3146484670
:1035800004F052FE34E006AB0093327805984346CF
:10359000514600F09BFD031E049329DA5FE042468A
:1035A0003178484600F013FE10BB58E042463178AF
:1035B000484600F029FE002851D0D8F804301BBA44
:1035C000B3B19C4228BF1C4612E04146307804F05B
:1035D0007FFD002843D0B8F806305BBA9BB23BB100
:1035E0003C22B4FBF2F2934202D23C2202FB03F4EF
:1035F00098F80130029A02EBC30292B20292039A47
:10360000A2EBC3030393A3E7049B06AA59464846CB
:10361000FFF7C2FC05F5EE70FDF762FAB5F8C631AA
:10362000DA071CD504EB4404042C88BFA1084FF032
:10363000000498BF0121384685F8CB4104F030FCE6
:103640003B463A462146B7F91A0000F0FDFAB5F8B4
:10365000C6319B0703D501212846FFF756FA09B06A
:10366000BDE8F08F28110108DC02002040420F0065
:103670002DE9F041437E03F00703022B86B0044698
:1036800001D0052B7BD194F89420B4F91A50012A6B
:1036900071D9022B11D14FF080730493FF238DF861
:1036A0001430637B8DF8153040F2FF200021E38950
:1036B000ADF81630CDE902010BE094E8030002AB4F
:1036C00083E8030004F1080393E8030006AB03E971
:1036D0000300013A84F894201DBB01AE304601F08E
:1036E0007FF80746BD4208D036F9150002AB2246E6
:1036F000002100F0A9FA0135F4E7224B04F1380566
:10370000B3F900602846FDF7EBF940F21223A4F864
:103710004E3004F14C0233461B49284608F036FA75
:103720002DE02846FFF7DAF90646224602AB06F5F9
:10373000E075B4F91A00002100F086FA012128464C
:10374000FEF744FA0F4BD6F8D871B3F9008004F1B4
:1037500038063046FDF7C4F940F21223A4F84E3083
:103760003046434604F14C02394608F00FFA284629
:10377000FEF75CFA03E02146284609F0C9FF06B0CF
:10378000BDE8F081B41D002040420F00437E03F0ED
:103790000703042B03D0072B04D1032100E00521EC
:1037A00000F0B6BA7047000038B500F5E075044681
:1037B00001212846FEF70AFA05F096FB0A210A4B7A
:1037C000B0FBF1F202FB11000530C4F8D0314343E5
:1037D000B3FBF1F3C4F8D431044BC4F8D831284614
:1037E000BDE83840FEF722BA80C3C90140420F004D
:1037F00010B5044608462378FF2B14D00022182366
:10380000872109F003FE002270B183681A715A7192
:103810009A71DA7121686268DA609960A168E26879
:103820005A61196110BD002010BD38B50B78FF2B0F
:1038300005460C46104616D000221823882109F0B0
:10384000E5FD002280B1836825F01F051D71DA7146
:103850009A715A7121686268DA609960A168E268B9
:103860005A61196138BD002038BD08B5002208230F
:10387000852109F0CBFD28B1836800221A715A71A5
:103880009A71DA7108BD10B5002304461046CA1DAE
:1038900002F0F802194601F0EBF920B182681470C9
:1038A000C368DB08537010BDF8B516460F461A46BC
:1038B000B11CFFF7E8FF044660B18568C2680235B5
:1038C000023A002128460BF073FA32463946284660
:1038D0000BF0D4F92046F8BD13460A4601460120F4
:1038E000FFF7E2BF13460A4601460220FFF7DCBF9E
:1038F0002DE9F04180460F4616461D460022102352
:103900008621079809F082FD60B1069B846827F044
:103910003F0776BA2DBA1BBA84F804806771E68037
:10392000A560E360BDE8F0812DE9F04107468846D7
:1039300016462021079A03201C46FFF7A4FF0546E0
:10394000C8B1806824BA0021846028F03F0800F1E3
:10395000100436BA017341738173C173877080F8A4
:1039600003804660102220460BF022FA3A46069960
:10397000204605F0D1F92846BDE8F08110B50A4689
:10398000044608210520FFF77EFF28B18368002246
:1039900024BA9A70DA705C6010BD000008B510227D
:1039A00003490BF039F9B0FA80F0400908BD00BFB7
:1039B0003811010810B50822094904460BF02CF90A
:1039C00048B12378FF2B08D1607800F00F00831EE8
:1039D0005842584110BD012010BD002010BD00BF4D
:1039E0002811010870B506460846194609F098FDE9
:1039F0000446A0B18368FF22DA7100231A461946F3
:103A0000184600F003FF054620B92146204600F085
:103A1000E1FF02E083685E804460284670BD70BDAF
:103A2000002101F017BA0000F7B51F46537C802B28
:103A300005460E46144603D911490320FDF7D4F874
:103A40001046FFF7ABFF08B1002017E02046FFF754
:103A5000B1FF0028F8D1217CCB07F5D43388607CF6
:103A6000626913F0010F14BF002680268DE89000D4
:103A7000A3693143FFF758FF2860012003B0F0BD70
:103A80005D0C010830B585B0022300930D460DF1A1
:103A90000E0300220521044600F08EFC002803DB03
:103AA000BDF80E30062B10D80823009300222B46B9
:103AB0000221204600F080FC002802DBADF80E0059
:103AC0000EE00023ADF80E300AE008230093002238
:103AD0002B460321204600F06FFC0628E4DDEDE7CD
:103AE000BDF80E0005B030BD38B5002009F032FE3B
:103AF000044658B1637E03F00703013B012B03D951
:103B00000A4B00221A600EE02046EFE7074D2868B6
:103B100009F020FE034618B909F01CFE034610B157
:103B20002B60184638BD204638BD00BF68260020EF
:103B30002DE9F7430A9C0F46994680461646FEF744
:103B4000CDFFB0F8C631990701D4002507E0404603
:103B5000FEF7C4FFB0F8C6315A07F6D580253046C7
:103B6000FFF71CFF38B11022334930460BF086F8BE
:103B70000223737001E045F04005B9F1000F0BD04E
:103B800069464046FFF77EFF30B1C1B22246684623
:103B9000FFF7A8FE68B1044624B13B7CDB0758BFA1
:103BA00045F02005224639462846FFF73EFE81466D
:103BB00008B920463BE00146002332464046FFF765
:103BC00011FF054608B9484631E03B7CDFF87490A8
:103BD00013F0010F23D005F087F9184BB0FBF3F772
:103BE000314607FB1307404609F06AFD044618B941
:103BF00013490320FCF7F8FF00F154063046FCF7A8
:103C00006FFF40F20223A4F86A30E566B9F900308C
:103C100004F168023946304607F0B8FF09E0014672
:103C2000B9F9000000F0ADFB002802DC2846FFF7E0
:103C3000F7FE03B0BDE8F0834811010840420F00D1
:103C40005D0C0108B41D00202DE9FF4707460D4615
:103C500090469946FEF742FF824618B92A4903204A
:103C6000FCF7C2FF35B92A4641463846FFF710F83F
:103C7000054668B102A93846FFF704FF064650B171
:103C8000C1B2002202A8FFF727FE044620B935E0A2
:103C90000646044600E00446BAF8C631DB0714D5F0
:103CA000082E0AD00823009300226B4403213846D3
:103CB00000F082FB80B208281FD1234602AA0F2100
:103CC000002004F019F9C0B1044621464046FFF730
:103CD0008FFD064688B101462B464A463846FFF717
:103CE00081FE044608B9304608E0084B0146B3F9A6
:103CF000000000F046FB002802DC2046FFF790FEA3
:103D000004B0BDE8F08700BF5D0C0108B41D0020C1
:103D10002DE9F041437E23F007030B4305290446B8
:103D2000437620D0072903D004294BD1264E05E045
:103D3000B0F91A00FEF7D2FED0F8D461234B04F19B
:103D40003805B3F900702846FCF7CAFE40F2172385
:103D5000A4F84E3004F14C023B4631462846BDE8FB
:103D6000F04107F013BFB0F91A00FEF7B7FE0323C6
:103D70000646224606F5E07584F89430B4F91A0038
:103D800023460021FFF760FF01212846FDF71EFFB3
:103D90000E4BD6F8D871B3F9008004F138063046DE
:103DA000FCF79EFE40F21223A4F84E303046434604
:103DB00004F14C02394607F0E9FE2846BDE8F0411F
:103DC000FDF734BFBDE8F081404B4C00B41D00202E
:103DD0002DE9F3411B4D002918BF0D46002229464D
:103DE0008046FEF755FF074670B169464046FFF72B
:103DF00049FE38B1C1B200226846FFF76DFD0446A6
:103E000018B91AE0044600E004462046FFF72DFDED
:103E1000064688B101463B462A464046FFF7E2FD8A
:103E2000044608B9304608E0074B0146B3F90000E4
:103E300000F0A7FA002802DC2046FFF7F1FD02B0EF
:103E4000BDE8F08178110108B41D00202DE9F04F84
:103E50008BB0002791468A46039302900797FEF79E
:103E60003DFE964B064600F5E07801214046B945F7
:103E700008BF9946FDF7AAFEB6F8C65115F0010530
:103E80001BD1344606F5E377B3465C4500F0ED8080
:103E9000627C9BF811309A4240F0E48059462046FB
:103EA00004F014FF637C834200F2DC8000E01D46D6
:103EB0003834A045E8D1079D4FE004F06DF9054680
:103EC00000284AD0846906F5E37BECB163689E4222
:103ED00018D1AB699C4200F0D780A268996892F82B
:103EE00011E0487C864540F0E3801046059304923B
:103EF00004F0ECFE049A059B527C824200F2D880CA
:103F000000E01F462468E0E74FF0010B05EBD40307
:103F10009A7D04F007030BFA03F31A420CD0E0B2C7
:103F200002F0D8FC428A417C0346007C009704F0F2
:103F30004DFA079060B107460134102CE6D12A46AD
:103F4000A98A28693B4604F067FA0546079020B91C
:103F50004046FDF76BFE384681E0B6F8C6311B07D8
:103F600007D52946B6F8C801FFF708FD0790F8B154
:103F70000546BAF1000F0FD14046FDF757FE4946FE
:103F800001220298FEF784FE012182464046FDF799
:103F90001DFEBAF1000F10D008A90298FFF772FDBC
:103FA00058B1C1B22A4608A8FFF796FC079018B985
:103FB0004046FDF73BFE3DE00546B6F8C62102F05F
:103FC0001004A4B20CB196F8CA4102F020039BB2CF
:103FD0004BB1D6F8D4313A498B4206D84FF47A7BAC
:103FE000B3FBFBFB03E09B4601E0DFF8DCB002F033
:103FF0004007BFB22FB1D6F8D8714FF47A73B7FB30
:10400000F3F7039B13B9B6F8CC2100E00022404639
:104010000392FDF70BFEB6F8C611039A019509123B
:10402000204600975B4601F0C001FFF761FC0446A3
:10403000079008B9284612E0014653464A460298BE
:10404000FFF7D0FC0146079008B9204607E01D4B5A
:10405000B3F9000000F095F900282BDC0798FFF772
:10406000DFFC27E00BF1380B0FE72B4622463946E1
:1040700007A8FFF7D9FC00283FF41AAF079B002BD5
:104080007FF415AF28460DE03B46A268594607A8C5
:10409000FFF7CAFC00283FF435AF079B002B7FF4E5
:1040A00030AF3846FFF7BCFC4046FDF7BFFD01E0EE
:1040B0001B680FE70BB0BDE8F08F00BF5811010877
:1040C00000A493D6B41D002080EE3600F8B51E463D
:1040D0009F1C5B780446154613B96FF01500F8BDB8
:1040E00001F10800FFF75AFC0028F6D17CB394F9DF
:1040F0001030013304D1A3681C78022C04D001E0F5
:104100006468F3E7082C06D17378012B14D0022BD6
:10411000E3D1082411E0853D022D1BD884B97278C3
:1041200008236FF0010413FB024402FB036616F838
:10413000013D2BB9013CFAE70224853D022D09D847
:104140002246394606980AF099FD2046F8BD853D7D
:10415000022DE4D96FF08500F8BD70B51D465B787F
:104160000446164613B96FF0150070BD01F1080042
:10417000FFF714FC0028F6D1882E27D1A91CA4B182
:1041800094F91030013304D1A3681C78022C04D0B8
:1041900001E06468F3E7082C06D16B78012B0ED0A0
:1041A000022BE0D108240BE054B96C78E408023CFF
:1041B000E4B20B1913F8013C13B9013CF8E70224EF
:1041C000224604980AF05AFD204670BD70BDF8B52D
:1041D00017460D46FEF782FC7C78012C06460FD16F
:1041E000862D0FD100F5E07521462846FDF7EEFC3F
:1041F0007B681BBAA6F8C8312846FDF717FD01E019
:104200000020F8BD2046F8BD2DE9F0415378042B7D
:1042100086B00746154671D186294ED102F11008A5
:104220004046FFF7C7FB0646002846D13846FEF752
:1042300055FCB0F8C631DA0703D595F90330002BE9
:104240003BDB41463846FEF79FFC044618B1427CF2
:10425000AB789A422AD06B6843B31022002102A89F
:104260000AF0A6FDEB785B0616D4AA78414602A8B0
:1042700004F052FDEB78AA7803F0C00302A9384697
:10428000FEF74AFC0446002839D03846FEF726FCE3
:10429000012103F051FF09E00821009104AB002245
:1042A000384600F089F80028DFDA28E06B6833B977
:1042B0001CB121463846FEF757FC01261FE01BBA09
:1042C0006361AA68013312BAA2610CD00E4B69680F
:1042D0000E481B8809BA41431BB204F1300204F1B5
:1042E0001C0007F053FC237C23F07F03DBB2237414
:1042F000EA7822F03F0213432374DEE700263046BB
:1043000006B0BDE8F08100BFDC02002040420F0093
:104310002DE9F3410446884617461D4600F0F8FA99
:10432000064650B34146204600F0E0FA711E0446AE
:10433000284600F07DFD04B3237A53B1012B17D139
:10434000E068ADF8027000226946019508F03AFB7A
:1043500007E0B4F90C10ADF8027068460195FDF75E
:10436000CBFD002804DD204600F0E6FA0446E2E733
:104370000021284600F06EFDF5E7304602B0BDE8AA
:10438000F08107B540F20223019101466846ADF87D
:104390000230FDF7B1FD03B05DF804FB07B540F254
:1043A0000123019101466846ADF80230FDF7A4FDF6
:1043B00003B05DF804FB000000B589B006930A9BCA
:1043C000ADF81C304FF401738DF81410ADF81620C1
:1043D000ADF80630024605AB03A901A80293FDF72C
:1043E000AFFDBDF80E2040F205239A4203D00449E8
:1043F0000320FCF7F9FB049809B05DF804FB00BF4B
:104400005D0C010800B589B006930A9BADF81C301D
:1044100040F203238DF81410ADF81620ADF80630E5
:10442000024605AB03A901A80293FDF789FDBDF87B
:104430000E2040F205239A4203D004490320FCF7E2
:10444000D3FB049809B05DF804FB00BF5D0C0108C4
:104450002DE9F04384680746208F638D8FB000F00C
:10446000280EADF818304EF0010E0E4611B96FF05F
:1044700015005DE091F91030013354D18D682B792E
:104480002A7813F0C00F03BF02F108035B1995F8F7
:1044900001C0294B18BF4FF0020C12B105F1080101
:1044A00007E0420747BF04F12E01082204F12C0166
:1044B000022294F8360000F1010884F83680049056
:1044C0000DF12008BDF81800ADF80800ADF80400A3
:1044D000CDF80CE0CDF800C0404604F07BFA8146F0
:1044E0000028C4D0304607A900F048FA0646E8B1D3
:1044F000816881E800032B7913F0C00FBB6815BFFA
:104500001A69DA680132013214BF1A61DA6023686D
:10451000079A1B682046984700210446304600F061
:1045200099FC204604E06FF04C0001E06FF0680059
:104530000FB0BDE8F08300BF261101082DE9F0435C
:1045400087683B685C68002387B01A46194638467E
:10455000A047041E15DD002322461946184600F028
:1045600087FB054668B13B6881685E6822466B46FA
:104570003846B047B0F1000805DC0021284600F0BD
:1045800069FC002466E03E8F06F00206B6B2002EFB
:104590005BD1A86804F0B2FA044608B9014637E0D6
:1045A0000146C0EB08083246284600F07BFB8146F6
:1045B00008B90146E2E7866801AA04A9304604F07A
:1045C00013FB01AA044602A9304604F0BBFA002CF2
:1045D00001DA00241BE00028FBDBC1B2E3B204AA2D
:1045E00002A800F013F906460028F2D0022C0CD1E4
:1045F0009DF81030FF2B08D19DF81130FF2B01BF23
:104600008268137963F07F031371344626B9002161
:10461000284600F01FFC1DE0B3689DF801209A7148
:104620009DF800205A710D4A12885A8097F8283058
:104630002B744946284600F0CDF9002373602B46C1
:104640005A680AB11346FBE75E604146284600F00F
:1046500097FB2C46204607B0BDE8F083DC02002023
:10466000034B0360034B436081600020704700BF31
:10467000514400083D450008F0B5254E8468338854
:10468000838195B00821054604A8FDF7BBFC30885E
:10469000204B6360A56000B200F090F823682046CC
:1046A0009B68984740F2032741F234266846FDF79D
:1046B000A6FCBDF80230BB4213D0B3F5017F08D28F
:1046C00040F202229342F1D12B6801992846984783
:1046D000EAE70AD0B342E9D123682046DB6898476D
:1046E000E2E7236801995E6902E0236801991E6987
:1046F0000B894A6809782046B04740F205230390A9
:1047000002A96846ADF80A30FDF748FCCCE700BFC7
:10471000DC0200201947000813B50346806879B908
:1047200041F234230190B0F90C10ADF80230684624
:10473000FDF7C0FB002822DC12480AF0CBFC1EE08B
:10474000042919D0072913D0022918D143689847A2
:104750000446A0B103460C4990F9100040F2012232
:10476000FFF7D6FD014650B9204600F073FB06E086
:104770009A6901329A6102E05A6901325A6102B0C3
:1047800010BD00BFD81001080000FFFF30B585B094
:10479000089C6CB1A5685DB10293074B009301942E
:1047A0000823FCF7C1FA0028D8BF6FF0150001E01C
:1047B0006FF0120005B030BD79460008074B10B508
:1047C000B3F90040A04201D1002010BD14B16FF038
:1047D0000B0010BD1880FEF755F9F5E76C26002098
:1047E000044BB3F9003013B1038001207047184621
:1047F000704700BF6C260020034BB3F900301B1A32
:1048000058425841704700BF6C2600202DE9F04106
:10481000174603F108020A440E46002180461D4651
:1048200008464FF0FF3300F023FA00220446F8B1A7
:1048300083681E705D705A805A719A711A71B8F14E
:10484000000F08D03EB180680278B24203D14146E1
:1048500008300AF013FA5FB155B1A0684378AB4253
:1048600006D1037808332A46394618440AF006FA76
:104870002046BDE8F081000008B50B7A53B9B1F9C4
:104880000C200B4B53F822301B6A1BB9094903203B
:10489000FCF7AAF9C3B2042B9FBF074B53F82020A3
:1048A0000A6043F8201094BF00206FF0150008BD87
:1048B000280300205D0C010870260020C3B2042BE1
:1048C00011D8094A52F820308B4206D11B6842F8B1
:1048D00020307047914204D013461A68002AF9D15B
:1048E00001E00A681A60704770260020C3B2042BEA
:1048F00009D8064B53F8200020B143688B4203D0FF
:104900000068F9E770470020704700BF702600205C
:10491000C3B2042B0BD8074B53F8203000202BB127
:104920005A681B688A4208BF0130F8E770470020C8
:10493000704700BF7026002028B14368006810B19E
:1049400042689342FAD1704749B190F91030032B75
:1049500003D0042B06D103F0F3BF08F067BD6FF05E
:10496000150070476FF00100704728B190F91030C2
:104970008B4201D04068F8E77047000070B50446EC
:104980000E4619B912490320FCF72EF910B9002080
:10499000306070BD01460025496801350029FBD112
:1049A0006FF00103EA00204600F062F90028EED023
:1049B0008368002BE6D00833A26843F8082CE2682D
:1049C000646843F8042C0833002CF5D1356070BDC1
:1049D0005D0C010810B504468C42084601D164689C
:1049E00008E023465A682AB1904201D01346F9E7FD
:1049F00042685A600021416000F02CFA204610BD48
:104A000070B5556804460846EDB129464B680BB1B0
:104A10001946FBE71CB91A490320FCF7E5F8002802
:104A2000F9D0002AF7D043685360844206D0234669
:104A30005E6826B1B04219D03346F9E71446536890
:104A40004B60556015E0002CE5D00029E3D0002A2A
:104A5000E1D04B6853608C4206D02346596841B17F
:104A6000884205D00B46F9E7144602E05A60E6E7B3
:104A70005A600021416000F0EDF9204670BD00BF92
:104A80005D0C010870B503461A4A072B88BF033333
:104A900010688CBF23F003030823002140B344684F
:104AA000A34202D901460068F8E7E41A072C034440
:104AB000114E05D8046809B9146011E00C600FE0CC
:104AC000C6F108051D44B5F5C05F02D9002111608B
:104AD00003E009B9136000E00B60026883E814008A
:104AE000064A9B1B11889BB2994201D2138070BD6C
:104AF00070BD00BF882600208C2600208426002060
:104B000001210148FDF762B88C3E0020204A38B5EB
:104B1000831AB3F5C05F39D21E4D2C68002324B12F
:104B2000844202D223462468F9E707298ABF033169
:104B3000082121F003010460141AC1F5C052224477
:104B4000072A98BF891841600BB9286011E05A689C
:104B500018601A44821A072A0BD818B90E49032084
:104B6000FCF742F8026841681A60C21A0A445A60A7
:104B70001846036853B1426802449A1A072A05D8B6
:104B80001A6802601A1A5B681344436038BD00BF9C
:104B90008C260020882600205D0C01082DE9F843B2
:104BA000814614200F4616469846FFF76BFF0446D1
:104BB000D8B15EB13046FFF765FF054638B92046EB
:104BC0001421FFF7A3FF2846BDE8F88335460123EB
:104BD000C4F80490A560E66084F81080236027B1D3
:104BE0003246394628460AF049F82046BDE8F8839F
:104BF000F8B50F4D04460026CCB1631BB3F5C05F7A
:104C000003D30C490320FBF7EFFF94E88800012B46
:104C100009D1E168A0682660FFF778FF14212046DB
:104C2000FFF774FF01E0013B23603C46E4E7F8BD79
:104C30008C2600205D0C010808B5FFF761FF094ACA
:104C4000094B1360182100221A705A709A70DA709A
:104C50001A7159719A71DA710448BDE80840FCF77D
:104C6000E5BF00BF882600208C2600208C3E002057
:104C7000B2F5C05FF8B505460E4614461F460DD87E
:104C8000FFF73EFF22463B4631462846FFF786FFA8
:104C900004460348FCF7CAFF2046F8BD0020F8BDD3
:104CA0008C3E002007292DE9F84388BFCF1C0D4614
:104CB0008CBF27F00307082704469146FFF720FF23
:104CC0002DB124B1E3689D4201D8A3682BB92B48CC
:104CD000FCF7ACFF0020BDE8F8831420FFF7D2FEFC
:104CE00006460028F3D0E3689D422ED0AF4202D89A
:104CF0005A1B072A29D82846FFF7C4FE074610B9D1
:104D0000142130460BE0E068401BFFF7BBFE8046F5
:104D100040B914213046FFF7F9FE29463846FFF71F
:104D2000F5FED4E72A46A168384609F0A7FFE268F5
:104D3000A168521B2944404609F0A0FFE168A06821
:104D4000FFF7E4FEC4F8088005E0A7689D4214BFA1
:104D50007B190023A360E36808485B1BE36063687A
:104D600073600123B760F56086F810903360666069
:104D7000FCF75CFF3046BDE8F88300BF8C3E0020A6
:104D8000072970B588BFCE1C04468CBF26F00306E9
:104D900008260D46FFF7B4FE1CB922490320FBF795
:104DA00023FFE368A06813B90028F6D106E00028C5
:104DB000F3D01D4A821AB2F5C05FEED29D422CD0CC
:104DC0002DB930B11946FFF7A1FEA56024E09D4240
:104DD00002D8991B072917D82846FFF753FE064625
:104DE00020B91248FCF722FF0C2070BDA16829B140
:104DF000E268AA4228BF2A4609F040FFE168A0689D
:104E0000FFF784FEA66007E0033323F003039E420E
:104E100002D23044FFF77AFEE5600448FCF706FF53
:104E2000002070BD5D0C01088C2600208C3E002007
:104E300038B504460D46FFF763FE24B123682B44C2
:104E400023606468F9E70248BDE83840FCF7EEBE2D
:104E50008C3E002010B50446FFF752FE2046FFF7B7
:104E6000C7FE0248BDE81040FCF7E0BE8C3E0020C3
:104E700038B50446FFF744FE0CB1E26822B90E488B
:104E8000FCF7D4FE002038BD2368012B0FD994F91C
:104E90001030A1686068FFF781FE054610B12368F5
:104EA000013B23600448FCF7C1FE284638BD024898
:104EB000FCF7BCFE204638BD8C3E002007B501A89B
:104EC000FFF78EFCBDF9040000F020F903B05DF897
:104ED00004FB00002DE9F043082187B08248834C91
:104EE000834FFDF78FF840F20523ADF812302646C8
:104EF00002A8FDF784F8BDF80A30B3F5017F0AD89F
:104F000040F20322934280F0E68040F20122934275
:104F100000F08780ECE7B3F5106F04D040F6011283
:104F2000934273D0E4E7734D05F16C0815F8013C2A
:104F3000D3B1D5F81730022B0DD9042B05D8D5F8ED
:104F400013302946986900F0F9FAD5F81730023B7A
:104F5000C5F8173008E0D5F81390681F01F0ECF899
:104F60000021484601F076F924354545DED16378C5
:104F7000002B43D0238E013B9BB24FF6FD72934230
:104F80005D4B02D84FF4004201E04FF000429A61BD
:104F900096F98C30002B20DC96F83730022B18D88D
:104FA00094F8351051BB94F83430032B07D93C23C7
:104FB00084F8373084F8341084F835101EE001335B
:104FC00094F82920206A84F8343000F0C3FD0323CC
:104FD00000E0023B84F8373010E0E269002ADBD1C0
:104FE000218E4FF6FF729142D6D1023B5BB2002B6D
:104FF00084F88C30D0DC3D4801F0F9F8B7F9003086
:105000003E4A3F493F4806F0C1FD71E7039800283A
:105010003FF46EAF4369002B3FF46AAF06F01CFD0E
:1050200066E7DDF80C80B8F1000F03D136490320A4
:10503000FBF7DAFD02214046FFF797FC4FF0FF3106
:1050400005464046FFF791FC002DEFD018B183686C
:10505000B3F9021000E00146AA68D8F808506B784E
:10506000032B33D8DFE803F0020D1D2893885BBAC9
:105070009BB20093281D02F11803083200F0A0FA39
:1050800024E08368587928779B796B7793885BBA9B
:105090009BB20093281D02F11803083200F0ACFB0C
:1050A00014E093885BBA9BB20093281D02F11803A9
:1050B000083200F0B9FE09E093885BBA9BB2009316
:1050C000281D02F11803083200F008FF00214046B5
:1050D000FFF7C0FE0CE76FF0850304A902A8059353
:1050E000FCF75CFF04E700BF943E00207043002003
:1050F000903E0020E93E0020000C02403C020020CF
:1051000080841E00583F00205D0C01087FB51C4CB8
:10511000B4F90050064625BB1A4B1B481D701B4BAB
:1051200002931B4B00930195082305224FF48061E5
:10513000FBF7FAFD208000B316499B2288810320EB
:105140004A60FFF799FB00F011FF134A1349144816
:10515000B4F9003006F01AFD80222946114809F002
:1051600027FE0023802210493046FDF7D5FC0020A1
:105170000D4900F0E3F9B4F9000004B070BD00BFC0
:10518000903E0020503F00206C3F00200E1101088F
:10519000D54E0008D43E00203C02002080841E0032
:1051A000583F002000440020FE100108012380F831
:1051B0002F30002380F82C3080F82D3070473C23AE
:1051C00080F82F30002380F82C3080F82D30704785
:1051D00010B5012104460948FCF7F8FC084B187883
:1051E000421C1A7014B140F0800401E000F07F040A
:1051F0000248FCF71BFD204610BD00BF543F0020B5
:10520000503F002013B50C4612B11846FFF7E0FFDF
:105210002146022201F0EEF8044678B30022032171
:1052200080F8252080F82710012314220A2180F815
:10523000243080F8262080F8281084F82F3084F855
:1052400032304FF48073238694F83630052043F0D3
:10525000030384F8290084F836303C20094B60852C
:10526000F02084F82E00B3F9000001910092082389
:1052700040F6011204F1380106F014FC204602B099
:1052800010BD00BF903E00200021FFF7E3BD10F0ED
:10529000800F4BB202D0002B11DA01E0002B10DBA3
:1052A000884204D2C1F1800303440F2B09DD8842F8
:1052B00005D9401A0F28CCBF0020012070470020DC
:1052C0007047012070470000F8B5074615461E4696
:1052D0000C4639B920461949FDF77EFC044608B949
:1052E000384625E035B916492046FDF7AFFC05469E
:1052F0000028F5D0114A2946002E18BF32463846FC
:1053000008F00EF906460028EAD000231A4619468E
:105310001846FFF77BFA83680A495C8005464660B9
:10532000034640F202220220FEF7F2FF20B928468F
:10533000BDE8F840FFF7A8BFF8BD00BFFE100108A8
:10534000281101080000FFFF002370B510220C4651
:1053500019460646FFF78CFC054618B93046FFF79C
:1053600093FF24E0836804221A7000210E225A70F1
:105370009970A27FDA70E27F1A7194F820205A7136
:10538000A269B2F88A2052BADA80A269B2F88820FB
:1053900052BA1A81A269D2F884201288197352BABB
:1053A0005A8194F821205A73628C52BADA812846C5
:1053B00070BD002370B520220E4619460446FFF743
:1053C00057FC054618B92046FFF75EFF1EE08068CF
:1053D000082303701E2343704023C37033695A6946
:1053E00042609A6982605B7C8370002100F1100446
:1053F000017341738173C1731022204609F0D8FCF8
:10540000336931465A7C204603F086FC284670BD3D
:105410002DE9F3410F460446002800F0898090F8FA
:10542000363003F0020300F1080603F0FF0533B144
:1054300031460020FFF7BDFF0546002878D094F8DC
:105440003630DB070CD528463146FFF77DFF054691
:1054500000286DD094F8363023F0010384F83630FC
:1054600000231A2219462846FFF702FC804608B995
:10547000284637E0836822781A7094F82E205A70F4
:1054800094F83220022A04D14FF0FF329A70DA7079
:1054900002E0228E52BA5A8094F8802094F82F109D
:1054A000D20042EAC11294F825100A431A7194F806
:1054B00024205A7100229A71DA713546083304F1BA
:1054C000180E2A4603CA724518605960154603F142
:1054D0000803F6D1042301229B21404607F096FFE2
:1054E00028B9404602B0BDE8F041FFF7CDBE034603
:1054F0000022D9685B680A44002BFAD10E4B17B121
:105500003978FF290DD1996901319961D9690A4426
:10551000DA61B4F92C1000963B460022FFF7D4FE66
:1055200006E019690131196159690A445A61F0E7C5
:1055300002B0BDE8F08100BF00440020F0B51E4B72
:1055400085B000220546186803900F460A239B2168
:10555000104607F05BFF064658B3806800240471CC
:105560004471042203A9063009F088FB3246234621
:10557000D16852680B44002AFAD1104A17B1397821
:10558000FF290FD1916B01319163D16B0B44D36330
:1055900005B10835002200953B4611463046FFF71D
:1055A00093FE06E0116B01311163516B0B445363A1
:1055B000EEE705B0F0BD00BF121101080044002065
:1055C00030B41948BDF808505BB11978FF2908D0EC
:1055D000046A01340462446A2C444462052D07D8ED
:1055E00020E0846A01348462C46A2C44C462F5E712
:1055F0001B780E48FF2B09D143789BB190F83230CD
:10560000022B0FD0383030BC06F036BA43784BB19D
:1056100090F8363043F0010380F83630114630BC44
:10562000FFF7F6BE30BC70470044002070430020F6
:105630002DE9F04F8BB00026159F07933E600C4676
:10564000154600F054FF8246002800F0CF80B04697
:105650004FF47A7B079B434540F2C8802B78082B98
:1056600000F2BD80DFE803F0050FBBBB147698BBEA
:105670004C003B6808F1010843F001033B601FFA4E
:1056800088F80135E6E73B6843F002033B60A6E09B
:105690003B6843F010033B6094F8363043F001035D
:1056A00084F83630688940BA80B200F067FC10B1E7
:1056B000C4F8840003E000F061FCC4F88400E878DA
:1056C00084F8260095F804E084F827E0697984F8E6
:1056D0002810EB885BBAA4F88A302B895BBAA4F84F
:1056E00088306B7B84F82930EA8984F839000123FB
:1056F00052BA03FA0EF36285E36384F838106EE061
:105700003B68B4F92C0043F480733B6094F8363066
:10571000082143F0020384F83630009108AB0022E0
:10572000FEF74AFE002802DAEB785B0657D508221E
:1057300008A905F1100905F1180009F09FFA0023E6
:10574000AA78B4F92C004946FDF7E6F9002846D0BE
:10575000A06144E03B68B4F92C1043F020033B60A7
:1057600094F82900638DEA7843430BFB03F3002E82
:1057700008BF2E460493802A4FF0010394BF1206FF
:1057800000221498039310230190009202932A1D83
:10579000184807F0F5FA22E03B6843F040033B600D
:1057A0000EB900261BE04FF010096A79638DCDF821
:1057B000009053430BFB03F3029395F902300D481D
:1057C000DB43DB0F0193311D149B102207F060FBBC
:1057D000737802331E443378052BE6D0E1E76B780B
:1057E000023398441FFA88F81D4433E750460BB043
:1057F000BDE8F08F801D00202DE9F04786B01746E8
:105800000022039204460D46BDF83860AD4A5BB1F4
:105810001B78FF2B08D0136801331360536833449F
:1058200053601D2E07D849E1936801339360D36814
:105830003344D360F5E71E3E03A92078B6B200F0EA
:10584000B7FB002800F08F8063885BBA9BB24FF6ED
:10585000FF72934200F02F812379DDF80C80C3F3AF
:10586000C20388F88030002000F088FBC8F884006C
:105870004DB928469449FDF7AFF9054618B9934943
:105880000320FBF7B1F92A46002304F1080103982D
:1058900000F0BEFB039D06AA05F10808002342F8AC
:1058A000083D3946404600F0F3FB18B9049B002B35
:1058B00000F00181637885F82E3023790399DB09A4
:1058C00085F82F30237903F0070385F82530049BF2
:1058D000227E83F82020627E83F82120628852BADB
:1058E000DA8206AB002243F8042D012001930097D1
:1058F000334604F11A02FFF79BFE002800F0DB801C
:10590000059810F0100407D1039800F070FC394698
:105910002046FFF713FED1E0AB6943B94146B5F924
:105920002C00FDF793F9002800F0C580A8614046DF
:10593000FFF73CFC664A95F82730B2F9000095F86D
:105940002820019295F826200092012202FA03F302
:1059500005F1380140F6011206F0A4F8049940461A
:1059600000F078FCAAE0039D002D00F0A78005F16F
:105970000808102204F10801404609F04DF981465B
:10598000002840F09B80039A237992F88020C3F38B
:10599000C2039A4240F09280627895F82EA0104699
:1059A0005146FFF774FCC8B195F83230012B0FD186
:1059B000130601D5FF2A00E07F2A1ABF0132D2B2B6
:1059C0004A4685F82E2005F1380006F055F80BE020
:1059D00085F82E20404600F01BFC05E0114650469D
:1059E000FFF755FC00283DD195F83230012B0BD143
:1059F00063885BBA9BB24FF6FF72934205F13800A1
:105A000032D006F082F859E006AA002342F8083D99
:105A10003946404600F03CFB049B08B9002B4DD0B2
:105A20001BB105F1380006F070F8049900293FF425
:105A300026AF237E81F82030637E81F82130638891
:105A40005BBACB82404600F005FC049B1A7972B920
:105A500063885BBA9BB24FF6FF7293422ED12A8EB7
:105A60009A422BD005F1380006F006F826E0EA69E4
:105A7000934223D15A7D63799A4202D04046FFF780
:105A800095FB049B62795A7523790399DB0985F8A4
:105A90002F30237903F0070385F8253006AB002269
:105AA00043F8042D012001930097334604F11A02B4
:105AB000FFF7BEFD10B9039800F099FB06B0BDE8F2
:105AC000F08700BF00440020FE1001085D0C0108B3
:105AD000903E0020F8B500230C46164619461422C5
:105AE0000746FFF7C5F8054618B93846FFF7CCFB5F
:105AF00011E0836805221A7012225A7000229A70EF
:105B0000DE702146043304F1100251F8040B43F80F
:105B1000040B9142F9D12846F8BDF8B500230E4692
:105B20001546194606220746FFF7A2F8044618B99B
:105B30003846FFF7A9FB0AE0836806221A700422A0
:105B40005A70ED0100229D70DA701A715E71204664
:105B5000F8BD00002DE9F04F8DB00E4606920546C7
:105B6000002800F0FD8090F83230012B00F0F88022
:105B700021B9C669002E00F0F38005360CA805F1A6
:105B800008030024194640F8044D059309940A942B
:105B9000FDF736F80B9B002B00F0E28001217248E4
:105BA000DFF8D8B1FCF712F8A04604940394DBF8B0
:105BB00008309C4268D2DBF8007007EB4417D7E945
:105BC000022313435ED0BB69DA070CD4039BD3B91D
:105BD000012206991846FFF7A0FF0A9088B962488B
:105BE000FCF724F8BCE0049B83B91A4606991846D2
:105BF000FFF793FF804609900028F0D0012304931B
:105C000004E0012303930DF1280901E00DF12409BB
:105C10007B699A78FF2A03F1020A07D1D87800F04D
:105C20000F00A0F10E035842584120E008224F49CE
:105C30000793504608F0F0FF079B08B9002016E0D4
:105C40009A78FF2A04D1DB7803F00F03022BF5D0FA
:105C500010224749504608F0DFFF0028EED01022FE
:105C60004449504608F0D8FF003018BF012048B121
:105C7000FA7CD9F800005146FFF72CFFC9F8000064
:105C80000028ACD0013492E73748FBF7CFFF0A9BDE
:105C9000B8F1000F02D0C8F8043000E00993802268
:105CA0000B990998FFF716FF04460990002857D072
:105CB00095F90070002F07DA002310220599FEF7EE
:105CC000D7FF0A9030B30990DDF824800023042226
:105CD00019464046FEF7CCFF04460A9008B94046F4
:105CE00019E083682A781A70002FB4BF402200227E
:105CF0005A705A78099062F07F025A7095F83320F2
:105D0000DA7000279F70022204239B2107F07EFB9C
:105D10000A9018B92046FFF7B7FA21E00990024629
:105D20003B46D16852680B44002AFAD13278FF2AE8
:105D3000114A0ED0116D01311165516D0B4453653F
:105D4000059BB5F92C10009300223346FFF7BCFAEF
:105D500006E0916D01319165D16D0B44D365EFE79C
:105D60000DB0BDE8F08F00BF8C1D00202811010888
:105D7000381101088811010800440020801D00200E
:105D80002DE9F7430E4691460446002846D090F987
:105D90000080B8F1000FACBF0823182303229B2119
:105DA000002007F033FB0546002837D087682378AA
:105DB0003B71B8F1000F09DA80237B71102204F1E6
:105DC000080107F1080008F059FF01E000237B718A
:105DD000002387F80690FB712A46D16852680B446D
:105DE000002AFAD10F4A16B13178FF290FD1916FED
:105DF00001319167D16F0B44D367B4F92C1008348B
:105E00000094334600222846FFF75EFA06E0116F41
:105E100001311167516F0B445367EEE703B0BDE8E2
:105E2000F08300BF004400202DE9FF4117460546DE
:105E3000BDF82840284A8BB11B78FF2B0ED0136C7D
:105E400001331364536C234453646B7813F0400F95
:105E50000CBF082318239C423AD306E0936C01330D
:105E60009364D36C2344D364EFE7287800F0C2F83E
:105E7000064668B36B785B0605F1040106F1080875
:105E800001D4083C07E01022404608F0C5FEF8B9EE
:105E900005F11401183C96F83220022AA3B217D05B
:105EA00004AA002042F8040D0097019202200A463D
:105EB0003146FFF7BDFB58B195F90130002B04DAEC
:105EC000EA7839463046FFF75BFF4046FFF76EF948
:105ED00004B0BDE8F08100BF0044002070B5224A44
:105EE0000446BDF81000A3B11978FF2911D0116E36
:105EF00001311166516E014451661B78FF2B32D07F
:105F000094F90130002BACBF0823182398422AD102
:105F100006E0916E01319166D16E0144D166ECE7E5
:105F2000207800F067F80546E8B194F90130002BBD
:105F300005F1080602DBE37843B90CE01022211DCD
:105F4000304608F069FE0028F5D070BDA27895F8BB
:105F500033309A4207D1012385F835303046BDE809
:105F60007040FFF72CB970BD0044002008B500F068
:105F70002DFB014B186008BD80440020054B1B68B9
:105F80000BB900F023BB1A8882420CBF18460020D0
:105F9000704700BF8044002090F83220022A02D1CE
:105FA000383005F0AFBD0149FFF732BAFE100108E5
:105FB00010B500230E4A0B6054780CB90A6004E057
:105FC0001478844201D10A600FE00B686BB118703D
:105FD0000B68012058700B6800224FF48071A3F801
:105FE0008A20A3F88810DA6110BD184610BD00BFE2
:105FF00070430020054A53782BB1137883420CBFBD
:106000001046002070471846704700BF70430020BC
:10601000F8B5044608B1407818B91B490320FAF7CF
:10602000E3FD0D4604F1080701F1100E28686968C8
:106030003E4603C6083575453746F7D14FF6FF7122
:1060400021861249E164142184F82610032184F882
:1060500027100A2184F82810052184F829103C21F2
:106060006185F020002184F8330084F8321084F830
:10607000241084F83410246584F835102462A28535
:10608000A3610120F8BD00BF5D0C0108995F000805
:106090002DE9F8430026264F166080460D4614462B
:1060A0004FF0010917F8013C33B9B9F1000F14D0D2
:1060B0007A1F2260994610E0D7F8133043450CD17F
:1060C0002946384602F0EDFD38B11A4A242303FB75
:1060D000062626600020BDE8F8830136032E07F16E
:1060E0002407DFD1206800B3C0F81880236800229D
:1060F0001A60D8F8143033B11A680AB11346FBE7B6
:1061000022681A6002E02368C8F81430236801226C
:106110001A7123682946053305F1100251F8040B62
:1061200043F8040B9142F9D10120BDE8F88300BF88
:10613000E93E0020E43E002030B5044687B018B99F
:1061400020490320FAF750FD85696B6998422AD1EE
:1061500010221D491D4806F0E4FE2368D3B100203B
:10616000FBF710FB22681A4BB0FBF3F0D369B5F9CB
:106170002410181A4FF47A735843053201230393FD
:106180000192102300220490009202930E4A0F48BD
:1061900006F0F6FD6B699C4205D123686B6108E04F
:1061A000944204D013461A68002AF9D101E022680B
:1061B0001A6024220021204608F0FAFD012007B0D1
:1061C00030BD00BF5D0C010838110108801D0020A2
:1061D00040420F0038B50446406920B10568FFF71A
:1061E000ABFF2846F9E74FF6FF73238538BD10B59E
:1061F00004460830FFF7EEFF04F1380005F082FC9A
:1062000090220021204608F0D3FD012010BD00009F
:1062100010B5037F013303774369044633B1FFF7B9
:10622000D9FF102209490A4806F07BFE228D4FF65D
:10623000FF739A4208D0238504F1300005F01CFC5E
:10624000A369052283F88C2010BD00BF3811010816
:10625000801D00202DE9F04F0A4689B00446E1B1C7
:10626000438C90F821105943D16141698A4214D17D
:10627000B0F9241090F8210043434FF47A7043435F
:10628000053204930123039301921023002200920C
:106290000293564A564806F073FD6369228D0692B2
:1062A000002B00F099804FF0010B002266696261BB
:1062B00092469146002E36D00AF1010A3546002753
:1062C0002D6801370DB9D84610E05F45F8D1FAE7DF
:1062D000B8F1000F0DD12A4635463668013FB9F1B5
:1062E000000F1CD0C9F80050A9461546002FEFDC5E
:1062F00001E02DB9EFE7B8F1000F12DD8DB157B114
:10630000A2690793D2F884202946D2683046904784
:106310000028079BDFDD2A6808F1FF38DFE76561A9
:10632000E2E72E46C6E7B9F1000F01D0C9F80060D8
:10633000BAF1010F4FEA4B0BB7DC6269D08A4FF616
:10634000FF71884248D0934223D0A06990F8802002
:10635000023A012A06D80022591DFFF7FBFB20460E
:10636000FEF724FF638C94F82120B4F92410204810
:106370005A434FF47A7353436269049305320123FD
:10638000039301921023002200920293174A06F011
:10639000F7FCA3696069D3F8843000215B689847F3
:1063A000069B2085834203D004F1300005F064FB96
:1063B000606978B1A369228DB3F88810C38AB2FBF3
:1063C000F1F2B3FBF1F39A42056801D8FFF7B4FE8E
:1063D0002846EEE763692BB9204609B0BDE8F04FC7
:1063E000FFF716BF09B0BDE8F08F00BF38110108F4
:1063F000801D0020334BB3F900302DE9F3410646F0
:106400000C4615460BB9002058E0002301930B7889
:10641000FF2B0BD14B7803F00F030E2BF3D121464A
:106420006846FCF7D9FB074608BBECE7082226497B
:10643000204608F0F1FBA0B12378FF2B04D163784C
:1064400003F00F03022B0CD010222049204608F045
:10645000E3FB30B110221E49204608F0DDFB002886
:10646000DDD123780433DBB2012BD8D9CBE7DDF8BB
:106470000080B8F1000FC6D001A93046FFF798FDA3
:106480000028C0D00020019EFFF778FDC6F88400E8
:1064900001984FF48073A0F888300023A0F88A3068
:1064A000214680F8805043463A46FFF7B1FD044646
:1064B000019814B9FFF79BFEA5E7006202B0BDE8A2
:1064C000F08100BF903E002028110108381101081A
:1064D00088110108022380F82A3000218069FEF724
:1064E00097BF002380F82A30303005F0C5BA70B568
:1064F00000249C422ED21578082D25D8DFE805F01F
:1065000005242424091319240E000134A4B20132F5
:10651000EFE7012822D155780E2D14E001281DD176
:1065200055781E2D0FE0022818D15578122D0BD961
:1065300014E0022812D191F880505678012D14BF32
:1065400004251425AE4209D1557802352C44A4B255
:106550002A44CEE70CBF0120002070BD002070BD92
:10656000704721B910B94FF6FF707047C18A90F893
:10657000202090F8213013446FF0090293FBF2F3CE
:10658000826903F5807392699BB20028A2F8883073
:1065900008BF4FF4807358188142E4DC80B2704722
:1065A000C28ACB8A9A4203D38CBF01200020704755
:1065B0004FF0FF30704738B50446FFF7F1FF002871
:1065C000CCBF0846204638BD7047000000487047E1
:1065D000440200200021FEF73DBC00002DE9F041FF
:1065E0009EB0102200210AA808F0E2FB804B0B931A
:1065F000804B08211B88ADF834300EA8FBF702FD54
:106600000AA90120FEF738F940F20523ADF81A3047
:1066100040F2032440F2012504A8FBF7F0FCBDF88A
:106620001230B3F5017F09D8A34280F0D880AB4285
:106630000CD040F2022293426ED0EDE740F22522C8
:106640009342E9D1059800F0EDF9E1E7059D284670
:10665000FEF70EFC044600287ED00121FEF785F9E6
:10666000054608B1C3681BB92046FFF7B3FFCFE763
:1066700083681B78412B11D1FEF7FAFB05460028F1
:10668000F2D001221146FEF70DFB01460028EBD0A7
:106690002046FEF79FF90223044631E003F0D802BA
:1066A000C02A03D1204600F0B1FAB1E703F0E003BD
:1066B000602BD9D10021022328220846FEF7D8FA00
:1066C000089010B9089890B9CEE703AB0093002367
:1066D00021461A4608A800F0DFFC01460028F1D048
:1066E00001222046FEF7DEFA014618B90898FFF7A6
:1066F00071FFB9E72046089AFEF782F900230446A5
:106700002B7440F20122234639490220FDF700FE96
:1067100000287FF47DAFA7E7059DEDB1EB68072B5F
:106720001AD96B68C3B193F91030022B14D12846E3
:10673000FEF79EFB044678B18768B7F9020001F0C6
:1067400095FE61688046002619B1CB6849681E44F1
:10675000FAE7B8F1000F01D1284686E798F804302F
:1067600023B1204600F086FF70B97DE701231A4669
:106770000846FEF77DFA00283FF476AF6368436071
:106780006060836841221A70626800231AB1D16880
:1067900052680B44FAE7B8F80210994208D3214630
:1067A000B7F90200FDF7EDFD00283FF731AF5BE7D9
:1067B000114B596800297FF457AFB6F5006FBFF44D
:1067C00053AF79889A8108A840F2252219805C602D
:1067D0009E60ADF822200993FBF730FB18E76FF0BD
:1067E000850306A904A80793FBF7D8FB10E700BFB1
:1067F0000000FFFFDC020020844400201FB50A4C8B
:10680000B4F9000000280DDC084B0293002301932B
:10681000074B0093032208234FF480610548FAF7E1
:1068200083FA208004B010BD94480020161101089E
:10683000DD6500089444002038B50E4B142404FB99
:1068400000340546638A63B10020FAF79BFF0A4BC8
:10685000B0FBF3F0094B53F82530834206D80023F0
:106860006382637C23F01003637438BD1B1A638258
:1068700038BD00BF9648002000879303D849002008
:106880002DE9F041012180461048114DFBF79EF99A
:10689000002426462746E0B2FFF7CEFF2B7C53B1FB
:1068A0004146284602F012FA2B7C834203D8B842B4
:1068B00084BF2E4607460134102C05F11405EAD199
:1068C0000248FBF7B3F93046BDE8F081184A0020D2
:1068D000964800200F2838B5044615D801210B48EA
:1068E000FBF774F92046FFF7A7FF094B142000FBC4
:1068F000043506482C7C1CB1FBF798F9284638BDB6
:10690000FBF794F9204638BD002038BD184A002016
:10691000964800202DE9F8430F280646884615467C
:106920001F469DF820903FD8002A40D001212148E1
:10693000214CFBF74BF9002F4FF0140303FB0643E8
:1069400008BF4FF00009802D88BF80225F828CBF76
:106950001A741D74B9F1000F02D046F0100300E064
:106960003346142000FB064441466374204602F07F
:1069700098F9014640B91022204608F019FA227C05
:106980004146204602F0C8F90020FAF7FBFE0B4B07
:10699000B0FBF3F00A4B0744064843F82670FBF7B8
:1069A00045F92046BDE8F8830020BDE8F88310468D
:1069B000BDE8F883184A002096480020008793031A
:1069C000D84900200021FEF745BAF8B50E460178F7
:1069D0004378174601F10802024405460830FDF7E6
:1069E00015FF0446E0B18368B5F902205A802A7980
:1069F0001A716A795A71AA799A71B7424FF00001F7
:106A00003A464FF0010328BF32460846FEF730F9F8
:106A1000054620B92046FFF7D5FF2846F8BD60603F
:106A20002046F8BD2DE9F04F054685B0B0F90000CD
:106A300001F01CFDD5F80480D8F8044083464FF0DF
:106A4000000A1CB1E36864689A44FAE7BBF1000FDE
:106A500005D14046FFF7B6FFC5F804B0D0E0B5F861
:106A60000C90B9F1000F42D1674FAE683B88D8F85F
:106A7000080001333B80CAEB06039AB2BBF8023030
:106A8000043B134403F0F8039B1A1FFA83F909F13E
:106A900004025146FFF799FF034600283AD04268A6
:106AA000D2F808A076BAAAF800609AF8002062F03E
:106AB0003F028AF800203A8852BAAAF80220D8F891
:106AC0000470002F7CD0FA68B9680093C4EB090603
:106AD000964228BF1646201D344432465044A4B284
:106AE00008F0CCF8A145009B6AD97F68E9E7D14559
:106AF00080F08280BBF80260D8F80800AF68053EDD
:106B000006F0F806C9F10501721D5144FFF75DFF5B
:106B1000034628B96868FFF755FF00236B606FE0F4
:106B200042689268511D009179BA1180117861F024
:106B30001F01117034494F440988CAEB070A49BA4A
:106B40004FEADA0A518082F804A0D8F80470FFB145
:106B5000A1451BD0FA68A11889B2894513D2C4EBAC
:106B600009041FFA84F9C9EB0204B442B968009819
:106B7000019328BF34462246494408F07FF8A4B266
:106B80007F68019B05E07F680C46E0E7002400E099
:106B90003C46A64214D99FB1FA680193C4EB06089B
:106BA0009045009BB96828BF904618194444424656
:106BB000A4B208F063F8A642019B01D07F68EAE71F
:106BC0001946BBF900000093FDF7DBFB0028009B92
:106BD00002DC1846FFF7F6FE002C9BD0AB8903952C
:106BE0001C44AC8140F2252302A8ADF80A30FBF723
:106BF00025F9FAF75FF803E04046FFF7E3FE6C6023
:106C000005B0BDE8F08F00BF1C4A002010B58268B7
:106C1000137803F0F803C02B044606D0E02B0DD107
:106C20001379C268DB00053A02E0C2680023043A27
:106C300060682146806800F013F82046BDE81040E7
:106C4000FFF7C0BE002203682BB119689A80DA8072
:106C50001A600160F7E7436070470021FEF7FAB859
:106C60002DE9F04F8FB081460020924604911F46D7
:106C70008E68AA4DFAF786FDA94A834605F1900869
:106C80002C46606858B1A368C3EB0B03934206D946
:106C90000292FFF7E2FF2046FFF7D4FF029A243466
:106CA0004445EED199F800B009F1080307930BF1C0
:106CB00008034B44069399F80130029333885BBA7A
:106CC000C3F30A03059373885BBAADF8263000203E
:106CD0009BB20A93FAF756FD002308901C460393D3
:106CE0006A68A846002A00F02581D2680599914279
:106CF00023D1EA8B0A998A421FD12A7F93451CD15E
:106D00006A7F0299914218D15A4607990B9305F16F
:106D10000C0007F081FF0B9B78B9029A069905F1E8
:106D2000140007F079FF0B9B38B97C4C039A24239D
:106D300003FB0244089BA3604EE014B96A6802B9E1
:106D40002C463BB1A9689A68521A76498A4294BF88
:106D5000A8469846039B0133042B039305F12405B1
:106D600001D04346BCE784B9B8F1000F03D16E49A6
:106D70000320F9F739FFD8F804000028F7D0FFF70F
:106D80006CFF4046FFF75EFF444600210223059A50
:106D90000846FDF76DFF6060002800F0DD80836825
:106DA00000210020C3E90001089BA3605A4607990F
:106DB00004F10C0007F062FF029A069904F1140036
:106DC00007F05CFF9DF808306377BDF82630E38359
:106DD000002384F81CB0238425680FBB3379412B32
:106DE00003D105360AF1FF331FE003F0E003602B07
:106DF00006F1040618D10EAB204643F8047D50F886
:106E0000042F0093D2680499042300F045F9002868
:106E10007CD00D9A28320AEB020306441B1A05E0C7
:106E200005365346002201E053463A466068C16881
:106E300003EB070E8E456AD81FFA87FE0EF1FF316D
:106E4000194489B26DB1B5F804804145C0F0828023
:106E5000B5F806C0E6457DD8C6456FD161456DD110
:106E600078E01FFA83F80EF1FF314144DFF8C0A04B
:106E700089B2AC460AEBCC05B5F806B0BBF1000F01
:106E800011D1ADB1E98021682960A5F804E0218C19
:106E9000256080684144174421849A1A3146384459
:106EA00007F0ECFE04E00CF1010CBCF1340FE1D171
:106EB0006368228CDB689A424ED1637F217F04F1A4
:106EC000140204F10C00FDF7A1FCF8B18368B9F9D4
:106ED00002205A8099F804201A7199F806209A71B4
:106EE00099F805205A710023436063682BB15A68F2
:106EF0000AB11346FBE7586000E0606063680B4925
:106F000040F201220220FDF703FA10B96068FFF792
:106F1000A4FE2046FFF796FE1EE000BF204A002098
:106F2000C0C62D00FEFFFF7F5D0C01080000FFFFC3
:106F3000B04A0020002C7FF404AF01E7FFF78DFE7C
:106F40002046FFF77FFE3B46524604994846FFF72E
:106F500087FE01E02D6875E70FB0BDE8F08F00BF38
:106F6000037823F00F0343EA11130370437803F00F
:106F70000F0343EA011141707047000008220149E4
:106F800007F07CBE281101081022002107F010BF75
:106F900010B508220949044607F03EFE48B123789F
:106FA000FF2B08D1607800F00F00831E5842584133
:106FB00010BD012010BD002010BD00BF2811010828
:106FC00073B51546194A04460E46106851686B465B
:106FD00003C32CB3637CDB0624D4227C802A1DD01F
:106FE000402A1FD9D208D11F501C2944C2F10F02D8
:106FF000304407F011FEA8B9237CD9080D44725C17
:1070000015F8080C03F0070302A90B44424013F8DB
:10701000083C1A420CBF0120002004E0012002E0DD
:10702000204600E0002002B070BD00BF1A11010828
:107030000023042A10B54370037016D0082A02D02A
:10704000022A26D118E00B7883F0020303704B78F4
:1070500043708B788370CB78C3700B7903714B7955
:1070600043718B798371CB7911E00B7883F0020344
:1070700003704B7843700223FF240022C470FE2467
:10708000827004714271CA5C82710B445B78C37177
:1070900010BD184610BD00002DE9F74F1E464B6885
:1070A00000920F46D3F808A0D1F808B0019018B9A3
:1070B000C0490320F9F798FD019B1B68002BF7D00E
:1070C000DA68272AF4D90BEB06089D6898F9013095
:1070D000002B2B7803F00F0343F060032B701BF899
:1070E000063003F01803ACBF02240324082B27D07A
:1070F00017D8002B52D118F804102846FFF730FF9C
:1071000008EB04014B7803F00F026B7813436B70AC
:107110008978AA78E31C0A43AA7018F8032004347B
:1071200029E0102B2AD0182B38D100212846FFF750
:1071300017FF6B7823F00F036B700023AB702CE00C
:1071400018F804309B099B0043F060032B706B78A8
:1071500003F00F01697018F8043003F00F0308EB17
:1071600004020B436B705178AA78A31C0A43AA70DF
:1071700018F803200334EB7813430EE018F80410DA
:107180002846621CFFF7ECFE6B7823F00F036B7050
:107190000023AB70EB70144600E0EB701BF8063078
:1071A0005B075CBF18F80430AB711BF8063003F0C6
:1071B000030358BF0134022B08D0032B08D0012B46
:1071C00007D018F80430EB71013403E0402300E0ED
:1071D000FF23EB7198F8013003F0400202F0FF0941
:1071E00072B118064ABF98F802000020000913F097
:1071F000300905D0FFF76EFB8146002800F0318290
:1072000098F8013003F07003302B42D00FD8102BC8
:107210001CD0202B26D0002B40F08C8008EB0401E2
:10722000102205F1080007F029FD103482E0502BF0
:107230003BD006D8402B7DD105F10800FFF7A4FE16
:1072400078E0602B45D0702B62D073E005F1080028
:10725000FFF794FE082208EB040105F1100007F087
:107260000DFD34E005F10800FFF788FE4FF0FF3216
:107270000023EA746FF001022A752B746B74AB74EF
:107280006B75022208EB040105F1160007F0F6FC0D
:107290003CE0514605F1100011F8082BFFF7C8FE3D
:1072A00005F10800FFF76AFE44E0B9F1000F3FF472
:1072B000FFAE082208EB040105F1100007F0DEFC28
:1072C00099F81020494605F1080001F025FD083421
:1072D00030E0B9F1000F3FF4EBAE4FF0FF32002386
:1072E000EA746FF001022A7508EB040102222B7484
:1072F0006B74AB746B7505F1160007F0BFFC99F861
:107300001020494605F1080001F006FD023411E0A5
:10731000B9F1000F3FF4CCAE514605F1100011F861
:10732000082BFFF785FE99F81020494605F1080063
:1073300001F0F2FC98F8013059070FD51A064ABF40
:1073400098F80200002000F00F0013F00B0F05D09A
:10735000FFF7C0FA8146002800F0838198F80130D9
:1073600003F00F030C2B00F27C81DFE813F00D001B
:107370001600250042007A015100610082000D00D4
:107380009400A600B800C60008EB0401102205F125
:10739000180007F073FC1034D9E005F11800FFF76E
:1073A000EDFD082208EB040105F1200007F066FC62
:1073B0003CE000BF5D0C010805F11800FFF7DEFDA1
:1073C0004FF0FF32002385F823206FF0010285F88B
:1073D000242085F8203085F8213085F8223085F882
:1073E0002530022208EB040105F1260007F046FCD7
:1073F0003DE09AF800109AF801200831514405F157
:107400002000FFF715FE05F11800FFF7B7FD9EE01D
:10741000082208EB040105F1200007F02FFC99F881
:107420001020494605F1180001F076FC08348EE082
:107430004FF0FF32002385F823206FF0010285F81A
:10744000242008EB0401022285F8203085F8213041
:1074500085F8223085F8253005F1260007F00EFC6E
:1074600099F81020494605F1180001F055FC023446
:107470006DE09AF800109AF801200831514405F1A6
:107480002000FFF7D5FD99F81020494605F11800B6
:1074900001F042FC5BE005F11800FFF775FDFF23EA
:1074A0002B7618F804306B76611C0522414405F1F7
:1074B000230007F0E3FB063449E005F11800FFF76D
:1074C00063FDFF232B7618F804306B76611C0322D2
:1074D000414405F1250007F0D1FB043437E005F104
:1074E0001800FFF751FDFF232B7602236B7618F867
:1074F000043085F82730013429E005F1180099F8A7
:1075000010A0FFF741FD99F81030402B84BF4023B5
:1075100089F81030FF232B7618F804306B7608EBCF
:10752000040349465B78AB7699F81030EB7699F80E
:10753000102005F1580001F0EFFB211D0422414409
:1075400005F1240007F09AFB063489F810A0009B8F
:1075500013B9FB681B1B01E0009B283B5BBAAB80A7
:107560001BF806305B077ED518F8043003F0F803EB
:10757000F02B78D1019BBD68D3F800A0009BDAF80E
:107580000890344404F1010815F804B04BB900998F
:10759000042308220846FDF76BFB002865D08268AB
:1075A00002E009F1280200200BF00303022B14D0A3
:1075B000032B1FD015F808101170012B05EB0403E5
:1075C0009978517004D0D978917005341B790FE007
:1075D000DB780434A3F5805318E015F80830A3F5E0
:1075E00080535BBA13802B19043499789170DB783F
:1075F000D3700DE015F808301909A1F5756149BA85
:1076000003F00F0302341180A3F575635BBA538056
:107610001BF0040F03D00021FDF71CFC25E02B5DBF
:107620009371A31C2C446178D17118B1F9680831A9
:10763000C91A01E00099283949BA9180112189F8C5
:1076400006109288A9F8042018B1019AC0F804A085
:10765000106053B19C1B0C9B0C9A1B680833136081
:1076600001E0002003E0204601E00024F3E703B03E
:10767000BDE8F08F2DE9F04F4268D0F80890966889
:10768000D268002189B0824601230846FDF7F0FA4E
:10769000029038B38568AB4960232B7006F1080B64
:1076A00000236B701022584607F0B6FA38B15846DE
:1076B000FFF7E6F8804610B1437CD90601D44FF0BD
:1076C0000008337EFF2B00F0628206F11800FFF7FE
:1076D000D7F80746002800F05A82437CDA0640F1CA
:1076E000568201E0029858E2B8F1000F04D098F8F1
:1076F00011301B0703D15FB17B7C1C0708D06B786E
:1077000063F07F036B700023AB70032401E04746F6
:10771000022431683378727821F4704121F0FF013E
:107720001B01A9B943EA121313F0FF0F2B7803D101
:1077300043F018032B7036E043F010032B7073787E
:1077400031781B09621C43EA01132B5594B22AE0DD
:107750005BB203F030011209114304F101010ED1B3
:107760002B7843F008032B7032688BB2317812BA51
:107770008910C2F3034242EA81122A5509E01343F9
:107780002B55326889B212BAC2F30342A31C6A5461
:107790009BB2326812BA120AEA549C1C01339BB2A3
:1077A0000022EA54A4B2B379112B6DD1DAF8043077
:1077B000586883681A88B3F802E052BA92B222F08D
:1077C0000F0C1FFA8CFC4FF2B0018C451AD19EFAB7
:1077D0009EF121F00F010904090C614512D1032229
:1077E000B271598849BA1FFA81FE198849BA89B21B
:1077F0000EEB011101F5AA61197099795970D979C7
:10780000997026E09EFA9EFE0EF47F4EBEF5704FF4
:1078100004D10122B2715A8852BA0CE002F47F42BC
:10782000B2F5704F0ED10222B2711A8852BA1A7094
:107830009A785A70DA789A709A79DA70DA791A71D5
:10784000052206E00022B2719A791A71DA795A712A
:107850000622B17961F00F01C2F1080EB1711A442C
:10786000C168C3EB020CCEEB01018C4504D212F8C7
:107870000E1002F8011BF3E7FDF782FA2B7843F0B4
:1078800004032B70012303E0621C2B5594B20023E8
:107890000393F379402B07D0FF2B0AD0012B0CD197
:1078A0002B7843F0010302E02B7843F002032B70A6
:1078B00006E02B7843F00303F9E7621C2B5594B2E2
:1078C00010222049584607F0A7F918B96B7843F001
:1078D000400335E0B8F1000F0CD06B7843F0400363
:1078E0006B7098F8112010070AD0AB7843EA0213A6
:1078F000AB7005E05846FFF74BFB002800F04081D5
:1079000008AB0020002163E9040199F80020082A4F
:1079100000F224814FF48A71D140C90740F11E81E1
:1079200009F108011846FFF783FBDDE904237169BB
:107930003069994208BF904206D16B7843F030031A
:107940006B7021E03811010804AA59464046FFF740
:1079500037FB0028F1D13369B3F17F4F05EB040009
:107960006B7840F00381B28A52BA92B2B2F57E4F80
:1079700040F0FC8043F020036B70022206F11601F8
:1079800007F07CF90234A4B2337EFF2B72D16B78FE
:1079900043F008026A70728BCABBF269BABB328CC0
:1079A000AABB727E022A0FD1326A6AB9B28C5AB966
:1079B00096F8262042B943F00B036B7096F8272007
:1079C0002A55631C9CB2B4E0728C8AB996F82420C4
:1079D00072B943F00A036B70737E2B55601C03224F
:1079E00006F1250115FA80F007F048F904349FE00C
:1079F00096F82220002A40F0948043F009036B702F
:107A0000737E2B55601C052206F123012CE0B38BFD
:107A1000ADF81030F38BADF81230338CADF8143074
:107A2000738CADF8163004A8FEF72AFF002878D032
:107A3000437CDB0675D5027CF37E9A4271D16B786C
:107A400043F004036B70437C13F00F031EBFAA784E
:107A50001343AB70737E2B55631C9BB2B27EEA540A
:107A6000A01C042206F1240115FA80F007F006F9A3
:107A700006345DE01FB199F801303BB951E006F1E1
:107A80001800FFF785FA0028F5D14AE057B16B7866
:107A900043F004036B707B7C13F00F031EBFAA78C6
:107AA0001343AB7099F8001099F80120083149444C
:107AB00004A8FFF7BDFADDE90423716A306A994230
:107AC00008BF904204D16B7843F003036B7030E041
:107AD00004AA06F118013846FFF772FA0028F2D11D
:107AE000336AB3F17F4F05EB04006B780FD1B28C92
:107AF00052BA92B2B2F57E4F09D143F002036B70D5
:107B0000022206F1260107F0B9F8023410E043F032
:107B100001036B70082206F1200107F0AFF808346A
:107B200006E02819102206F1180107F0A7F8103412
:107B3000A4B2039B1BB1631CB2792A559CB22146A7
:107B40000298FDF71DF9DAF804105046FCF742FFE1
:107B5000029A43685360426001201EE00821B9F98F
:107B6000020000910022FCF727FCDEE643F0100340
:107B70006B70082206F1100107F080F8083402E764
:107B800028191022594607F079F81034FBE6B8F1AD
:107B9000000F3FF4BCAD0027A9E509B0BDE8F08FA8
:107BA00010B508220949044607F036F848B1237891
:107BB000FF2B08D1607800F00F00831E5842584117
:107BC00010BD012010BD002010BD00BF281101080C
:107BD000F8B5B0F8C631DB07044603D415490320D5
:107BE000F9F702F800F5E0760121002504F5EE77BB
:107BF0003046F9F7EBFF384684F8CB51F8F770FFC1
:107C00004FF40873A4F8F2310B4B0C49B3F9003070
:107C1000C4F8F44104F5F872384603F0B7FF304673
:107C2000FAF704F82946B4F9C401BDE8F840FCF7B6
:107C3000CFB800BF5D0C0108B41D002080969800ED
:107C4000F8B5B0F8C631DB07044603D42449032055
:107C5000F8F7CAFF00F5E07601213046F9F7B6FFE4
:107C600094F8CB31022B03D8013384F8CB3116E0E2
:107C7000DD1E01F039F90123AB403B2BB0FBF3F5DE
:107C800005FB13009EBF94F8CB31013384F8CB3150
:107C9000092804D93C2828BF3C20054600E00A25D5
:107CA00004F5EE773846F8F71BFF4FF40873A4F895
:107CB000F2310C490C4BC4F8F4416943B3F900307C
:107CC00004F5F872384603F061FF3046F9F7AEFF6D
:107CD000B4F9C4010021BDE8F840FCF779B800BF51
:107CE0005D0C010840420F00B41D002010B5044691
:107CF000B0F91A00FAF7F2FEB0F8C631DA0703D489
:107D000010490320F8F770FF637E1B070BD4002097
:107D100005F020FDA8B9B4F91A00FAF7DFFEBDE8B6
:107D20001040FFF755BF10220749204606F074FFA8
:107D30000028ECD02146B4F91A00BDE81040FCF749
:107D400047B810BD5D0C0108381101082DE9F0435A
:107D500080468DB01846894614461F46FFF720FF1F
:107D60000546B8B910230693029308AE07AB0790F7
:107D700003900093019706AB32460DF11601474878
:107D800005F009F9002806DB069B102B0CBF3546D1
:107D9000002500E000253946204605F091FC064606
:107DA000002D74D030B93946BDF9160005F088FCB5
:107DB0000646E0B1B6F91A00FAF790FE18B1B0F82D
:107DC000C631DA0706D5737E03F03003302B08BFC7
:107DD0003D4600E03D4645B93846FFF7E1FE002844
:107DE00051D03D46002D3CD00EB1AF4204D02946C3
:107DF000204605F065FC06462846FFF7D1FE58B33D
:107E000026B1737E03F03003202B25D107AE304618
:107E1000FCF7E6FC0822074689F80020A91840462E
:107E200006F02CFF98F8003083F0020388F8003049
:107E3000CCB9BC4215D036F91400FAF74FFE48B160
:107E4000B0F8C631DB0705D50CAB03EB440434F9BD
:107E5000140C1FE00134ECE7737E03F03002202A9B
:107E600003D1002016E0204614E003F00703032BA3
:107E700003D104213046FBF74BFF324649464046CA
:107E800005F09EFC06E0FBF72FFE0546AAE700285A
:107E9000A2D08FE70DB0BDE8F08300BF801D0020A9
:107EA00070B50E4618B911490320F8F79DFE002958
:107EB000F9D0B0F91A00FAF711FE00F5EE75044694
:107EC0002846F8F70DFE4FF40873A4F8F23108497C
:107ED000084BC4F8F44104F5F87271432846B3F92D
:107EE0000030BDE8704003F051BE00BF5D0C0108DA
:107EF00040420F00B41D0020F8B507460D46164657
:107F000010211A462120FBF7BEFC044660B18068B0
:107F100000236DBA0822877043710371C370C58056
:107F20003146104406F0AAFE2046F8BD2DE9F04F78
:107F300085B080460E9E7578022D0F4692461C46EF
:107F400040F0B8800823009300226B440321FCF723
:107F500033FA0028C0F2AE804046FAF7BFFD214652
:107F60008146404605F0ACFBBAF1870F04464ED07F
:107F7000BAF1880F40F09E80B9F8C631D90740F1B8
:107F80009980DDE90223D6F80CB0D6F808A05B454D
:107F900008BF524540F08E80002800F08B80B578F5
:107FA000012D2ED00BD3022D40F08480404607F1E6
:107FB000080105F0ADFB4846FFF70AFE7AE009F537
:107FC000E07901214846F9F701FEF6883D4B04F1BE
:107FD0003807384676BAB3F90080B6B2F8F780FDB4
:107FE000394940F21223013EA4F84E303846434648
:107FF00004F14C02714303F0C9FD4846F9F716FE3F
:108000005BE007F118014046FAF7AEFD52E0B9F81F
:10801000C6319A074ED0B378002B4BD108371022C7
:108020002A49384606F0F8FD002843D0D4B1637ED3
:108030009B060CD5D4F88C20D4F8903052EA03017A
:1080400005D0F168B0688B4208BF824234D1B6F8DF
:108050000690B9F1000F05D13946404605F058FBAE
:108060004D462AE0F3882BB384B9032300930F9A7B
:10807000109B3946404605F0B5FA0446E8B1324651
:1080800000F18C0352F8080F516803C3637E0E4859
:1080900023F0300343F030036376F188094B49BA8B
:1080A00089B24143B3F9003004F1840204F1700055
:1080B00003F06CFD002500E00125284605B0BDE871
:1080C000F08F00BFB41D0020008793033811010812
:1080D00013B58A784B78402A01D8022B00E0032B95
:1080E0000ED186280ED1C878CB88C0F300145BBAB5
:1080F00000949BB2083100F00F00FEF70BFC01E08A
:10810000002000E0012002B010BD000008B50146CB
:10811000074800F0C6FD48B910220649044806F099
:108120007BFD0028024818BF002008BD004808BD9C
:10813000504C00203811010838B50446E1B1012344
:1081400080221449B0F9C401FAF7E6FCA0B104F5A5
:10815000E07528460121F9F739FDB4F8C63143F03E
:108160000403A4F8C6314FF4E163A4F8CC312846E7
:10817000BDE83840F9F75ABDB4F8C631B4F9C401C6
:10818000044923F00403A4F8C631BDE83840FAF7E7
:10819000EBBC00BF7811010808B51022044905485E
:1081A00006F03AFD0028034808BF002008BD00BFC4
:1081B00038110108504C00202DE9F04700240546F5
:1081C00000F116074FF00109A2464FEAD40804F067
:1081D000070617F8083009FA06F633420AD0E0B26B
:1081E000FEF778FB80F810A017F8083023EA06069F
:1081F00007F808600134102CE7D10026AC695CB1A7
:108200002368AB616368A168B3F9C401FAF7ACFCF9
:1082100026606660A660F1E710222146284606F037
:10822000C7FD2C61BDE8F0872DE9F04F87B003F161
:10823000080A02905046039117461E46FFF766FF54
:108240000446002800F0B480F3885BBA9AB21AB9E9
:1082500042F210738382ABE0DFF860918382103FBB
:108260004FF00008002F70DD08F11003039AD518B5
:10827000D35C032B02D0222B4AD05EE00298FAF79F
:108280002DFC6B780190042B42D105F1100B0822D4
:108290004949584606F0C0FC002839D02A7CFF2AFC
:1082A00004D16A7C02F00F02022A31D0EA7851062A
:1082B0002ED413062CD46A6852B359460298FAF7A2
:1082C000C5FCAA7804905946D9F80800059200F038
:1082D000FDFC059A824209D8D9F808305B7C9A42A5
:1082E00004D1D9F80430019A9A4207D0334B9868E8
:1082F00020B11022324906F08FFC48B92F4B5A6842
:1083000032B9019A5A60049A9A60A2691A60A3610C
:10831000AB783F2B6B7801D8022B00E0032B0CD1FC
:10832000EA7804F11603C2F3C001012002F007024B
:1083300000FA02F2585C02435A546B7808EBC30807
:108340001FFA88F8A7EBC3078CE773885BBA9BB268
:108350002361B28852BA43EA02432361DAF800008B
:10836000DAF80410234603C356F8100F716802228E
:1083700003C3002104F1160006F01AFD0023A361D7
:10838000A58A104B04F11C0630465D43F8F7A8FBA4
:1083900040F2232363860C4B6463B3F9003004F18D
:1083A00030022946304607B0BDE8F04F03F0EEBB7F
:1083B00007B0BDE8F08F00BF28110108884C0020ED
:1083C0003811010800879303B41D00202DE9F04106
:1083D0008846C108064614460831069A22201F46E0
:1083E000FBF751FA0546A0B18068002164BA01711B
:1083F0004171C480867080F80380EA6800F1080447
:10840000083A204606F0D4FC32463946204600F0B1
:1084100083FC2846BDE8F08170B505460E4614463B
:1084200018211A462320FBF72EFA80B183686ABA16
:108430002D0C6DBA76BA5A809D80DE8022689A60D3
:108440006268DA6054F8082F1A6162685A6170BD78
:10845000054BB3F90020904204D01AB901221880CC
:1084600059801A71704700BF944C0020034BB3F938
:10847000002082420CBF184600207047944C002018
:1084800008B518B907490320F8F7AEFBC31C133031
:1084900013F8012F1AB98342FAD1012008BD002038
:1084A00008BD00BF5D0C01082DE9F0410C461546E2
:1084B0009846064618B926490320F8F795FB11B1EE
:1084C000CB8A002BF7D02DB1EB8A002BF3D00CB167
:1084D000A28AB2BB06F1680718220021384606F0CE
:1084E00067FC5CB12368042B03D06FF06900BDE822
:1084F000F08118222146384606F0C0FB06F18007BD
:1085000018220021384606F053FC7DB12B68042B5D
:10851000EBD12846FFF7B4FF18B16FF01500BDE8A6
:10852000F08118222946384606F0A8FB24B1E28AD9
:108530000421304605F008FAA6F898800020BDE82E
:10854000F081AB8A002BC5D09A42C3D0E5E700BFCB
:108550005D0C010808B5014618B904490320F8F775
:1085600043FB0420BDE80840FCF7A8B95D0C0108F6
:108570002DE9F04188B090460E461A460E9F0446FB
:1085800018B111B1B8F1000F03D12E490320F8F74B
:108590002BFB836E002B50D008AD01A945F8183D88
:1085A0002B4605F0E9F9002849DB0198C368984596
:1085B00005D20021FCF74EFC6FF068003FE004217B
:1085C000FCF7D3F90028E0D0D0F8088047B1182292
:1085D0002946384606F052FBB8F800305BBAFB82F9
:1085E000D4F88030E3B1B8F80030B4F896205BBA24
:1085F0009BB29A4206D001980021FCF72BFC6FF049
:1086000046001CE0843410220F49204606F004FB8B
:1086100030B1102203A9204606F0FEFA0028EAD164
:10862000019B30469968DA6806F028FB0198002122
:10863000FCF710FC019BD86801E06FF07C0008B0EB
:10864000BDE8F0815D0C0108381101082DE9F04109
:108650000F4686B090461D46044628B9002B7CD1B3
:1086600042490320F8F7C0FA0AB10029F8D0ADB1A9
:10867000EB8A13B96FF0150074E02846FFF700FF8E
:108680000028F7D12B68042B5ED16CB1B4F87C20A4
:1086900042B1AB8A33B19A4204D0EBE7D4F88030D0
:1086A000002B54D0A36EF3B918220021684606F0BF
:1086B0007FFB2F4A138803EB03166FEA86466FEAA7
:1086C00096460133B6B21380ACB1A4F87E6015B9FA
:1086D000D4F8803000E02B68A3663246042120469F
:1086E00005F032F907E0182204F168016846B4F891
:1086F0007E6006F0C3FA25B904F18005B4F896400F
:1087000000E0EC8A009A2B680AB9009301E09A42D3
:10871000B0D10023394642461846FCF7A9FA07466D
:10872000C0B13146224600F025F9014618B9384655
:10873000FCF790FB0EE011232A46694605F080F90C
:1087400000280FDD08380DE06FF069000AE06FF0D7
:108750007F0007E06FF00B0004E0002A88D00029BA
:1087600086D17DE706B0BDE8F08100BF5D0C010851
:108770009A4C00200021FCF76DBBF8B507468489B0
:108780000E46154600204DB900230822B96800F0B6
:1087900061FA96F91030022B25D10DE0BD42F3D0DD
:1087A000B542F1D02346AA89A96800F053FAEB68D4
:1087B0006D681C44A4B2E6E702194FF6EE739A42C4
:1087C000C4BF013080B2B16811342044002320229C
:1087D000083180B200F03EFA4FF6FF73984203D0A2
:1087E000C04380B2F8BD0020F8BD000070B5102273
:1087F00098B000210DEB020006F0DAFA4D4B05931C
:108800004D4B1B88ADF81C3040F20523ADF80A3003
:1088100008216FF0850308A80393F9F7F3FB04A977
:108820000420FCF729F86846F9F7E9FBBDF80230A7
:108830006FF400721344032BF5D8DFE803F0023B1A
:108840007575019D2846FCF713FB044608B92846B8
:1088500067E00221FCF789F8064618B9374903207A
:10886000F8F7C2F9606830B190F91030042B02D1EA
:10887000C368082B06D0042208212046FCF712FA10
:1088800000284DD0002385682374EB885BBA9BB227
:10889000002B45D022463146FFF76FFF4FF6FF739E
:1088A00098423DD1698849BA234640F2012289B2F3
:1088B000042031E0019E304696F91050FCF7D8FABA
:1088C000044608B930462CE0406826460028C5D04A
:1088D00090F91030042B07D0FCF7CAFA0346F8B120
:1088E000706040681E46F1E7FCF7C2FAC0B18268CA
:1088F00070600023C16840680B440028FAD15BBA5D
:1089000093806B1C08BF63680A4908BF93F9105035
:1089100040F2022223462846FBF7FAFC002882D1C7
:108920002046FFF727FF7EE702A96846F9F736FBE6
:1089300079E700BF0000FFFFDC0200205D0C0108AA
:1089400010B5044668B161B190F91030042B0BD119
:108950004268FFF712FF50B1A36840BAD8800020E8
:1089600010BD6FF00D0010BD6FF04C0010BD6FF02A
:10897000010010BD38B50D4614460423082200211D
:10898000FCF776F938B1836800226DBA64BA1D80AD
:108990005C809A71DA7138BD1FB50A4CB4F90030A9
:1089A00063B9094A0193094B0292009305220823F7
:1089B0004FF480610648F8F7B7F92080B4F9000059
:1089C00004B010BD9C50002022110108ED87000862
:1089D0009C4C0020F8B504469DF8245025701E4696
:1089E00005F0070310250F46657006989DF82810BE
:1089F00015460AB1002F68D018B1002E69D1304653
:108A0000F8BD23B1022B02D00DB9002873D0A1709C
:108A100080B39DF82030E37002289DF82130237147
:108A200004D0082816D0002851D120E0024632494F
:108A3000304606F0F1F818B9237823F020032370AC
:108A4000637843F008036370737863713378A371BC
:108A5000072040E01C236370221D06F1080313F871
:108A6000011D02F8011F9E42F9D10D2033E00520BF
:108A70001DB9F8BD0320002D3DD0431C9DF81C20DE
:108A800022549DF81D20E2540230022D03D0082DFF
:108A90000CD0E5B9F8BD637863F07F0363707A7832
:108AA0002254431C3A78E2540230F8BD637863F0F4
:108AB0003F03637007F10803044413F8012D04F821
:108AC000012BBB42F9D10830F8BD3846F8BD002073
:108AD000F8BD63B90DE075B1BDF81C20BDF82030BC
:108AE0009A42CAD1237843F040032370CDE7022B8A
:108AF0008AD1A1708DE7F8BD26110108427802F0F5
:108B00000C03082B07D00C2B07D0CBB901784906F2
:108B100014D4032302E0072300E00D2312F0C00267
:108B20000CD00178490658BF0233802A01D1981C25
:108B30007047C02A04D103F10800704718467047F7
:108B40000020704770B501B11AB926490320F8F723
:108B50004BF8437803F00C03082B07D103785C062D
:108B600017D5C37813700379537012E00C2B07D11B
:108B700003785B060FD5C3781370037953700AE04E
:108B800013B16FF0150070BD03785E06F9D40323AE
:108B900002E0072300E00D23447814F0C00411D054
:108BA00005786D0605D4C65C16705D1C0233455D04
:108BB0005570802C08D1C25C4A70034402205B7857
:108BC0000B7070BD204670BDC02CDAD1034401F19A
:108BD000080213F8010B02F8010D8A42F9D10820AE
:108BE00070BD00BF5D0C010808B501B11AB9184984
:108BF0000320F7F7F9FF437803F00C03082B09D1A2
:108C0000C37813700379537043794B7083790B7079
:108C1000022008BD0C2B0ED1C378137010F8043F4E
:108C2000537001F1080310F8012F03F8012D8B4256
:108C3000F9D1082008BD3BB9037813F0400F14BFE9
:108C40006FF01500002008BD6FF0150008BD00BFD3
:108C50005D0C0108F0B51AB3DC0705D511F8014B1E
:108C6000013A204492B20133570801EB47054C1CEE
:108C700003350234AC4207D014F803EC14F8026C4C
:108C800006EB0E263044F4E71A44D30703D511F857
:108C9000173000EB0320030C80B201D01844FAE730
:108CA000F0BD30B54B68456804680A689D4208BF4E
:108CB000944209D1C568CB6884688A689D4206BF22
:108CC00094420120002030BD002030BD30B510B3EB
:108CD000E1B188421CD001380139002210F8015F4F
:108CE00011F8014FA54202F1080303D1DAB2802A3C
:108CF000F4D10FE085EA0401D8B20B060AD40132A0
:108D0000D2B249008242C9B2F7D130BD084630BD67
:108D1000802030BD104630BD802A28BF8022F8B5A3
:108D2000D50814462A4606460F4605F0A7FF6307F6
:108D30000ED0A4EBC504725DFF23C4F1080403FA4E
:108D400004F422EA040272557B5D1C4014437455FE
:108D5000F8BD10F8013F43B18B42FAD100230370F4
:108D6000437813B1013005F0D1BB104670470000C5
:108D70002DE9F04707468AB008B90020A8E000298D
:108D8000FBD000204FF0FF3406462346054631F85D
:108D900010E0BEF1000F07D1B3F1FF3F13BF013563
:108DA00003B201252DB20BE0B3F1FF3F08D0B4F1BF
:108DB000FF3F01D0B54201DD2E461C464FF0FF3388
:108DC00001300828E3D1581C04D0601C7DD0B54286
:108DD00002DD7AE0601C03D0012ED8BF4FF0FF34D3
:108DE0003D4800256B46E8464FF03A09AC4203D1B6
:108DF00083F80090A5194EE015B183F80090013377
:108E000011F815E01EF0F00F4FEA450C17D04FEAAD
:108E10001E1A0EF00F0E10F80AA010F80EE083F8DC
:108E200001E001EB0C0E83F800A09EF801E04FEA90
:108E30001E1E033310F80EE003F801EC21E0BEF132
:108E4000000F10D010F80EA09E460EF802AB01EBFA
:108E50000C0A9AF801A04FEA1A1A10F80AA083F82F
:108E600001A073460DE001EB0C0E9EF801E01EF030
:108E7000F00F1FBF4FEA1E1E10F80EE083F800E04F
:108E800001338C4401359CF801E00EF00F0E10F810
:108E90000EE083F800E0072D03F10103A6DD611C5D
:108EA00005D03444082C02BF3A2119700133002147
:108EB00003F8011BC8EB030393423FF65EAF414644
:108EC000384606F06BFB384602E02E461C4683E728
:108ED0000AB0BDE8F08700BF9811010801460148BB
:108EE00002F056BDA0500020124BF0B593E83400BC
:108EF000D8681E691C6084EA050122F000424A40DD
:108F000082EA420280EA500050405969D86040F33A
:108F1000000782EA802239404A4004EB12249A601A
:108F20009A693E40604044F30004754014405D601F
:108F30006040F0BDA05000200C4B014618688268CC
:108F40009368013B002B10B4936005DA9469A34247
:108F500008DBCBB20A2B05D01368581C10601970BF
:108F600010BC704710BC06F08FBD00BF6C02002023
:108F700008B53E20FFF7E0FF2020FFF7DDFF034BA1
:108F80001B689868BDE8084005F098BB6C0200209B
:108F90002DE9804885B0814600AF0E469246FFF726
:108FA000E7FFB0460AF1FF340025C6EB0803A342F1
:108FB000F5DA844B186841684B68013B002B4B6025
:108FC00004DA06F08FF8002804DAE8E70B685A1C88
:108FD0000A6018780D2801D00A280FD100240D202E
:108FE00088F80040FFF7A8FF0A20FFF7A5FF4645D5
:108FF000D5D033462246254620462BE0082801D00E
:109000007F280DD14645D0D0082008F8015CFFF735
:1090100093FF2020FFF790FF08F1FF3B082003E0BB
:1090200008F1010B88F80000FFF786FFD846BCE77F
:10903000222913D15C781CB35C2C25D001331C7819
:109040008C42F7D1597820291AD80135197811B3F3
:1090500003F8010B19782029F8D9E9E7272906D167
:10906000E8E74B1C497822290AD02029EDD91C7841
:109070005C2C1946F5D1591C5B780132002BF0D1DC
:10908000514806F027F88AE79C1C9B780132002B98
:10909000F6D02346D3E7002D81D0AB000E3323F06A
:1090A0000703EB46ADEB030D6C464DF8251030463B
:1090B00090F800E003460130BEF1000FF8D0BEF199
:1090C000220F02D0BEF1270F00D1013344F8213026
:1090D0001846013390F800E0BEF1000FF8D10131DD
:1090E0008D42E5D1201FBAB150F8043FA3B1194613
:1090F00013F801EBBEF1000FF5D0BEF15C0FF6D115
:1091000091F800E0BEF1000F04D091F801E001F801
:1091100001EBF5E7013AEAD12C4B2268FB60C7F876
:109120000890002307F1080151F82380B8F1000FDF
:109130000DD10133022B16D0F4E711463B607A6063
:1091400006F0C2F87A683B6830B108F10C08D8F82C
:1091500000000028F1D1ECE7D8F808301BB1214617
:10916000284698472CE02168194806F0ADF80546D6
:1091700010BB184A1849194805F022FF184805F095
:10918000A9FF124BC7F80890FB602C4607F10803B3
:1091900053F824500DB10C3503E00134022CF5D105
:1091A0000EE00C3555F8181C0029F6D055F8142C93
:1091B0000A4805F005FFF4E721680A4805F000FFBA
:1091C000DD46ECE66C020020A9110108C01301087D
:1091D000C2110108C7110108D3110108DB110108F0
:1091E0008A2B0108E511010808B503F071FC002085
:1091F00008BD08B5F7F75AFE002008BD012810B5D4
:1092000006D10020F8F7BEFA04460146074805E0FB
:10921000486805F07BF904460146054805F0D0FE94
:109220002046FFF75BFE002010BD00BF5014010870
:109230007614010808B5FFF757FE0146024805F00D
:10924000BFFE002008BD00BF8B3A0108014606287A
:1092500014D8DFE800F004060B0D0F1109000948CF
:1092600000E0094805F0ACBE0848FBE70848F9E70C
:109270000848F7E70848F5E70848F3E7084805F025
:109280009FBE00BF981401089C140108A214010895
:10929000AA140108AF140108B2140108B51401089A
:1092A000BB140108102828D00BD803281BD003D8E2
:1092B000E8B1022815D07047052816D006281AD024
:1092C0007047262815D004D8162818D0202818D082
:1092D00070472A2817D02B2817D0272818D10D48D7
:1092E00014E00D4812E00D4810E00D480EE00D4866
:1092F0000CE00D480AE00D4808E00D4806E00D4876
:1093000004E00D4802E00D4800E00D4805F058BEAD
:10931000704700BF47150108C0140108D0140108A8
:10932000DD140108F3140108FB14010800150108FD
:1093300013150108251501083A1501085E150108E5
:109340006915010808B50146034805F039FE0348D0
:10935000BDE8084005F0BEBE781501089D1501085E
:1093600013B5044601A8FBF73BFA20B1BDF9040090
:10937000031B5842584102B010BD00001FB504AB9A
:10938000012403F8012D00940022FBF73BF800288C
:1093900004DA094805F09EFE20460BE09DF80F1008
:1093A000064B074A0748002914BF1146194605F025
:1093B00007FE002004B010BD2B1901082819010870
:1093C0003835010847190108A0F13003DAB2092A3B
:1093D00004D9A0F16103DAB2052A01D81846704712
:1093E0004138C3B2052B88BF4FF0FF3070470000F3
:1093F0007FB50C46082105460DEB0100164604F02A
:1094000029FA08B911480FE0009002AB002221466A
:109410002846FAF7F7FF00280ADA0D4805F0D0FDD4
:109420002046FFF73FFF0B4805F054FE01200BE0FC
:10943000094805F0C5FD2046FFF734FF32462946AE
:10944000064805F0BDFD002004B070BD5E1901089E
:10945000D119010838350108E7190108F519010883
:109460007FB5064610460D4605F050F804AB0124C2
:1094700003F8010D0022009429463046FAF7C2FF96
:1094800000280ADA0C4805F09BFD2846FFF70AFF82
:109490000A4805F01FFE20460CE0094805F090FD43
:1094A0002846FFF7FFFE9DF80F200648314605F0DD
:1094B00087FD002004B070BDD119010838350108BE
:1094C000E71901080E1A01087FB506460D46104639
:1094D000531E13F8014F1CB1303C092CF9D908E098
:1094E0000A22214606F0C4FA0390013009D11C4833
:1094F0001CE01022002106F0BBFA03900130F6D0E8
:109500000124039BB3F5803FF1D202230093002294
:1095100003AB29463046FAF775FF00280ADA1148EE
:1095200005F04EFD2846FFF7BDFE0F4805F0D2FDC1
:10953000012012E00D4805F043FD2846FFF7B2FE7A
:1095400031460B4805F03CFD039924B1094805F06C
:1095500037FD002001E00848F9E704B070BD00BF06
:10956000271A0108D119010838350108E71901083F
:10957000751A01088B1A01089F1B0108022808D0E0
:10958000FF2808D0054A064B01280CBF1846104694
:109590007047044870470448704700BFA41A010888
:1095A000931A01089B1A0108A01A010870B5012935
:1095B00088B00C46164609D104230093002207AB5D
:1095C0002921FAF7F9FE051E0EDA09E0022905D174
:1095D000F9F7DCFC079008B1012505E06FF085057F
:1095E000154805F077FD24E0E4B266B11C220021A5
:1095F000079805F0DDFB2046FFF7C0FF01460F4846
:1096000005F0DEFC15E02046FFF7B8FF079AD368A7
:10961000516804939368039313690293019113684B
:109620000B440093936952690146054805F0C8FC54
:109630003546284608B070BDAC1A0108E61A010884
:10964000071B01082DE9F04790B002AF0026044641
:10965000FE70F9F743FA21460546CB4805F0B0FC09
:10966000082300933246FB1802212046FAF7A4FE95
:10967000061E1CDB06EB460808F1070323F0070370
:10968000E946ADEB030D0DF1080AC04805F098FC62
:10969000334607F108024146504604F0AFF8014650
:1096A000BB4805F08DFCBB4805F08AFCCD46022383
:1096B0000022009311463B1D2046FAF77DFE00284C
:1096C00003DBB988B44805F07BFC02230093002239
:1096D0003B1D26212046FAF76FFE002803DBB988E0
:1096E000AE4805F06DFC0223009300223B1D0621CD
:1096F0002046FAF761FE002803DBB988A84805F088
:109700005FFCA84805F05CFC082300930022FB18CE
:1097100003212046FAF750FE061E1EDB06EB460824
:1097200008F1070323F00703E946ADEB030D0DF144
:10973000080A9D4805F044FC334607F108024146FB
:10974000504604F05BF80146984805F039FC98480B
:10975000CD4605F035FC012600E0002602230093EB
:109760000022BB1D10212046FAF726FE002804DB4C
:10977000B7F906108F4805F023FC0123009300225F
:10978000BB1C18212046FAF717FE002808DB8A4880
:1097900005F016FCB878FFF759FD7E4805F010FC7F
:1097A000012300930022FB1816212046FAF704FE3D
:1097B000002803DB7978814805F002FC4FF00108AE
:1097C000CDF8008007EB0803002220212046FAF79D
:1097D000F3FD002810DBCDF80080FB1C00221F21C8
:1097E0002046FAF7E9FD002806DBFB78434503D164
:1097F0007978734805F0E4FB6A4805F0E1FB012342
:1098000000930022FB1C13212046FAF7D5FD002807
:1098100008DB97F80380B8F1010F03D1694805F020
:10982000CFFB4646012300930022FB1C1421204657
:10983000FAF7C2FD002808DB97F80380B8F1010FA2
:1098400003D1614805F0BCFB46460123009300228A
:10985000FB1C15212046FAF7AFFD002808DB97F81E
:109860000380B8F1010F03D1584805F0A9FB464623
:10987000012300930022FB1C12212046FAF79CFDD5
:10988000002808DB97F80380B8F1010F03D1504896
:1098900005F096FB4646012300930022FB1C19218C
:1098A0002046FAF789FD002808DB97F80380B8F115
:1098B000010F03D1474805F083FB4646012300937F
:1098C0000022FB1C1F212046FAF776FD002808DB4A
:1098D00097F80380B8F1010F03D13F4805F070FB02
:1098E0004646012300930022FB1C1E212046FAF766
:1098F00063FD002808DB97F80380B8F1010F03D15E
:10990000364805F05DFB4646012300930022FB1C10
:1099100023212046FAF750FD002808DB97F8038042
:10992000B8F1010F03D12E4805F04AFB4646FDB1C0
:10993000B5F8C8112B4805F043FB95F8CA112A4821
:1099400005F03EFBB5F8C631D80702D5274805F02B
:1099500037FBB5F8C631990702D5254805F030FB2D
:10996000B5F8C6315A0702D5224805F029FB012671
:109970002046FEF77BFD002840D00379002B3DD028
:109980001D4805F01DFB3AE0B21B0108E91B010868
:10999000F91C0108011C0108BE1B0108CD1B0108B0
:1099A000D91B0108E11C0108E51B0108F31B010894
:1099B000F71B0108031C0108161C01081F1C0108E5
:1099C000331C0108461C0108501C01085A1C0108E0
:1099D000641C01086E1C0108781C01087F1C01082A
:1099E000891C0108981C0108A21C0108AA1C010876
:1099F000B01C0108B61C0108C01C010816B139488A
:109A000005F0DEFA0223009300223B1D05212046CB
:109A1000FAF7D2FC002803DBB988334805F0D0FA06
:109A2000002D58D0B5F8C6313049314813F0800FB9
:109A3000304B08BF194605F0C3FA2A4805F0C0FAB2
:109A400005F5E07610222C49284605F0E5F80028B7
:109A500031D02A4805F0B4FA2822294607F110002F
:109A6000FFF786F908B36A7C254807F1100105F075
:109A7000A7FA08222349284605F0CEF838B12B78FA
:109A8000FF2B06D16B7803F00F03022B01D11E4888
:109A900000E01E4805F094FA2B7CDB0708D52B78F4
:109AA000FF2B0CBF1A481B4800E01B4805F088FA42
:109AB0000C4805F085FA3835B542C3D1174805F092
:109AC00009FB002201212046FFF770FD0022022140
:109AD0002046FFF76BFD114805F0FCFA3837BD460C
:109AE000BDE8F087E11C0108C71C0108A31B0108A1
:109AF000EE1C0108A91B010838110108FC1C010813
:109B0000091D010828110108181D01081E1D010862
:109B1000251D0108321D01083D1D010838350108C9
:109B20002DE9F04F012889B0804602AF0E460BDCCC
:109B300007F10800FAF754FE18B1B7F90800FFF76B
:109B400081FD002400F06EBC4868431E13F8014FED
:109B50003CB3303C092CF9D93168A94805F030FAFA
:109B60003068FFF7EFFB3168A64805F029FA316845
:109B7000A54805F025FA3168A44805F021FA3168B6
:109B8000A34805F01DFA3168A24805F019FA3168BA
:109B9000A14805F015FAA14805F09CFA012400F04F
:109BA00041BC04F0B3FC05B22846FFF7D9FB0028FE
:109BB00000F01984B8F1020F04D12846FFF742FDE6
:109BC00000F030BC9649B06805F07EFB002840F0FC
:109BD0002482B8F1040F01DC30681BE2D6F80C8057
:109BE0009048D6F800903669414605F06DFB10B9F3
:109BF000324602210CE041468B4805F065FB002807
:109C0000F6D04146894805F05FFB28B9324603216A
:109C10002846FFF7EDFBACE34146854805F054FBD1
:109C200010B93246002151E04146824805F04CFB14
:109C30000028F6D04146804805F046FB10B9324670
:109C4000262143E041467D4805F03EFB10B93246EF
:109C500006213BE041467A4805F036FB0028F6D065
:109C60004146784805F030FB0028F0D04146764860
:109C700005F02AFB044610BB304604F047FC07F110
:109C80001803022223F8100D1021009228462246C4
:109C9000FAF7B8FB002807DA6C4805F091F96C4830
:109CA00005F08EF96B4877E76B4805F089F968484D
:109CB00005F086F9B7F908206848294607E34146C8
:109CC000674805F001FB28B9324605212846FFF711
:109CD000FBFB4EE34146634805F0F6FA04460028D4
:109CE00063D13146604805F0EFFA08B9002332E04D
:109CF00031465E4805F0E8FA0028F7D031465C4866
:109D000005F0E2FA08B9012325E03146594805F08B
:109D1000DBFA0028F7D03146574805F0D5FA08B9E4
:109D2000022318E03146554805F0CEFA0028F7D056
:109D30003146534805F0C8FA08B905230BE031460F
:109D4000504805F0C1FA0028F7D031464E4805F0DA
:109D5000BBFAB8B9062301263B720022009607F130
:109D6000080318212846FAF74DFB002812DA474865
:109D700005F026F9387AFFF769FA364805F0AAF9AE
:109D800034464FE33146424805F09EFA0028E1D0C0
:109D9000404801E72946404805F012F9387AFFF7B4
:109DA00055FA2C4805F096F93CE341463B4805F04E
:109DB0008BFA10B9324616210EE04146384805F0BC
:109DC00083FA10B93246202106E04146354805F0B5
:109DD0007BFA28B9324627212846FFF741FBC8E223
:109DE0004146314805F070FA0446002840F097805B
:109DF00031462E4805F068FA002859D1012363E066
:109E000099240108792101083E2201082C24010827
:109E1000272001082C210108AE240108D9240108BB
:109E20002E1E0108EC1D0108F11D0108FC1D010892
:109E3000F3140108061E0108FB1401080B1E01089B
:109E40000F1E0108131E01081A1E0108D11901086E
:109E50001315010838350108E71901080E1A010821
:109E6000201E0108240D0108281E0108981401086D
:109E7000072301089C140108EB0C0108AA1401082F
:109E80002C1E0108B5140108321E01087B1E0108B2
:109E9000A21401083A1E01089A1E0108C21E0108F8
:109EA000CA1E0108D71E0108E51E01084E1D010843
:109EB0003146B04805F008FA00289FD03146AE4838
:109EC00005F002FAC8B900234FF001083B720022E6
:109ED000CDF8008007F108032A212846FAF792FA04
:109EE000002812DAA54805F06BF8A54805F068F8D7
:109EF000A44805F0EFF8444694E23146A24805F044
:109F0000E3F90028DFD0A14846E6A14805F058F85B
:109F10009B4805F055F8324629469E48D7E1414610
:109F20009D4805F0D1F90446002872D1304605F06D
:109F3000A7FB4FEA500909F1070323F00703EA469C
:109F40000E28ADEB030D83460DF1080801D19348AF
:109F500006E0102801D1924802E0202804D191485F
:109F600005F02EF8002117E0302801D18E48F7E7E0
:109F7000402801D18D48F3E7802801D18C48EFE7D4
:109F80008C4805F01DF817E0421C12D04A0800EB7F
:109F9000031008F8020002318B450FD9705CFFF7FF
:109FA00013FA721878605078FFF70EFA7B685A1C23
:109FB000EAD1814805F08EF8012428E0CDF8009020
:109FC000434600222B212846FAF71CFA002807DA1C
:109FD0006A4804F0F5FF794804F0F2FF6948E9E7C0
:109FE0006B4804F0EDFF754804F0EAFF2946744819
:109FF00004F0E6FF4546C144A94505D015F8011B0C
:10A00000704804F0DDFFF7E75E4805F063F8D546D9
:10A0100008E24846FFF796F9C0E56B49B06805F0DD
:10A0200053F9044600286AD1B8F1030F01D1316811
:10A0300027E0A8F10308B8F1010FD6F80C9022D060
:10A040006249D6F800A0484605F03EF920B9D6F896
:10A0500010904FF0020A17E05D49F06805F034F9FE
:10A0600020B9D6F810904FF0010A0DE05949F06878
:10A0700005F02AF920B9D6F810904FF0000A03E055
:10A0800051465548ABE182462F2140224846FEF713
:10A0900060FE431E802B0646494628BF402607F136
:10A0A00008005FFA86FB03F029FD00283AD0B8F1DA
:10A0B000010F07D03B7AFF2B04D1BAF1010F07D073
:10A0C000464869E5BAF1020F14BF4023412300E07E
:10A0D00040235A4607F108012846F8F71DFD18B934
:10A0E0003F4804F06DFF59E54FF0FF334361836152
:10A0F00032462B4649463B4804F062FF92E13A491A
:10A10000B06805F0E1F80446B8B9B8F1030F02D120
:10A110003168364863E1F66807F10800314603F01C
:10A12000EDFC08B9324837E507F108012846F8F791
:10A130001BFD2A4631462F48C9E02F49B06805F07B
:10A14000C3F80446002869D1B8F1030F02D1316881
:10A150002A4844E1F06804F0D9F9A0F5A063B3F50A
:10A160007B4F06464ED34FF6FF724FF4A061244852
:10A170009FE000BFED1E0108281E0108D11901084B
:10A180005E1501083835010898140108F01E010811
:10A19000E7190108F519010803200108201F01082B
:10A1A0003D1F01085A1F0108781F0108961F01086A
:10A1B000B41F0108D21F0108EC1F0108691501082E
:10A1C000072001081E200108232001087320010830
:10A1D0007B2001088520010827200108B220010802
:10A1E000DE20010801210108282101082C21010895
:10A1F0008D2001084F2101087521010879210108EE
:10A20000942101082846F8F769FC08B98848C3E496
:10A21000A0F8C8612A463146864858E08649B068A9
:10A2200005F052F8044670BBB8F1030F17D083490C
:10A23000F06805F049F8002800F0EA808049F068ED
:10A2400005F042F8002800F0E6807E49F06805F04D
:10A250003BF8002800F0CA80F1687B48BAE04FF074
:10A26000FF0919F0010F04D0224601212846FFF70B
:10A270009DF919F0020F3FF491AC224602212846C5
:10A28000FFF794F98AE47149B06805F01DF80446B7
:10A2900000BBB8F1030F02D131686D489FE0F06850
:10A2A00004F034F9FF28064606D96A484FF6FF72D3
:10A2B000002104F085FE71E42846F8F70FFC08B988
:10A2C000654869E480F8CA6164482A46314604F06A
:10A2D00077FEA7E0D6F80880614998F80030D6F8F4
:10A2E00000902D2B08BF08F1010840460CBF002646
:10A2F000012604F0E9FF10B93246132136E059492E
:10A30000404604F0E1FF10B9324612212EE05649D2
:10A31000404604F0D9FF10B93246142126E05349D3
:10A32000404604F0D1FF10B9324615211EE05049D5
:10A33000404604F0C9FF10B93246192116E04D49D4
:10A34000404604F0C1FF10B932461F210EE04A49D1
:10A35000404604F0B9FF10B932461E2106E04749D5
:10A36000404604F0B1FF30B9324623212846FFF7BA
:10A3700005F8044656E04249404604F0A5FF04466D
:10A3800078B92846FEF772F808B93E4804E426B1C9
:10A390000123037129463C481CE0067129463B48CD
:10A3A00018E03B49404604F08FFF0446A8B9284610
:10A3B000F8F794FB10B93748FFF7EEBB2EB1012137
:10A3C000F8F7A3FB2946344804E03146F8F79DFB33
:10A3D0003248294604F0F4FD24E03148494604F0AF
:10A3E000EFFDFFF7DBBB2F48FFF7D6BBB8F1040F3B
:10A3F0000AD04FF0020905222B49306905F0AEF969
:10A40000B0FA80F464092CE704464FF0020930E703
:10A410004FF0FF0901E04FF00109B8F1040FEAD154
:10A42000002421E720461C37BD46BDE8F08F00BF61
:10A43000BC210108D6210108F9210108A01A010850
:10A44000FF210108D0100108022201083B22010867
:10A450003E2201085822010886220108A62201088E
:10A46000CF220108D7220108DF220108E7220108D4
:10A47000EF220108F3220108F82201080023010855
:10A480000D23010812230108302301085723010876
:10A490007F23010887230108BB230108F323010858
:10A4A0002C2401087A1D01082C1E01082DE9F04F0B
:10A4B00087B006AF0546884691469A4605F0E0F813
:10A4C00028448542A0EB050413D010F801392F2B46
:10A4D00005D1601C284404F019F806460BE03A2B1D
:10A4E00001D02E2BEDD1284605F0CAF800260446EF
:10A4F00001E00024264604F1080323F00703ADEB36
:10A50000030D0DF1180B621C0021584604F050FC9D
:10A5100029462246584604F0B1FB404605F0B0F803
:10A520005946164803F0EAFAD0B1144D10244146BA
:10A53000134803F0E3FAD0B1114B10220021360684
:10A54000039102920193CDF810A0009623462A466B
:10A5500049460C4802F014FC0437BD46BDE8F08FB4
:10A5600003F0DCFF6A230360074D0424DFE703F0F8
:10A57000D5FF6A2303600422044BDFE7CC500020A0
:10A58000BC500020801D0020E0500020DC50002046
:10A5900001282DE9F34105460C4603D17A4802F023
:10A5A00099FDBBE002281AD14968784804F08CFE76
:10A5B000002800F0B1806168754804F085FE08B994
:10A5C0007448B8E06168744804F07EFE014620B922
:10A5D0006D4802F0C4FC7148ADE07148ABE053DD5A
:10A5E00049686A4804F070FE58B16168684804F030
:10A5F0006BFE30B16168684804F066FE08B16948D6
:10A6000099E0032D25D16168634804F05DFE05469D
:10A6100090B9A06803F07AFF04B22046FAF7ECF88C
:10A62000214628B1584802F09AFC21465E4800E0D5
:10A630005E4804F0C5FCA2E0A1685D4803F05EFA44
:10A64000054600286CD0102259494F4802F069FC99
:10A6500064E0052D18D161684C4804F035FE0028EF
:10A6600068D1E168534804F02FFE0546002861D107
:10A6700001A8FAF7B5F8012831D14FF0FF33BDF941
:10A6800004202169A0683DE0072D3ED161683F4864
:10A6900004F01AFEC8B9E168464804F015FEA0B9F6
:10A6A0006169454804F010FE054670B901A8FAF743
:10A6B00097F8012813D1A069BDF90480A66827691D
:10A6C00003F024FF424603461AE061682F4804F075
:10A6D000FBFD20B9E168374804F0F6FD08B13748C2
:10A6E00029E06169364804F0EFFD05460028F6D1FF
:10A6F000A069A668276903F009FF4FF0FF3302B293
:10A7000039463046FFF7D2FE39E0092D12D1616893
:10A710001E4804F0D9FD90B12A480CE000252EE037
:10A7200003F0FCFE6A23036004222749164802F066
:10A73000F8FB24E0254804F0CDFC01251FE0E1688A
:10A740001C4804F0C1FD0028E6D161691C4804F0F2
:10A75000BBFD0028E0D1E169174804F0B5FD0546CE
:10A760000028D9D1A069A668276903F0CFFE8046EA
:10A77000206A03F0CBFE0FFA88F20346C0E72846B2
:10A7800002B0BDE8F08100BF801D00202320010839
:10A7900028210108F3260108872701088D270108D1
:10A7A000AE2701082B2801087B280108AF280108E3
:10A7B000CC500020CD280108432A0108D1280108E7
:10A7C0004C2A010813250108E0500020502A0108F6
:10A7D00013B5044601A8FAF703F820B1BDF9040047
:10A7E000031B5842584102B010BD000000F00700A2
:10A7F000072813D8DFE800F00406080A0C0E121030
:10A8000008480CE008480AE0084808E0084806E064
:10A81000084804E0084802E0084800E0084804F05E
:10A82000CFBB00BFA02A0108AD2A0108BA2A01083F
:10A83000C72A0108D42A0108E12A0108EE2A0108E2
:10A84000FB2A010800F03000202805D0302805D070
:10A85000102805D1044804E0044802E0044800E060
:10A86000044804F0ADBB00BF082B01080B2B010806
:10A87000102B0108B02B0108F0B5012893B0064653
:10A880000D4607D16B4804F025FC6B4804F022FC10
:10A89000002005E04968694804F016FD30BBF1E787
:10A8A00002F040FF0446002800F0C1802822214623
:10A8B00008A8FEF75DFA237EB4F91A60054604F194
:10A8C0001002182102A802F099FF324603462946D9
:10A8D0005B4804F075FB607EFFF788FF607EFFF742
:10A8E000B1FF584804F0F6FB2046D9E7012E40F3AB
:10A8F0009680022E74D06968534804F0E5FC044643
:10A90000002857D1023E012E02D0022E0CD022E0A8
:10A9100008A8F9F765FF012898BFBDF92060AF6866
:10A9200088BF264600251CE0AF6808A8394603F01A
:10A93000E5F828B9A86803F0E9FDEF6806B2F1E789
:10A9400002A8F9F74DFF012898BFBDF90860ED682E
:10A9500088BF264605E0A86803F0D8FDEF682D699A
:10A9600006B23046FFF734FF08B9384805E03946EB
:10A9700008A803F0C3F820B9354804F0ABFB012464
:10A9800055E04DB108212A460DEB010002F062FFAF
:10A99000034610B92F48F0E72B460022009208A981
:10A9A00002AA304602F01EFE08B92B48E5E73946F8
:10A9B0002A4812E069682A4804F086FC044678B9FF
:10A9C000AD6808A8294603F099F80028D4D008A952
:10A9D000204602F09DFE2348294604F0F1FA26E0C5
:10A9E0006968214804F070FC0446C0B902F09AFE80
:10A9F0002146054655B119B1B1F91A0002F088FE99
:10AA0000284602F08FFE29460546F3E719B1B1F951
:10AA10001A0002F07DFE154804F0D2FA07E02B6818
:10AA200000931A461946124804F0CAFAA7E72046CE
:10AA300013B0F0BD142B0108632B01084D1301085E
:10AA4000B22B01083835010823200108C72B010863
:10AA50008D200108E72B0108122C0108422C010867
:10AA600028210108742C01082C1E01089D2C0108C6
:10AA7000BC2C010870B501288AB00C460DDD486871
:10AA800003F044FD05B22846FFF7A2FE30B9216865
:10AA9000164804F095FA012025E00025144804F03A
:10AAA00019FB144804F016FB002002F053FE044684
:10AAB000C8B1B4F91A600DB1AE4212D128222146B4
:10AAC0006846FEF755F9314602460B4804F078FA1D
:10AAD000607EFFF78BFE607EFFF7B4FE074804F050
:10AAE000F9FA2046E1E70AB070BD00BF682D010801
:10AAF000812D01087E2B0108B52D0108383501088C
:10AB000008B501460B4804F05BFA0B4804F0E2FA82
:10AB10000A4804F0DFFA0A4804F0DCFA094804F0B5
:10AB2000D9FA094804F0D6FA0848BDE8084004F00C
:10AB3000D1BA00BFC32D01081F2E0108292E01081C
:10AB4000372E0108912E0108A52E0108B62E010806
:10AB50000C4AF0B514880830260AE5B200238B426F
:10AB600009D2FF2C85BFC718C654C5547D708CBF51
:10AB700002330133F3E781BF138809181B0A01F878
:10AB8000013CF0BD680200202DE9F0430D4685B080
:10AB900002210446F9F7E9FE032107462046F9F7AA
:10ABA000E4FE07B108B9274845E08668264AB3881D
:10ABB000F48812885BBA9BB264BA9A42A4B239D1C3
:10ABC0002249234B0A881B889A4203D9944203D313
:10ABD000012307E0944204D39C428CBF002301234D
:10ABE00000E0002333B3BF68D0F80C9019489442BA
:10ABF00098BF013207F1080898BF0A802822414611
:10AC0000FEF7B6F84FF47A72B388B5FBF2F102FBA7
:10AC1000115502910395FA7901925BBA02469BB2F3
:10AC2000494600940C4804F0CBF9404602F09AFDE6
:10AC3000012003E0094804F04DFA002005B0BDE80A
:10AC4000F08300BFD12E0108680200200C510020C3
:10AC50000E510020E4500020082F01084B2F01085E
:10AC60002DE9F04F99B081460C461022002114A81E
:10AC700004F09EF881231593994BB9F1010F1B88BD
:10AC8000ADF85C303BDDB9F1020F00F0C2816068C5
:10AC900003F03CFC051ED4BF4FF000084FF0010844
:10ACA00008F101034FEA830754F82330089308F1B1
:10ACB0000203D8BF0325994505DDE319586803F061
:10ACC00025FC049001E00423049308F10303994553
:10ACD00005DDE319986803F019FC064601E04FF41E
:10ACE0007A7608F10408C14505DD2744F86803F0C9
:10ACF0000DFC099000E00995049B002B03DA206805
:10AD0000FFF7FEFE3FE04FF0FF3225210898FEF7E7
:10AD100020F804B2621C089910A808BF002402F0B1
:10AD2000EDFE08B96F482CE008226F4910A803F027
:10AD300073FF50B19DF84030FF2B05D19DF8413095
:10AD400003F00F03022B00D0A4B10EA8F9F748FDC1
:10AD500044B1002800F05881BDF938309C4240F0E1
:10AD6000538106E0012802D1BDF9383001E05F4887
:10AD700007E01C4614A90320F9F77EFD002804DA39
:10AD80005B4804F0A7F901204BE1F5F733FE4FF4DF
:10AD90007A7373430D9300220023CDE90A01002743
:10ADA000CDE906234FF0FF332E460593BA46BB4646
:10ADB000013E731C4F4A00F006814E4B19884E4BE2
:10ADC0001A88013292B21A80049B009380200023DB
:10ADD00002F046FB804698B104998068FFF7B8FE00
:10ADE00010AA0021404602F09BFB814640B1ACB165
:10ADF0004FF0FF3308220021F9F73AFF814618B9D6
:10AE00003E4804F067F9D3E7836800221A705A704D
:10AE10005A719A711A715A8083685C800020F6F723
:10AE2000B1FC4B46804640F2022235490220F9F738
:10AE30006FFA0C9038B9334804F04CF90C99484635
:10AE4000FAF708F8B4E7304A00230EA800F0B8FE7D
:10AE500000282DDBBDF83A2040F201239A4220D190
:10AE60000020F6F78FFCDDF83C90C8EB0008414667
:10AE70004846FFF789FE002183444846F9F7EAFF78
:10AE8000059B474538BF4746434528BF4346059382
:10AE9000DDE9062312EB080243F10003CDE90623A6
:10AEA0001AE00F4B19880EA809B2F7F703F813E060
:10AEB000164804F00FF90FE00EA8F7F79DF80028E8
:10AEC00028DDBDF83A304345F6D1114804F078F852
:10AED00000210F98F9F7BEFF40F20128ECE700BF10
:10AEE000DC020020682F010828110108812F0108C9
:10AEF000CF2F0108680200200E510020BC1D010860
:10AF00000000FFFFEF2F010840420F001A30010838
:10AF1000273001081EB100210D9800F00DFE099B9D
:10AF20000AF1010A534502D0002E7FF441AFF5F734
:10AF300061FD089980463C4804F042F8BBF1000FDF
:10AF4000C6EB050A38DD5246DDE90601D31703F0EA
:10AF500051F9DDE90A23B8EB02029046334AB8FB07
:10AF6000F2F1642302FB11828DE806000C905A4630
:10AF7000514603FB0BF32E4893FBFAF3C3F1640332
:10AF800004F01EF84FF47A72B7FBF2F002FB107E69
:10AF900001900C980C9BB3FBF2F302FB13000090A2
:10AFA00005980599CDF808E0B1FBF2F102FB11021A
:10AFB000204804F005F803E051461F4804F000F86B
:10AFC0004FF0000AF4E61D4B00211980138814A9E4
:10AFD000013303201380F9F771FC40F201240EA81D
:10AFE000F7F70AF800280BDDBDF83A30A342F6D196
:10AFF000134803F0E5FF00210F98F9F72BFFECE76A
:10B00000BBFA8BF040090CE021460E4803F0D8FF54
:10B01000B9E66368089304274FF0000803250497F6
:10B0200053E619B0BDE8F08F6C30010840420F00C4
:10B0300088300108D1300108053101080E51002087
:10B04000273001083C3101089368013B002B10B404
:10B05000936008DA9469A34202DBCBB20A2B02D1D7
:10B0600010BC04F011BD1368581C10601970C8B2F0
:10B0700010BC704710B503F049FA04B22046F7F748
:10B080002DFD20B9064804F025F8012010BD20460A
:10B09000FAF73CF82146034803F092FF002010BD68
:10B0A000623101087E31010830B58FB00D4603F0E2
:10B0B0002DFA2946C4B2684602F020FD18B90E48A0
:10B0C00004F008F810E000231A4669462046FAF713
:10B0D00099F858B92822694604A8FDF749FE224686
:10B0E0000146064803F06CFF012003E0044803F02A
:10B0F00067FF00200FB030BDAC310108A50F01087B
:10B10000D70F010810B503F001FAC4B22046FAF7D0
:10B1100071FF10B92146084804E0FBF768F82146A2
:10B1200020B9064803F04CFF012010BD044803F08D
:10B1300047FF002010BD00BFDB31010804320108C9
:10B140002B32010830B58BB003F0E0F9C5B22846C8
:10B15000FAF750FF044620B90A4803F0BBFF01206C
:10B160000EE0383000F088FC282204F1080168461F
:10B17000FDF7FEFD2A460146034803F021FF0020AB
:10B180000BB030BD4B3201087332010830B58BB0C3
:10B1900003F0BCF9C5B22846FAF72CFF044620B9E3
:10B1A0000A4803F097FF01200EE0383000F0AAFCB7
:10B1B000282204F108016846FDF7DAFD2A46014617
:10B1C000034803F0FDFE00200BB030BD4B320108F8
:10B1D000B232010870B58CB003F098F9C6B23046AF
:10B1E000FAF708FF0125044620B9134803F072FF5F
:10B1F00028461EE0114A90F82730B2F9000094F872
:10B200002820019294F82620009205FA03F340F6D4
:10B21000011204F1380100F045FC282204F1080174
:10B2200002A8FDF7A5FD32460146054803F0C8FE19
:10B2300000200CB070BD00BF4B320108903E0020D2
:10B24000F332010808B504490020FAF777F90348FA
:10B2500003F040FF002008BDFE1001083433010850
:10B2600013B5234C234803F035FFA36900932269EB
:10B27000A3682168204803F0A3FEE3690093626994
:10B28000E36861681D4803F09BFEA36B0093226B8B
:10B29000A36A216A1A4803F093FEE36B0093626B82
:10B2A000E36A616A174803F08BFEA36D0093226D79
:10B2B000A36C216C144803F083FEE36D0093626D70
:10B2C000E36C616C114803F07BFEA36F0093226F67
:10B2D000A36E216E0E4803F073FEE36F0093626F5E
:10B2E000E36E616E0B4803F06BFE002002B010BDF0
:10B2F00000440020493301088C330108BE330108A3
:10B30000F03301082234010854340108863401085E
:10B31000B8340108EA3401082DE9F041514C524893
:10B3200092B003F04DFE63780BB9504800E05048EE
:10B33000504DDFF86C8103F043FE286809218268D4
:10B34000FFF782FE28680A218268FFF77DFE4A48DF
:10B3500003F036FE002606EB08031B790BB94348C1
:10B3600000E04348434F03F02BFE28680921826820
:10B370002436FFF769FE6C2EEDD13868394D8268AE
:10B380000A21FFF761FE38680A218268FFF75CFE38
:10B39000F5F730FB637806460F46002B5DD0B5F815
:10B3A0008A0095F880302978B5F92C200290B5F8FC
:10B3B00088000190D5F88400008800902F4803F0A1
:10B3C000FFFDE86E296F801B61EB0701002871F11A
:10B3D000000305DB2A4A002302F00CFF064600E0CA
:10B3E0000026236A274993F98C50282208A8FDF7E4
:10B3F000BFFC94F8363094F83270228E069613F023
:10B40000020F214B214918BF1946638F059394F809
:10B410003830049394F82630039394F827300126AB
:10B420009E4025EAE5758DE86200194B1949022F07
:10B4300008BF0B460146184803F0C2FDE46964B139
:10B44000611D282208A8FDF793FCE369E28A014602
:10B45000124803F0B5FD2468F1E7002012B0BDE802
:10B46000F08100BF704300202835010839350108FC
:10B470003D3501086C0200204135010850350108B6
:10B4800040420F00784300204E1D0108281E01088D
:10B49000213501081C35010894350108EB350108F8
:10B4A000E43E002038B50546084603F02FF8C4B244
:10B4B0002046FAF79FFD28B921460B4803F080FD8E
:10B4C000012038BD083015B1FBF704F801E0FBF7A7
:10B4D00008F8064B064A0748002D08BF1A462146C1
:10B4E00003F06EFD002038BDDB3101082136010874
:10B4F0001C3601082836010838B50C4603F006F85A
:10B50000C5B22846FAF776FD28B929460B4803F05C
:10B5100057FD012038BD90F83630094923F0020369
:10B5200043EA440380F83630064B0748002C08BF36
:10B53000194603F045FD002038BD00BFDB3101088E
:10B54000383501081712010851360108012838B5AD
:10B5500005460C4603DCBDE83840FFF7DDBE634915
:10B56000606803F0B1FE0028F5D0032D09D16049D1
:10B57000606803F0A9FE88B9A068BDE83840FFF70D
:10B5800079BD042D0AD15B49606803F09DFE28B99E
:10B59000E168A068BDE83840FFF786BD564960689D
:10B5A00003F092FE30B9032D7AD1A068BDE838408F
:10B5B000FFF7A8BD5149606803F086FE00BB042D6B
:10B5C0006ED14F49A06803F07FFE20B9E068BDE866
:10B5D0003840FFF7B7BD4B49A06803F075FE20B9AE
:10B5E000E068BDE83840FFF7D1BD4749A06803F0E7
:10B5F0006BFE002854D1E068BDE83840FFF7EABD93
:10B600004249606803F060FE58B9032D48D14049B3
:10B61000A06803F059FE002842D1BDE83840FFF78A
:10B6200011BE3C49606803F04FFE20B9032D37D1AD
:10B63000A168012007E03849606803F045FE30B991
:10B64000032D2DD1A168BDE83840FFF72BBF33494A
:10B65000606803F039FED0B9022D21D03049A068CE
:10B6600003F032FEE0B9052D1AD12E49E06803F04F
:10B670002BFE08B9012105E02B49E06803F024FE08
:10B68000014668B92069BDE83840FFF735BF274952
:10B69000606803F019FE18B9BDE83840FFF7E0BD57
:10B6A000234803F017FD234803F014FD224803F05C
:10B6B00011FD224803F00EFD214803F00BFD214847
:10B6C00003F008FD204803F005FD204803F002FDCB
:10B6D0001F4803F0FFFC1F4803F0FCFC1E4803F06A
:10B6E000F9FC1E4803F0F6FC002038BD793601084D
:10B6F000641201087E360108833601088636010887
:10B700002C1E01088E36010893360108440E0108EC
:10B71000993601081C360108213601082E1E010841
:10B720009D3601084E1D0108281E0108F921010857
:10B73000A1360108B9360108F33601082C37010893
:10B74000653701089E370108D53701081838010808
:10B75000613801089E380108C33801080E39010814
:10B760002DE9F04301288DB005460C4605DC09683B
:10B770002D4803F025FC2D481DE0182200210DEB7B
:10B78000020003F015FB0423069361687B2307A8DE
:10B79000ADF82E3002F0B2F9022D04D0A06802F00C
:10B7A000B5FE014601E041F2883106A800F046F8F6
:10B7B000002804DA1E4803F08DFC01202DE000F083
:10B7C000A1F804460D46F5F715F915A3D3E90023B2
:10B7D0008018594100196941164A002302F00AFDF8
:10B7E0000CAB43F81C0D184603F0E0F802694469FD
:10B7F000C6688768D0F80480D0F80090551C00F027
:10B8000081F804F26C7403908DE8800333462A4675
:10B810002146094803F0D4FB00200DB0BDE8F083B9
:10B82000006043B7EF26F8FF3A3901085F39010895
:10B830007739010840420F009039010800232DE9B3
:10B84000F34102460E462A481946FCF72DFE002811
:10B850004ADB284D30220021284603F0A9FA2B7834
:10B86000234823F03F0343F023032B7030220023AF
:10B870002946FCF7EBFE041E03DA1D48FCF76AFEBE
:10B8800031E0002433460094302229461848FCF762
:10B890006FFE061E164803DAFCF75CFE304623E016
:10B8A000FCF758FE01211448F6F790F9D5F82880E6
:10B8B000ED6AF5F79FF82DBA0646E8200F460023FB
:10B8C0000E4AA5FB000102F045FC0C4B98FA88F8E3
:10B8D000E3FB0801801B0A4B61EB0701C3E9000190
:10B8E0000548F6F7A3F9204602B0BDE8F08100BF95
:10B8F00010510020BC510020B851002040420F00E0
:10B90000B0510020D0B5074C01212046F6F75EF972
:10B91000054BD3E900672046F6F788F930463946EB
:10B92000D0BD00BFB8510020B051002030B5036831
:10B9300045688468C168056085EA040223F0004315
:10B94000534083EA430381EA510183EA010242F34F
:10B95000000583EA8223C2600169426929402A40C6
:10B960004C4053404460836030BD036823F0004383
:10B9700063B9436853B9836843B9C36833B9542181
:10B9800049224E234FF0590C80E80E1070470000FA
:10B9900038B5036943604369836083690160044685
:10B9A000C3600F4801256B1E03F0030305F003027B
:10B9B00054F8233054F8221083EA937300FB0353A6
:10B9C00001354B40082D44F82230ECD12046FFF7DA
:10B9D000CCFF2046FFF7AAFF013DFAD138BD00BFDA
:10B9E0006589076C2DE9F341856804461DB919493D
:10B9F0000320F5F7F9F8427843689340C268C2EB38
:10BA000005086A0093424FF000072CBF82608360F4
:10BA1000478038BF5D088668FDF766FA711BB0FB8A
:10BA2000F1F202FB11000544B4F91030E5604FF467
:10BA30007A7245446A43019304F11C030093A262A5
:10BA4000E7623B4604F1300000F0AAF802B0BDE81E
:10BA5000F08100BF5D0C010810B5428803789A425E
:10BA6000044600D313B96369A06998472046BDE82E
:10BA70001040FFF7B7BF0000826843689A4210B5D4
:10BA8000044603D806490320F5F7AEF83030F5F741
:10BA900027F86368A3602046BDE81040FFF7A2BF07
:10BAA0005D0C0108F8B50C46174606469DF81810BF
:10BAB0009DF81C201D461BB910490320F5F794F88A
:10BAC00003FA01F00E4B9842F6D8002363802270EF
:10BAD000656026826170FDF707FAC5EB8503B0FB50
:10BAE000F3F202FB13000544E560A56026822462A0
:10BAF000E7832046BDE8F840FFF774BF5D0C0108FE
:10BB0000FEFFFF7F3030F4F7EBBF43880133438003
:10BB10007047F6F78BB8B0F90010F6F7A7B938B54B
:10BB200004460020F5F72EFE05460020F5F72AFE14
:10BB3000401BA042F9D338BD30B587B004460D464E
:10BB4000F4F799FC40B11DB10E490320F5F74CF80C
:10BB50002046FFF7E4FF13E00B4B009003900290A8
:10BB6000012168460493CDF814D0F6F72FF821464A
:10BB700001A82A46F4F7E6FF01216846F6F726F801
:10BB800007B030BD5D0C010813BB000830B4034D95
:10BB9000C560026130BC1380F4F7B4BF17BB000866
:10BBA00070B41146039ABDF91050044EC66002618C
:10BBB00015801A4670BCF4F7C5BF00BF17BB00085C
:10BBC00070B58AB00021079106911049098803AC2D
:10BBD00009B2054643F23906019105A80094ADF873
:10BBE0000E600494FFF7DCFF2846F6F708FA6B882E
:10BBF000B34202D16B68A34204D005A8F4F770FFEA
:10BC0000012001E04FF0FF300AB070BDDC020020DF
:10BC100010B5084B0446182240F83C3B03F02EF8C0
:10BC2000082384F85630002384F8543084F85730C1
:10BC300010BD00BFF039010837B5044600F03CFBE9
:10BC400094F854301BB90321204600F060FA002517
:10BC50000821684684F83650258701F0EBFF9DF8EF
:10BC60000030019A23F0010343F002038DF8003005
:10BC7000009B12BA1BBA204600F000F9BDF8001074
:10BC800049BA204689B200F0E5F82046232100F0A9
:10BC900028F920461A2100F015F92946204600F01F
:10BCA0003DF920460122202100F0B8F9204601226A
:10BCB0004FF4807100F0B2F92A4620464FF400514B
:10BCC00000F0ACF9204601224FF4804100F0A6F9C3
:10BCD000204601224FF4805100F0A0F9012384F89E
:10BCE0002830802220460C2100F057FA04212046FB
:10BCF00000F065FA042100F0FD02204600F04DFA44
:10BD00000321204600F05BFA032100F0F0022046F8
:10BD100000F043FA082220460E2100F03EFA0F21DF
:10BD2000204600F04CFA1621204600F0F0F903B04E
:10BD300030BD10B590F857300133044680F85730C5
:10BD4000204600F094FAA0F11103DBB2012BF7D9E1
:10BD5000192818BF84F856001921204600F0D7F999
:10BD6000022384F8553010BD70B51D4690F855304B
:10BD70006E1C1344144680F8553013460A46F1B23F
:10BD800000F02FFA601970BD10B5012300F15502C3
:10BD90000021044600F025FA02221146204600F058
:10BDA000FCF963683BB1228F120504D520460321BC
:10BDB000BDE81040184710BDF8B50821044600F052
:10BDC000A6F915210746204600F0F9F960F07F0238
:10BDD000D2B215210646204600F0DFF906212046A2
:10BDE00000F095F90821204600F0E9F960F07F02A3
:10BDF000D2B20821204600F0D0F90121204600F0FF
:10BE0000DEF903060546F8D532462046152100F036
:10BE1000C4F90821204600F07AF93946204600F09E
:10BE200076F9C5F38010F8BD38B50D4602210446F9
:10BE300000F0B3F9162D07D0204600F018FA85421D
:10BE4000FAD184F8545038BD204600F010FA1F286B
:10BE5000FAD0F6E710B50A0A044601F07F0180F82F
:10BE60002D2080F82C10202100F097F994F82C2038
:10BE700020462121BDE8104000F08FB92DE9F8439C
:10BE8000054616461F4600F12D0800246FF00709ED
:10BE9000E2003046394602F051F909FB04F208F895
:10BEA000010F38323046394602F048F904F12401D6
:10BEB000C2B2C9B22846013400F06FF9082CE7D1AC
:10BEC000BDE8F883A1F10B020F2A07D890F83720BC
:10BED0008A4203D080F8371000F00ABA7047002079
:10BEE000704737B50D0A4185CAB22221044600F0D9
:10BEF00054F92A462321204603B0BDE8304000F023
:10BF00004CB9000008B5052100F059F9024B00F0CA
:10BF10000F0033F9100008BDD0390108113109B202
:10BF20001429A8BF142121EAE171024B5A5C0521B2
:10BF300000F033B9BB39010808B52C2100F03FF9F6
:10BF4000C0F3071008BD38B50C462C21054600F09B
:10BF500036F9072C28BF072400F00F0040EA04122E
:10BF6000D2B228462C21BDE8384000F016B908B5F9
:10BF70002C2100F024F9C0F3420008BD0529A8BF18
:10BF80000521002938B50C46A8BF0C464FF02C01FE
:10BF90000546B8BF072400F012F920F00E0040EA71
:10BFA0004402D2B228462C21BDE8384000F0F5B852
:10BFB00038B505460C4699B10A782D2100F0EDF808
:10BFC0002E21284600F0FBF8637800F0F80203F019
:10BFD00007031A4328462E21BDE8384000F0DDB89B
:10BFE00038BD08B5092100F0EAF800F00F00400064
:10BFF0005B3840B208BD0029C4BF494249B25B3139
:10C00000C1F3430242F0C002092100F0C6B808B5EE
:10C01000072100F0D4F85B3840B208BD10B5038F9B
:10C020000446B2B30B43B1F5807F03870AD002D830
:10C03000202925D010BDB1F5007F0ED0B1F5005FED
:10C0400020D010BD00F12E01FFF7B2FF04212046E1
:10C05000FFF794FF53222F2153E02E2100F0AFF879
:10C0600040F01002D2B22E21204600F096F817219F
:10C07000204600F0A4F840F00202D2B2172140E0BE
:10C080002E212BE00E2100F09AF840F00402D2B2EB
:10C0900036E023EA0103B1F5807F03870AD002D896
:10C0A000202921D010BDB1F5007F09D0B1F5005F86
:10C0B00021D010BD4FF0FF31BDE81040FFF75EBF4B
:10C0C000172100F07CF8172100F0FD02204600F057
:10C0D00064F8238F9B0619D52E21204600F06FF8B7
:10C0E00000F0EF022E210CE02E2100F068F840F065
:10C0F0001002D2B2F6E70E2100F061F800F0FB0268
:10C100000E212046BDE8104000F047B810BD70B5C4
:10C1100004460D46204600F0AAF8A0F11103DBB258
:10C12000012B0646F6D91F28F4D0032D02D12A464A
:10C13000082126E0A84227D0162801D1192D02E0B7
:10C14000192807D1162D0AD1092211462046FFF7DA
:10C150006BFE04E00F2802D1204600F094F80F2D6A
:10C160000DD103212046FFF7D2FF2946204600F0DB
:10C1700026F8E06CF5F77CFA84F8545004E02A467F
:10C1800029462046FFF750FE304670BD90F84030FB
:10C19000416CC06B0022F5F7DBB870B504460D4664
:10C1A0001646FFF7F3FF334645F0C002616CE06BC3
:10C1B00001F091FEE06BBDE87040F5F709B938B5C4
:10C1C00004460D46FFF7E2FF45F080020023616C54
:10C1D000E06B01F080FE0546E06BF5F7F9F82846C4
:10C1E00038BDF7B504460F4615461E46FFF7CEFF8D
:10C1F000616CE06B4023012201F05CFE3B46616C08
:10C20000E06B012201F056FE0022E06B01960092E5
:10C210002B46616CF5F7F8F8E06B03B0BDE8F04031
:10C22000F5F7D6B810B50446FFF7B0FF616CE06BC8
:10C2300020230122BDE8104001F03CBE07B58DE887
:10C2400006000023416CC06B0122F5F7DDF803B056
:10C250005DF804FB10B50446416CC06B012300225D
:10C2600001F028FEE06BBDE81040F5F7B1B808B565
:10C2700090F854300F2B04D00121FFF7A0FF00F0FD
:10C280001F03184608BD10B50446FFF7F0FF0F283E
:10C2900011D1E06CF5F7F5F900214FF49970FFF733
:10C2A0004BFC01212046FFF78AFF00F01F00082801
:10C2B00084F85400F5D110BD10B50446006DF5F7B3
:10C2C000E0F900213E20FFF737FC206DF5F7D0F9AB
:10C2D00000213E20FFF730FC01212046FFF76FFFD1
:10C2E00000F01F0310F0170F84F85430F4D110BD84
:10C2F00038B508210446FFF70AFF08210546204605
:10C30000FFF75DFF94F8373000F0E00203F01F0301
:10C3100020461A430821FFF740FF29462046BDE882
:10C320003840FFF7F4BE43680BB10021184770474F
:10C330002DE9F0470446884616461F46FFF797FF4B
:10C340008146002C00F0D3800F2840F0DF80B8F148
:10C35000180F66D02046FFF796FFB8F1270F00F2BE
:10C360002B81DFE818F04200290128003300290161
:10C3700029013B002901290129012901290129015C
:10C38000290129012901550029018B008F007E0018
:10C3900029018400290129012901930097009B00AC
:10C3A0009F002901A300AA002901290129012901CF
:10C3B00029014E00BA00022F03D98B490320F4F75C
:10C3C00013FC31882046FFF745FD94E0082FF4D890
:10C3D000D6E900232046FFF751FD8CE0022FECD870
:10C3E00031882046FFF77DFD85E0012FE5D03178CB
:10C3F000A1F10B030F2B00F2EC802046FFF762FD4A
:10C4000079E0012FD9D03378002B40F0E2806CE046
:10C41000022FD2D8B6F900102046FFF77FFD022583
:10C42000D9E0012FC9D83378013B052B63D8DFE869
:10C4300003F00507620C1403082102E00F2100E05D
:10C4400016212046FFF763FECBE0238F5A0540F10B
:10C45000C8802046FFF798FCC3E02046FFF7ECFBBE
:10C46000BFE0327820212046FFF7D8FD43E0012FBE
:10C47000A3D831782046FFF766FD36E032784FF4D6
:10C48000806116E032784FF4007112E032784FF498
:10C4900000510EE032784FF480410AE032784FF4D8
:10C4A000006106E032784FF4805102E032784FF4B8
:10C4B00080712046FFF7B2FD17E0012F3FF67DAFF8
:10C4C000238FDB0503D43378052B40F2828096F965
:10C4D00000102046FFF752FD07E0012F3FF66DAF39
:10C4E00096F900102046FFF786FD012573E06FF0F6
:10C4F0001200BDE8F087B9F10F0F5DD03B46324620
:10C5000041462046BDE8F04701F056BCB8F1270F80
:10C51000F4D801A353F828F0EBC30008FDC40008C9
:10C52000B7C30008CDC30008FDC40008FDC400085F
:10C53000DDC30008FDC40008FDC40008FDC40008F8
:10C54000FDC40008FDC40008FDC40008FDC40008C7
:10C55000FDC40008FDC4000811C40008FDC40008A3
:10C560007DC4000885C4000863C40008FDC4000839
:10C570006FC40008FDC4000823C40008FDC40008FF
:10C580008DC4000895C400089DC40008A5C4000817
:10C59000FDC40008ADC40008BBC40008FDC4000809
:10C5A000FDC40008FDC40008FDC40008FDC4000867
:10C5B00003C40008DBC40008B8F1180F9ED06FF068
:10C5C00085050F212046FFF7A2FD15F1860F05D145
:10C5D00094E76FF01505B9F10F0FF2D02846BDE8CA
:10C5E000F0870120BDE8F0875D0C01082DE9F041DE
:10C5F0000446FFF73CFE0F2806464CD00F2120468C
:10C60000FFF7DDFD022107462046FFF7D8FD7B0737
:10C61000054603D5636801212046984738073AD577
:10C62000162E01D0112E05D1238F590433D56368FE
:10C6300002212CE0192E01D0122E2CD194F8573063
:10C640001BB916490320F4F7CFFA013BDBB284F89B
:10C65000573023B994F856102046FFF758FD636809
:10C66000CBB1228FD20416D505F0E000202809D0E6
:10C6700002D838B1BDE8F081602807D0A02803D0E7
:10C68000BDE8F081042102E0062100E007212046F8
:10C69000BDE8F0411847BDE8F08100BF5D0C01081E
:10C6A00013B50446416CC06BF4F724FE0121E06C25
:10C6B000F4F71AFFE06CF4F7E4FF0121206DF4F7C2
:10C6C00013FF206DF4F7D4FF0D4B009401220021DD
:10C6D000A06CF4F743FF2046FFF7AEFA1C2120467A
:10C6E000FFF76DFD032807D11C22002104F10C0087
:10C6F00002F05EFB002001E04FF0FF3002B010BD01
:10C7000027C300082DE9F34104460F4690461E4614
:10C71000FFF788FD01220DF103012046FFF78EFD92
:10C720009DF8035005F07F05023D37B3454505D917
:10C730002046FFF78FFD6FF0680521E0236A013383
:10C740002362636A2B442A46394620466362FFF718
:10C7500075FD022201A92046FFF770FD6EB101228E
:10C76000B1182046FFF76AFD2046FFF773FD072149
:10C770002046FFF724FD307002E02046FFF76AFDF7
:10C78000284602B0BDE8F0812DE9F04106460D468D
:10C790009046FFF7CEFA00273C46474512D06A681C
:10C7A000A31C13447F2B05F1080514D8F36955F831
:10C7B000081C2344F36130462346FFF7D5FA0137BE
:10C7C0000446EAE7338F5B0502D43046FFF7DCFA14
:10C7D0002046BDE8F0816FF08A00BDE8F0810000DE
:10C7E00008B5FFF744FD0838C0B211289ABF024BC4
:10C7F000185C022008BD00BF083A01082DE9F84383
:10C800000F46164698460546002800F0B780A1F16D
:10C810001103152B4DD8DFE803F01827344C4C4C8E
:10C820004C204C383C40444C484C4C4C4C4C4C0BF1
:10C83000B8F1010F03D857490320F4F7D5F90023C5
:10C840007370FFF74CFB307004E0B8F1010FF2D9C0
:10C85000662333800220BDE8F883B8F1000FEAD0E8
:10C86000FFF7BEFF307009E0038F13F4806F03D031
:10C8700001203070BDE8F883002333700120BDE84B
:10C88000F883038F13F4007FF1E7038FC3F3403382
:10C89000F3E7038FC3F38033EFE7038FC3F3C023C2
:10C8A000EBE7038FC3F30033E7E7038FC3F3002302
:10C8B000E3E74346324601F0CBF910F1860F044618
:10C8C00060D12846FFF7D3FC0F28814611D12846B6
:10C8D000FFF7D9FC162F1CD004D8012F35D0102F0C
:10C8E0000ED046E0272F28D02F2F36D0202F1DD056
:10C8F0003FE0162F0DD013D8012F26D0102F44D192
:10C90000B8F1010F97D92846FFF7FCFA02243080CE
:10C910002CE0B8F1000F8ED02846FFF70DFB23E086
:10C92000272F0AD02F2F18D0202F2ED1B8F1000F8B
:10C9300081D02846FFF71BFB16E0B8F1000F3FF44B
:10C940007AAF2846FFF74DFB0EE0B8F1000F3FF439
:10C9500072AF2846FFF730FA06E0B8F1000F3FF457
:10C960006AAF2846FFF753FB30700124B9F10F0F6F
:10C9700008D10F212846FFF7CAFB03E06FF0120031
:10C98000BDE8F8832046BDE8F8836FF08500BDE878
:10C99000F88300BF5D0C0108094B70B51C680646A2
:10C9A0000D4620460821F3F761FC21463046F4F796
:10C9B0009BF92846F3F75CFDBDE87040F4F77AB9BF
:10C9C000E00200202DE9F04104460E461546F3F73B
:10C9D00047FD27688046A7B13B68236096E80300BF
:10C9E0007B6883E803000A21A7F10800F3F73EFC07
:10C9F00017F8034C4046F3F73BFD2046F3F776FC6F
:10CA00001FE0A268E3689B1A2269934207DDDDB14B
:10CA10004146201DFFF7C0FFF3F722FD80460D4B76
:10CA2000E1681B8833804B1CE360236962690B401B
:10CA300096E8030002EBC30383E803004046F3F7E4
:10CA400017FD0120BDE8F081F3F712FD2846BDE88F
:10CA5000F08100BFDC020020F8B504460F46154601
:10CA6000F3F7FEFCA168E3688B4206461CD04B1C22
:10CA7000A3602369626965680B4002EBC30393E816
:10CA8000030087E80300E5B128460A2150F8083979
:10CA90006360F3F7EBFB15F8034C3046F3F7E8FC63
:10CAA0002046F3F723FC0FE03DB1084B1B6801461D
:10CAB000DF602046FFF770FF06E0F3F7D9FC284659
:10CAC000F8BD3046F3F7D4FC0120F8BDE0020020A9
:10CAD000BFF34F8F0549064BCA6802F4E062134367
:10CAE000CB60BFF34F8F00BFFDE700BF00ED00E05C
:10CAF0000400FA050121F5F769B810B5044640694C
:10CB000008B101F067FAE06908B101F063FA0020AA
:10CB10000022002360612061E061A0612080C4E9FF
:10CB2000022310BDF3F766BF2DE9F04F89B08A46A6
:10CB300015469B460446FFF7F5FFCDE90401EB00DF
:10CB40000393079355445346AB4205D013F8012B8A
:10CB5000002AF9D0002300E00123002702936FF0A0
:10CB600075030193B846B9463E46A268974270D213
:10CB700022687D0102EB050EDEE90201002908BFF3
:10CB8000B0F1FF3F23D0DDE90423994208BF904272
:10CB90001DD200220023CEE9022322682A44166116
:10CBA00022682A4496612268565322682A445069B2
:10CBB00020B101F00FFA22682A44566122682A4403
:10CBC000D06920B101F006FA22682A44D661039B9D
:10CBD00098453CD222682A445069002837D007AAD9
:10CBE000514601F02DFA38B923681D44129BCBF849
:10CBF00000500120186034E0029B13B102282DD1AF
:10CC0000F2E7012814D122681544296911F07F4FF9
:10CC10001BD0079AB2EB116F17D3B8F1000F01D0F8
:10CC2000904512D20023CBF80050904601930AE0C1
:10CC300002280AD1B8F1000F07D12268CDF804808C
:10CC40001544CBF800504FF00109039B07930137BF
:10CC50008BE7129B0198C3F8009002E00128F4D101
:10CC6000D1E709B0BDE8F08F38B505460C46FFF7AF
:10CC700059FF4FF47A736B43C01841F10001C4E9C6
:10CC8000000138BD2DE9F04788B0972990461BBFB9
:10CC9000109A0792424605AA8A461CBFCDF8148016
:10CCA0008DF81830ADF806100292DF0000F1120581
:10CCB00000F1200600F11C046FF0010935F9023F74
:10CCC000DBB1BAF1970F03D000976A46414607E0FF
:10CCD000D8F8183019684B78DB0000936A460231A7
:10CCE000306801F0ADF9023007D0B5F9002003A992
:10CCF00001A8F5F725F94FF00009A54206F1040651
:10CD0000DCD1484608B0BDE8F087000030B587B0F8
:10CD100006AA102302AD294642F8143D01F072F92B
:10CD2000A842014620D1019B102B08D128220F4890
:10CD3000FCF71EF801460E4802F042F914E0002408
:10CD4000019BA34204D3295D0A4802F039F902E0AD
:10CD5000094802F035F90134102CF1D107240748B5
:10CD600002F02EF9013CFAD107B030BDEC510020A1
:10CD70001A3A01081E200108001C0108011C0108C4
:10CD80002DE9F04F00F10C0787B0044638469A466B
:10CD90008B469046149EFFF7ADFE01230493B8F135
:10CDA000000F01D0119B2BB93846F4F73FFF6FF00D
:10CDB0000D006AE004AB0093524605AB41462046A5
:10CDC000FFF7B2FE012802D04FF000091CE01299D3
:10CDD0001198059C01F09CF8054610B96FF00B0402
:10CDE0004FE0E06901F0F6F8139BE561721CA36166
:10CDF00002D004F1080139E04FF0FF320023C4E90A
:10CE000002233DE009F10109A2689145E6D22268BA
:10CE10004FEA49152A44D2E9020150EA0103F1D14F
:10CE200051464046039201F073F8039A506122681C
:10CE30002A44516971B1109B1361226812991198AB
:10CE40002A44039201F064F8039A139BD06122688C
:10CE50002A44936122682A44D1690029D2D0A2F8D9
:10CE600000B0731C216805D0294408313046FFF713
:10CE7000FBFE05E00D444FF0FF320023C5E902231D
:10CE800000243846F4F7D2FE204607B0BDE8F08F04
:10CE90002DE9F04300F10C0585B0044628461F46F5
:10CEA000884691460E9EFFF725FE01230293B8F1B6
:10CEB000000F00D02FB92846F4F7B8FE6FF00D0030
:10CEC0002CE002AB00934A4603AB41462046FFF7F5
:10CED0002BFE012802D06FF00B041BE038460C99A2
:10CEE000039C01F015F807460028F4D0E06901F032
:10CEF00071F80D9BA361731CE76105D004F1080173
:10CF00003046FFF7B1FE04E04FF0FF320023C4E9E2
:10CF1000022300242846F4F789FE204605B0BDE828
:10CF2000F083F0B500F10C0485B0054620460E46AE
:10CF30001746FFF7DFFD0123029302AB00933A4649
:10CF400003AB31462846FFF7EFFD012802D10398D5
:10CF5000FFF7D3FD2046F4F769FE05B0F0BDF8B544
:10CF600000F10C06054630460F46FFF7C3FD0024CE
:10CF7000AB689C420AD22868630117B1C25EBA420C
:10CF800002D11844FFF7B9FD0134F1E73046BDE89E
:10CF9000F840F4F74BBE2DE9F04F00F10C0485B0DA
:10CFA000054620469B46894692460F9EFFF7A2FD06
:10CFB00001230293B9F1000F04D0BBF1000F01D09F
:10CFC0000E9B2BB92046F4F731FE6FF0150049E0B7
:10CFD00016B1BAF1000F05D12046F4F727FE6FF025
:10CFE0000D003FE002AF009703AB109A3146284690
:10CFF000FFF79AFD0128804615D9119B0093324610
:10D00000109B99212846FFF73DFE48B90123029362
:10D01000009703AB109A31462846FFF785FD8046FE
:10D02000B8F1010F0CD8039B5A465146D86900F05D
:10D03000E9FF58B92046F4F7F9FD6FF0680011E0F8
:10D040002046F4F7F3FD6FF075000BE0039BB3F996
:10D050000020A9F800200E9A9B6913602046F4F77F
:10D06000E5FD002005B0BDE8F08FF8B506460025C7
:10D0700046F80C5F04463046FFF73CFD04F112020F
:10D0800004F11C0304F1300122F8025F43F8045F4D
:10D090008B424FF00007F7D123792761022BA2685A
:10D0A0000BD1236852013946186801F081FE2368CC
:10D0B0009A685868D200394602E020685201394621
:10D0C00001F076FE01F01EF83046BDE8F840F4F7B6
:10D0D000ADBD00002DE9F04F044600F10C0585B010
:10D0E0002846FFF707FDFFF71DFD2379012B80463A
:10D0F00089466AD1674A684B684969488DE80C00DF
:10D10000684B01F05DFF4FF0000BA3689B456BD2AD
:10D1100021684FEA4B1A5144D1E90223134351D0FD
:10D120004869FFF7F3FD23685F485344196901F02C
:10D1300047FF23685344196911F07F4F04D0090E4B
:10D140005A4801F03DFF02E0594801F039FF2368D9
:10D150005344D869FFF7DAFD23685348534499696B
:10D1600001F02EFF23685344D3E90267002F08BF64
:10D17000B6F1FF3F1CD0B6EB080667EB0907002E9F
:10D1800077F1000301DA4B4913E0304639464A4A49
:10D19000002301F02FF8002303923046464A394617
:10D1A00001F028F8039A0146444801F009FF03E022
:10D1B0004349444801F004FF2368434833F90A1007
:10D1C00001F0FEFE0BF1010B9FE7022B0CD1324B5D
:10D1D00000933E4A3E4B3F493F4801F0F1FE4FF07D
:10D1E000000BA3689B4505D3284605B0BDE8F04F6A
:10D1F000F4F71CBD236819684FEA4B1A5144D1E972
:10D200000223134343D08B691868FFF77FFD23681F
:10D210001B6853445B691868FFF778FD23682F4843
:10D220001B685344196901F0CBFE23681B68534403
:10D23000D3E90267002F08BFB6F1FF3F1CD0B6EB61
:10D24000080667EB0907002E77F1000301DA194998
:10D2500013E030463946184A002300F0CBFF002384
:10D2600003923046144A394600F0C4FF039A01463F
:10D27000124801F0A5FE03E01149124801F0A0FE9A
:10D28000236811481B6833F90A1001F099FE0BF16D
:10D29000010BA6E75D3B0108183B0108733B010841
:10D2A000EF3A0108E63A0108203B01082A3B010851
:10D2B000333B01083B3B010840420F004A3B010859
:10D2C000543B0108433B01083F3A0108633B010816
:10D2D0005A3B0108703B01087F3B0108A13B010854
:10D2E000F8B5064684890F46154600206DB900231F
:10D2F000B289B168FBF7AEFC4FF6C57302199A42CA
:10D3000039680EDD013080B20BE0AE42EFD023462B
:10D31000AA89A968FBF79EFCEB686D681C44A4B25F
:10D32000E4E73A34204400232022083180B2FBF79E
:10D3300091FCC04380B2F8BD2DE9F3410C46804614
:10D3400003212046F7F711FB054618B92E490320A3
:10D35000F3F74AFC0221F7F708FB07460028F5D04F
:10D36000EB68032B4CD900F1080122462846AE6831
:10D37000FFF7B6FF002843D13378803B082B30D825
:10D38000DFE803F0052F2F2F2F0C151E2700AB8988
:10D39000B9683246404600F081F822E0EB6800931D
:10D3A000BA68334621464046F5F7C4FF19E0EB68FA
:10D3B0000093BA68334621464046F6F73DF810E040
:10D3C000EB680093BA68334621464046F5F71CFEE9
:10D3D00007E0EB680093BA68334621464046F5F70C
:10D3E000DFFE3178234640F201220320F6F790FF5A
:10D3F000014628B9204602B0BDE8F041F7F72ABD42
:10D4000002B0BDE8F08100BF5D0C010838B50D46E3
:10D41000144600211A460323F7F72AFC28B1836833
:10D4200000221D705C709A70DA7038BD10B5044629
:10D4300068B190F91030032B0CD142680831FFF726
:10D440004FFF50B1A36840BA5880002010BD6FF064
:10D450000D0010BD6FF04C0010BD6FF0010010BD4D
:10D460002DE9F041DDF81880154600220E461F46D2
:10D47000014608F108031046FFF7C8FF044650B103
:10D48000806876BA6DBA8680C58027B14246394633
:10D49000083001F0F3FB2046BDE8F081F7B5064601
:10D4A0000C46002A38D0072B36D99188D088083B03
:10D4B00040BA49BA009389B202F1080382B28120CE
:10D4C000FFF7CEFF074638B3237EFF2B04F1080297
:10D4D0000CBF002104F1180100F022F8054610B934
:10D4E0000146384613E000231A4619461846F7F756
:10D4F0008DF9836809495E8004464560034640F221
:10D5000002220220F6F704FF014628B9204603B0A4
:10D51000BDE8F040F7F79EBC03B0F0BD0000FFFF90
:10D52000F8B50F461646022328220021F7F7A0FB84
:10D53000054600B38468102204F10800394617B18B
:10D5400001F09CFB01E001F033FC04F11800102213
:10D55000314616B101F092FB04E001F029FC0123F1
:10D5600084F82730602200232270FF226370A370AA
:10D57000E370A271E3712846F8BD38B505460C4644
:10D5800019B301F17000F3F7ABFA2846F5F7A6FAE4
:10D5900038B1D0F810329C4203D100F5FC70F3F79B
:10D5A0009FFA04F11C00F3F79BFA04F13800F3F73B
:10D5B00097FA04F15400F3F793FA10220021204661
:10D5C00001F0F6FB00236383637638BD08B51022B3
:10D5D000034901F021FBB0FA80F0400908BD00BF0B
:10D5E000381101082DE9F74F904600901E469DF82E
:10D5F0003070894609B900205CE0082BFBD808464A
:10D60000FFF7E4FF0028F6D1824604464FF0980B5E
:10D610002A4B0BFB0AF29D18494628460192FBF75C
:10D6200040FB019A78B1B8F1000F42D0002E40D0F3
:10D63000224B02F1100041463246184401F01EFB15
:10D640002E766F7635E02846FFF7C0FF10B1002C2C
:10D6500008BF2C460AF1010ABAF1080FD8D1002CF4
:10D66000C9D0BDF80030638310224946204601F03E
:10D6700005FBB8F1000F07D036B13246414604F140
:10D68000100001F0FBFA2676677607F00707022FF5
:10D6900004BF032384F894304FF40973A4F8863050
:10D6A0004FF40473C4F8884063866463246520469D
:10D6B00000E0284603B0BDE8F08F00BF1452002000
:10D6C0002DE9F04107460E4611B90020BDE8F08172
:10D6D0000846FFF77BFF0028F7D10C4D0446A8460B
:10D6E000B5F91A3013B10FB1BB4209D13146284602
:10D6F000FBF7D7FA20B1982000FB0480BDE8F08149
:10D700000134082C05F19805EAD1DEE71452002017
:10D7100010B50446FFF7D4FF01462046BDE810408F
:10D72000FFF72BBF38B510B100F1980400E0074CAB
:10D73000074DAC4205D22046FFF748FF18B1983498
:10D74000F7E7002038BD204638BD00BF1452002046
:10D75000D456002008B5FFF7E5FF10B1437E1B0744
:10D76000F9D508BDF8B501460020FFF7A9FF04462A
:10D7700010B3437E13F0050F1ED0B0F91A00F5F771
:10D78000ADF90E4BD0F8D461B3F9007004F138054F
:10D790002846F3F7A5F940F21723A4F84E3004F118
:10D7A0004C023B4631462846FEF7F0F9637E23F0F3
:10D7B000070343F0070363762046F8BDB41D00203D
:10D7C00010B5144600B119B90B490320F3F70CFA50
:10D7D0002AB1537E03F00703013B012B01D800203F
:10D7E00010BD137E0B70127E04F1100101F046FA99
:10D7F000B4F91A0010BD00BF5D0C0108F0B503EBD1
:10D8000043048C424FF0000122D8017005465E1E91
:10D810000F464FF03A0E994219D014782409092C7A
:10D8200094BF3034573494462C709CF8004004F078
:10D830000F04092C94BF30345734B1426C700CBFC4
:10D840003C467446AC70013201310335E3E7F0BD6C
:10D850000846F0BD2DE9F04112B90020BDE8F08185
:10D860001378002BF9D01446264601347378002B28
:10D87000FAD107464FF0010C964217D33478A4F141
:10D8800030055FFA85F8B8F1090F06F1FF3E23D99C
:10D89000A4F14105052D02D8A4F137051CE0A4F13F
:10D8A0006105052D11D8A4F1570515E0BCF1000F55
:10D8B000D3D1013FB84205D23A780178397000F8E7
:10D8C000012BF6E71846BDE8F081BCF1000FC4D18A
:10D8D0004FF0010C7646CFE7724518D8A6F1020E3C
:10D8E00016F8016CA6F130045FFA84FCBCF1090F54
:10D8F0000ED9A6F14104052C02D8A6F1370407E0A1
:10D90000A6F16104052C02D8A6F1570400E000241A
:10D9100001338B42A1D845EA04143C704FF0000C4F
:10D920000137D7E713B5074A044692E803000022FF
:10D930008DE80300694604F11000FFF743F802B0D8
:10D9400010BD00BFAC3B010803460846002110B4DF
:10D9500083E80600072401221C621A7203F12804DE
:10D9600003F11002196159619961D9615C62DA6051
:10D97000194610BCF6F780BF70B51C46531E033322
:10D980000E4688B0114600F1100506D8294B0790C5
:10D9900003A80693F3F7B6F800E02AB1012201A923
:10D9A0002846FFF759F805E001A92846FFF754F883
:10D9B000002838D003A8F3F793F8BDF8063040F2FA
:10D9C000012293420CD048F2744293422ED1029A23
:10D9D000194B9A4214BF6FF003006FF0730027E0F9
:10D9E000029D02212846F6F7C0FF10B1C368272B1D
:10D9F00003D812490320F3F7F7F8816810220831A1
:10DA0000201D01F03BF9042323604FF0FF3128462D
:10DA1000F6F7ABFF08B9A08202E083685B88A382B7
:10DA20003560002004E06FF00A0001E06FF00300B1
:10DA300008B070BD25D90008630B8AF35D0C01089E
:10DA40002DE9F0478946064690469A46014600244D
:10DA500019B1CB6849681C44FAE7D9F80030D8F806
:10DA60000020934216D1042B14D108F1040209F1CD
:10DA700004013046FFF754FD0746C8B396F910502D
:10DA80000DB902253574BB6883F806A0B9F8146097
:10DA900056B906E03046F7F7DDF96FF06900BDE8EA
:10DAA000F087B8F8146086B1002319461A46184664
:10DAB000F6F7ACFE36B2014618B93846F7F7CAF9A0
:10DAC00016E08B685E804F600F460B493B4640F284
:10DAD00002222846F6F71CFC014630B93846F7F713
:10DAE000B9F96FF04C00BDE8F0872046BDE8F0873B
:10DAF0006FF00B00BDE8F0870000FFFF2DE9F04755
:10DB00000F46054610B90020BDE8F0870029FAD07D
:10DB10001022002101F04CF93B783A2B04D000246C
:10DB2000A1462646A04619E07A783A2A07F1010371
:10DB3000E9D11F46F3E751462B4801F051FB98B954
:10DB400051462A4801F04CFB80B1284BC01A40EAEC
:10DB50000616B6F5803FD6D24FF0010917F801AB93
:10DB6000BAF1000FE7D119E01F4BEFE7BAF13A0F16
:10DB7000C9D1B9F1000F05D1B8F1000FC3D105EB40
:10DB80000408EBE7A21C102ABDD8631CDBB2310AE3
:10DB900029558146EE54D4B20646DFE7B9F1000FAD
:10DBA00008D0A21C102AAED8631CDBB2310A29555A
:10DBB000EE54D4B2B8F1000F10D02C44C8EB0408D6
:10DBC00005F1100201230021434504F1FF3407DC75
:10DBD000207802F8010D01332170F5E7102C92D165
:10DBE0002846BDE8F08700BF98110108B43B010842
:10DBF0007FB50C46054600B119B90D490320F2F76F
:10DC0000F3FF0A4601AE232101F0D2F8304600F0BE
:10DC10004BF90023B3FBF4F204FB1232F15CA85C75
:10DC2000013341400C2BA954F4D104B070BD00BFA6
:10DC30005D0C010810B50446FFF7DAFF034B1A78B4
:10DC4000511C197023785340237010BD6A020020C4
:10DC5000062938B504460D46104636D006D80329A5
:10DC600022D029D8B1B3022911D09DE017294AD07A
:10DC700004D8082951D0152932D095E0252948D05B
:10DC8000292900F08980192940F08E8035E0012B88
:10DC900003D848490320F2F7A7FF0A4604F12C01F4
:10DCA00000F0ECFF284638BD072BF2D9082204F11A
:10DCB0002E0100F0E3FF7AE0022BEAD1228F520717
:10DCC00001D5082204E003806CE0022BE1D1628DD3
:10DCD000028067E0022BDCD194F8373013800AE031
:10DCE000012BD6D1238F13F0200F02D00123037014
:10DCF00058E000230370012038BD012BC9D1238FC8
:10DD000013F0020FF1E7012BC3D194F92820027020
:10DD100048E0022BBDD10322DAE7072BB9D9238FC4
:10DD20005B074CBF2B4602234FF000024CBF04F1AF
:10DD30002E0104F12C01042B4270027018D0082B24
:10DD400003D0022B33D1134619E00A7882F0020285
:10DD500002704A7842708A788270CA78C2700A79F2
:10DD600002714A7942718A798271CA79C27119E065
:10DD70000B7883F0020303704B7843700223FF2477
:10DD80000022C470FE24827004714271CA5C8271E8
:10DD900019444B78C3710AE0042B7FF47AAF04F185
:10DDA0000C011160184638BD6FF0850038BD0820A1
:10DDB00038BD00BF5D0C010870B515461C46192919
:10DDC0006AD8DFE801F00D691929393949696969AB
:10DDD00069696969696969696969694E69616958E7
:10DDE000022C03D02F490320F2F7FEFE1388FF2BED
:10DDF000F8D880F837304DE0022CF3D800F12C062B
:10DE000002220021304600F0D3FF22462946304648
:10DE100000F034FF022070BD082CE3D800F12E067C
:10DE200008220021304600F0C3FF22462946304632
:10DE300000F024FF082070BD022CD3D11388022BE0
:10DE400006D0082B2BD1038F43F00403038721E076
:10DE5000038F23F004030CE0022CC3D11388438505
:10DE600018E01278038F12B143F0200301E023F091
:10DE700020030387CEE71278038F12B143F0020329
:10DE8000F7E723F00203F4E7012CABD192F900305D
:10DE900080F82830204670BD6FF0850070BD6FF0AF
:10DEA000690070BD5D0C01080C22014900F0E6BE5E
:10DEB000107AFF1F10B586B006AC04F8093D0123A7
:10DEC00001930DF1170300932346F3F79DFA9DF894
:10DED000170006B010BDF0B585B01F4604AB002496
:10DEE00003F8012D012205460E4601920094F3F736
:10DEF0008BFA3B46224631462846FFF7DBFF05B04A
:10DF0000F0BD000001210148F3F760BED4560020A7
:10DF10002DE9F04780460E46FFF7F4FF294C002517
:10DF200014F8013C9E420AD132464146204600F098
:10DF300073FE20B9244B122404FB053428E001357C
:10DF4000282D04F11204EBD1204B1B68272B33D86A
:10DF50001D4B0025122202FB05F91B4F19F803A0E7
:10DF6000BAF1000F25D107EB090463789E4207D070
:10DF700010225146A01C00F01BFF07F809A0667094
:10DF8000122000FB057032464146023000F076FE5A
:10DF900023780F480133DBB2012B08BF0B4A2370F3
:10DFA00002BF136801331360F3F740FE2046BDE85B
:10DFB000F0870135282DCED10548F3F737FE002034
:10DFC000BDE8F087DE560020DC560020D856002041
:10DFD000D456002010B50446FFF794FF4CB12378C7
:10DFE0003BB1013BDBB223701BB9044A1368013B10
:10DFF00013600348BDE81040F3F718BED856002060
:10E00000D456002070B5154606460C46FFF77AFF39
:10E0100072782B6893420AD3B11C204600F02EFE82
:10E0200073782B600548F3F701FE204670BD2A6027
:10E030000248F3F7FBFD002070BD00BFD45600205E
:10E040002DE9F041174606468846FFF75BFF7278D8
:10E050003B68B3EBC20F05D1B01C002501244FF083
:10E06000FF3316E02648F3F7E1FD6FF00100BDE84D
:10E07000F081591C37D190F800E018F8051071456F
:10E0800037D02B46C4B1BEFA8EF46409A4B1013571
:10E0900001309542EDD33CB100233B601848F3F7C3
:10E0A000C5FD0220BDE8F0815D1C05D11448F3F7E1
:10E0B000BDFD2046BDE8F0811E4418F80310B2787B
:10E0C0004A40072142FA01F4E40748B202D4013978
:10E0D000F8D1084600EBC3033B600948F3F7A6FDFF
:10E0E0000120BDE8F081002CE6D00478B4FA84F475
:10E0F000CBE7002CCBD0B1FA81F46409C7E700BFAD
:10E10000D456002070B5FFF7FDFE0A4C002504F53B
:10E11000347604F8025C04F8015C204610220021E9
:10E12000123400F045FEB442F3D10348BDE870401C
:10E13000F3F77CBDDE560020D4560020D0400B1CE7
:10E14000D1409C46203AD340184352426346934004
:10E15000184370477BB972B90029BEBF00204FF049
:10E16000004106E008BF00281CBF6FF000414FF0DF
:10E17000FF3000F0C9B9ADF1080C6DE904CE0029FB
:10E1800009DB002B1ADB00F04DF8DDF804E0DDE9D7
:10E19000022304B07047404261EB4101002B1BDBBE
:10E1A00000F040F8DDF804E0DDE9022304B040426D
:10E1B00061EB4101524263EB43037047524263EB10
:10E1C000430300F02FF8DDF804E0DDE9022304B09A
:10E1D000404261EB41017047524263EB430300F060
:10E1E00021F8DDF804E0DDE9022304B0524263EBDC
:10E1F0004303704753B94AB9002908BF00281CBF20
:10E200004FF0FF314FF0FF3000F07EB9ADF1080C58
:10E210006DE904CE00F006F8DDF804E0DDE9022344
:10E2200004B070472DE9F0478C460E460446089D21
:10E23000002B50D18A4217466CD9B2FA82FEBEF149
:10E24000000F0BD0CEF1200420FA04F401FA0EF6F0
:10E2500044EA060C02FA0EF700FA0EF44FEA1749E8
:10E26000220CBCFBF9F01FFA87F809FB10C642EA42
:10E27000064600FB08F3B34209D9F61900F1FF3254
:10E2800080F02281B34240F21F8102383E44F61AE8
:10E29000A2B2B6FBF9F309FB136642EA064403FB9C
:10E2A00008F8A04509D9E41903F1FF3280F00A818A
:10E2B000A04540F20781023B3C44C8EB040443EA1A
:10E2C00000400021002D62D024FA0EF400232C60BF
:10E2D0006B60BDE8F0878B4207D9002D55D0002137
:10E2E00085E841000846BDE8F087B3FA83F10029CC
:10E2F00040F09080B34202D3824200F2F880841A48
:10E3000066EB03060120B446002D40D085E81010CE
:10E31000BDE8F08712B90127B7FBF2F7B7FA87FE1D
:10E32000BEF1000F35D1F31B4FEA17481FFA87FCE7
:10E330000121B3FBF8F0220C08FB103642EA064636
:10E340000CFB00F3B34207D9F61900F1FF3202D2F9
:10E35000B34200F2CE801046F61AA2B2B6FBF8F332
:10E3600008FB136642EA06440CFB03FCA44507D9EC
:10E37000E41903F1FF3202D2A44500F2B58013463E
:10E38000CCEB040443EA00409CE729462846BDE85C
:10E39000F087CEF1200106FA0EF307FA0EF720FA05
:10E3A00001F94FEA1748CE4049EA0309B6FBF8FAEB
:10E3B0004FEA194408FB1A661FFA87FC44EA064331
:10E3C0000AFB0CF29A4200FA0EF40AD9DB190AF1A0
:10E3D000FF3180F087809A4240F28480AAF1020ADD
:10E3E0003B449B1A1FFA89F9B3FBF8F108FB113380
:10E3F00049EA034301FB0CF69E4207D9DB1901F100
:10E40000FF326BD29E4269D902393B449B1B41EAE1
:10E410000A418EE7C1F1200E22FA0EF48B4023430D
:10E4200020FA0EF706FA01F44FEA134C26FA0EF61C
:10E430003C43B6FBFCF9270C0CFB19661FFA83F86A
:10E4400047EA064609FB08F7B74202FA01F200FA6A
:10E4500001FA08D9F61809F1FF3041D2B7423FD985
:10E46000A9F102091E44F61BA0B2B6FBFCF40CFB9A
:10E47000146640EA064704FB08F8B84507D9FF18B8
:10E4800004F1FF3028D2B84526D9023C1F4444EAA3
:10E490000940C8EB0707A0FB02894F4544464E469A
:10E4A00014D329D065B3BAEB040367EB060707FA68
:10E4B0000EFECB40CF404EEA030385E888000021E2
:10E4C000BDE8F0871346F8E61046E0E6B8EB020434
:10E4D00069EB03060138E5E70446D8E7114695E7FE
:10E4E0008146C0E78A467CE7023B3C4448E7084651
:10E4F0000AE702383E442FE7C245E7D33E46D1E75C
:10E500002946BDE8F08700BF704700BF0A220021FE
:10E5100001F008BA0A23002201F070B9014B186813
:10E52000704700BF6C0200208B891A072DE9F0416B
:10E530000D46804635D44A68002A6BDDEC6A002C13
:10E5400047D003F48052002192B2D8F80060C8F896
:10E550000010002A62D06A6D5F0705D569686B6B91
:10E56000521A0BB12B6CD21A0023296A4046A047DD
:10E57000441C39D0AB892A692A60DB044FF00002C1
:10E580006A6045D4696BC8F8006011B305F14403B3
:10E59000994202D0404600F059FC00206863BDE873
:10E5A000F0810E69AEB10C680E6098070CBF4B6924
:10E5B0000023A41B8B600AE023463246AF6A296A17
:10E5C0004046B8470028A4EB0004064404DD002CB4
:10E5D000F2DC0020BDE8F081AB8943F04003AB8161
:10E5E0004FF0FF30BDE8F081D8F800201D2AF3D8A5
:10E5F000184BD34003F0010383F00101002BEBD053
:10E60000AB892C696960D9042C60BBD5002AB9D1CB
:10E610006865B7E70A6C002A90DCDAE70123296A0B
:10E620004046A047431C024602D0AB89EC6A93E700
:10E63000D8F80030002BF8D01D2B01D0162B02D1BA
:10E64000C8F80060C5E7AB8943F04003AB81BDE883
:10E65000F08100BF010040200B6933B310B50446C0
:10E6600082B008B18369ABB1114B994219D0114BFB
:10E67000994218D0104B994208BFE168B1F90C30AB
:10E6800013B9002002B010BD204602B0BDE8104012
:10E69000FFF74ABF019100F019F90199044B994223
:10E6A000E5D16168EAE7A168E8E70020704700BFAC
:10E6B000083C0108E83B0108C83B010820B1054BB4
:10E6C00001461868FFF7C8BF034B0449186800F0FB
:10E6D00043B900BF6C020020283C010859E600083D
:10E6E00000207047014900F037B900BF59E6000823
:10E6F0000020704770B568234D1E03FB05F50E46DC
:10E7000005F1740100F0E8FB044640B100210C3033
:10E71000666005F168022160A06000F049FB2046B8
:10E7200070BD00BF1F4B70B51D68AB69064613B9BD
:10E73000284600F039F848356B68AC68013B05D5D0
:10E7400021E0013B5A1C04F168041CD0B4F90C20F0
:10E75000002AF6D1002501234FF6FF72E281A38142
:10E7600065662560A560656025616561A5612946CE
:10E77000082204F15C0000F01BFB6563A563A5643F
:10E78000E564204670BD2B680BB11D46D4E704211B
:10E790003046FFF7AFFF286008B10546CCE70C23F1
:10E7A000336070BD283C01083D4B3E491A682DE995
:10E7B000F04F90424FF000038364C364036508BFC9
:10E7C000012383B008BF836181620746FFF7AAFF78
:10E7D00078603846FFF7A6FFB8603846FFF7A2FF1B
:10E7E0007D68F86000240423AB812C606C60AC6011
:10E7F0006C66EC812C616C61AC61214605F15C00BA
:10E80000082200F0D5FABE68DFF89CB0DFF89CA0C3
:10E81000DFF89C90DFF89C80C5F824B00123092222
:10E82000C5F828A0C5F82C90C5F830802D62214687
:10E83000F381B28134607460B46074663461746171
:10E84000B46106F15C000822019300F0B1FAFD68A2
:10E85000366212200222C6F824B0C6F828A0C6F8F4
:10E860002C90C6F830802146A881EA812C606C602B
:10E87000AC606C662C616C61AC6105F15C000822D7
:10E8800000F096FA019B2D62C5F824B0C5F828A0C7
:10E89000C5F82C90C5F83080BB6103B0BDE8F08F9F
:10E8A000283C0108E5E6000855F100087DF1000864
:10E8B000B9F10008D9F10008024B0349186800F0CB
:10E8C0004BB800BF283C010859E60008836903B92A
:10E8D0006AE77047704700BF704700BF704700BFCE
:10E8E000704700BF024B0349186800F00FB800BF23
:10E8F0006C020020F1E60008024B0349186800F0A2
:10E9000005B800BF6C020020E1E600082DE9F041E7
:10E9100010F148071BD0884600267D68BC68013D81
:10E920000FD4A389012B05F1FF3506D9B4F90E30B8
:10E930000133204601D0C04706436B1C04F1680434
:10E94000EFD13F68002FE8D13046BDE8F0813E4668
:10E950003046BDE8F08100BF2DE9F84310F14807CB
:10E960001FD0884606464FF000097D68BC68013D0F
:10E9700011D4A389012B05F1FF3508D9B4F90E3064
:10E9800001332146304602D0C04749EA00096B1CDA
:10E9900004F16804EDD13F68002FE6D14846BDE898
:10E9A000F883B9464846BDE8F88300BF38B50A4B3E
:10E9B0001C68E16B054621B12846BDE8384000F0EF
:10E9C0000DB8242000F018F9E06301462846BDE8A0
:10E9D000384000F003B800BF6C0200200268634BAF
:10E9E00063482DE9F04383FB02431344D417C4EB7F
:10E9F000234400FB14200028C0F2AE8004F52F242D
:10EA000004F66C245B4E5C4D5C4ADFF884E1DFF871
:10EA100084C15B4F86FB0436E317C3EBE63605FB88
:10EA20000645AB08A2FB038205EBD222AEFB0383B3
:10EA3000A2EBD3122B09ACFB03C3A2EB1313DFF839
:10EA400058C1504AACFB038CA2FB038205EBDC3CB3
:10EA50009D1A9B0802EB5505AEFB03232D0A4A4A7B
:10EA6000ACEBD31340F26D1E0EFB1533DFF82CC157
:10EA700082FB002E03EB830202328644ACFB02C20F
:10EA80004FEAE07CCCEBEE2C4FF4616E0EFB1C00E9
:10EA90000334DFF80CE1C1F808C084FB078904EBFC
:10EAA000090C8EFB007EE717C7EBAC07C7EBC70767
:10EAB000D209092AA4EB07044FEAE078864402EB66
:10EAC000C20C8CBF6FF009070227C8EB6E1E0CEB5F
:10EAD0000C1CDFF8D0808C614FF4C87404FB065620
:10EAE0003A440CF1020CCEEB0E17A8FB0C4CA0EB39
:10EAF00087005C1C012A98BF0136B3F5997FA4EB0F
:10EB00009C0481E8014024D2A80717D01F48A0FB2D
:10EB10000570C0094FF4C87707FB1055B5FA85F5A5
:10EB20006D093B332B44A6F26C76002008624E61DF
:10EB3000CB610A61CC600846BDE8F0831348A0FBB6
:10EB400005704009642707FB10500028DED001251E
:10EB5000E7E7A3F59973E6E700F5A83004F52F245D
:10EB600000F5C07004F66B244CE700BF07452EC2C9
:10EB700080510100BD066B394FC5FDFF7F206B3909
:10EB80009324499261F31967C5B3A2911F85EB5194
:10EB9000D97CC65941D672001F2BD3E5D7802BD61E
:10EBA00089888888CDCCCCCC70B50F4E0F4D761BA4
:10EBB000B61018BF002405D0013455F8043B98471F
:10EBC000A642F9D10A4E0B4D761BF1F7DFFAB610CB
:10EBD00018BF002406D0013455F8043B9847A642DC
:10EBE000F9D170BD70BD00BF703D0108703D0108D6
:10EBF000703D0108703D0108024B0146186800F0A5
:10EC00006BB900BF6C020020024B0146186800F08F
:10EC10001DB900BF6C020020032A70B426D940EA57
:10EC200001039B0711D004780D78AC4222D1024435
:10EC3000431C05E013F8014B11F8015FAC4219D1F8
:10EC40009342F7D1002070BC70470C4603461E6803
:10EC50002568AE421846214603F1040304F104047A
:10EC6000E1D1043A032A18462146F0D8002ADAD125
:10EC70001046E8E7601B70BC704700BF844641EA5D
:10EC8000000313F003036DD1403A41D351F8043B24
:10EC900040F8043B51F8043B40F8043B51F8043B76
:10ECA00040F8043B51F8043B40F8043B51F8043B66
:10ECB00040F8043B51F8043B40F8043B51F8043B56
:10ECC00040F8043B51F8043B40F8043B51F8043B46
:10ECD00040F8043B51F8043B40F8043B51F8043B36
:10ECE00040F8043B51F8043B40F8043B51F8043B26
:10ECF00040F8043B51F8043B40F8043B51F8043B16
:10ED000040F8043B51F8043B40F8043B403ABDD284
:10ED1000303211D351F8043B40F8043B51F8043B26
:10ED200040F8043B51F8043B40F8043B51F8043BE5
:10ED300040F8043B103AEDD20C3205D351F8043BB5
:10ED400040F8043B043AF9D2043208D0D2071CBF81
:10ED500011F8013B00F8013B01D30B8803806046AA
:10ED6000704700BF082A13D38B078DD010F0030320
:10ED70008AD0C3F10403D21ADB071CBF11F8013B90
:10ED800000F8013B80D331F8023B20F8023B7BE7DF
:10ED9000043AD9D3013A11F8013B00F8013BF9D20A
:10EDA0000B7803704B7843708B78837060467047A4
:10EDB00070B4840746D0541E002A41D0CDB2034619
:10EDC00002E0621EE4B3144603F8015B9A07F8D12F
:10EDD000032C2ED9CDB245EA05250F2C45EA054571
:10EDE00019D903F110022646103E0F2E42F8105C8E
:10EDF00042F80C5C42F8085C42F8045C02F1100234
:10EE0000F2D8A4F1100222F00F0204F00F04103225
:10EE1000032C13440DD91E462246043A032A46F811
:10EE2000045BFAD8221F22F003020432134404F0D8
:10EE300003042CB1C9B21C4403F8011BA342FBD14B
:10EE400070BC704714460346C2E700BF30B481B1BE
:10EE500051F8043C0439002BB8BFC9181D4B1A687F
:10EE60002AB18A420AD908680C18A24225D04A6001
:10EE7000196030BC70478B4203D81A465368002B88
:10EE8000F9D1146815198D420CD007D808680C18F0
:10EE90009C4218D04B6030BC516070470C2303601B
:10EEA00030BC704709680C44111999421460E0D1D4
:10EEB0000ACB0C4453601460DBE7146852684A6064
:10EEC00020440860D4E71C685B684B6020440860FD
:10EED0005160CEE7AC59002070B5CD1C25F003057C
:10EEE00008350C2D38BF0C25002D06463BDBA9420A
:10EEF00039D827490A6852B113685B1B04D436E03D
:10EF000023685B1B1AD522465468002CF8D1496847
:10EF10001F4C002936D029463046F1F73BF9431CF7
:10EF200021D0C41C24F00304A04205D0211A30468D
:10EF3000F1F730F9013016D0256004E00B2B0DD924
:10EF400023601C44256004F10B0020F00700231D02
:10EF5000C31A02D05A42E25070BD70BD94420ED026
:10EF600063685360EFE70C233360002070BD0B2B08
:10EF700003D8536814460B60E5E71446E0E71346F0
:10EF80001446F8E73046F1F705F96060C3E700BFC3
:10EF9000AC5900200EB410B5044683B018B1836993
:10EFA0000BB9FFF793FC06A803460190059AA168E8
:10EFB000204600F0F3FE03B0BDE8104003B07047F8
:10EFC0000FB410B50A4B1C6882B024B1A36913B901
:10EFD0002046FFF77BFC05A803460190049AA16830
:10EFE000204600F0DBFE02B0BDE8104004B07047E0
:10EFF0006C0200202DE9F0410E46804600283ED0EC
:10F000008369002B39D084682F4B9C4243D02F4B0F
:10F010009C4256D02E4B9C4208BFD8F80C40A38986
:10F020001B073DD52369002B3AD0013EA36816F893
:10F03000015F013BA360B5B1002B04DB23685A1CC0
:10F0400022601D70F2E7A769BB422246294640466E
:10F0500001DB0A2DF2D100F017FD0130E6D14FF0AF
:10F06000FF30BDE8F081002B21DB23680A22591C08
:10F0700021601A701046BDE8F081FFF727FCD8F830
:10F080001830D8F80840002BBED14046FFF71EFCD0
:10F090000D4B9C42BBD1D8F80440A3891B07C1D4B7
:10F0A0002146404600F052FD0028BED0D7E7224658
:10F0B00040460A2100F0E8FC0130D0D00A20BDE82B
:10F0C000F081D8F80840AAE7083C0108E83B0108AD
:10F0D000C83B0108024B01461868FFF78BBF00BF11
:10F0E0006C02002038B50C46054608B18369B3B1FF
:10F0F000114B9C4218D0114B9C4217D0104B9C4294
:10F1000008BFEC682846214601F07EF980B994E8F2
:10F110000C00013B511C84E80A00107838BDFFF751
:10F12000D5FB054B9C42E6D16C68EBE7AC68E9E7A0
:10F130004FF0FF3038BD00BF083C0108E83B010834
:10F14000C83B0108024B01461868FFF7CBBF00BF60
:10F150006C02002010B50C46B1F90E10F1F738F82A
:10F16000002803DB636D0344636510BDA38923F4AA
:10F170008053A38110BD00BF002070472DE9F041EE
:10F180001646B1F90C201F46D3050C46054607D597
:10F1900000220223B1F90E10F1F727F8B4F90C2080
:10F1A000B4F90E1022F48052A2813B463246284622
:10F1B000BDE8F041F1F710B810B50C46B1F90E10EA
:10F1C000F1F713F8A389421C0EBF23F4805343F4D4
:10F1D00080536065A38110BDB1F90E10F1F700B83E
:10F1E00070B411F0FF0434D085070FD00378002BE2
:10F1F0005AD09C422BD0431C05E013F8012B002A67
:10F200004FD0944223D09A071846F6D10E0206F446
:10F210007F462643036846EA064601E050F8043F6D
:10F2200086EA0305A5F10132A3F1013122EA0502C4
:10F2300021EA0303134313F0803FEFD0037823B98F
:10F2400032E010F8013F002B2ED09C42F9D170BC67
:10F25000704784070BD00378002BF8D0431C03E0E1
:10F2600002780133002AF2D099071846F8D10268D3
:10F27000A2F1013323EA020313F0803F08D150F8D2
:10F28000042FA2F1013323EA020313F0803FF6D0EA
:10F290000378002BDBD010F8013F002BFBD170BCB2
:10F2A0007047104670BC7047184670BC704700BF6E
:10F2B000000000000000000000000000000000004E
:10F2C000A2EB0300704700BF02780B78012A28BF29
:10F2D0009A42F5D16DE9044540EA0104CDE902679F
:10F2E0006FF0000C4FEA447212B380EA010414F08C
:10F2F000070F6AD100F0070420F0070004F00305AF
:10F3000021F007014FEAC505F0E8042314F0040FCB
:10F31000F1E804670CFA05F462EA040266EA0406FE
:10F320000AD063EA0403624667EA0407664603E01C
:10F33000F0E80423F1E8046782FA4CF582EA060457
:10F34000A4FA8CF46CBB83FA4CF583EA0705A5FAA2
:10F350008CF595B950E9022351E9026782FA4CF520
:10F3600082EA0604A4FA8CF483FA4CF583EA0705D2
:10F37000A5FA8CF52543DBD09CB92DBAB5FA85F4F6
:10F3800024F0070427FA04F1DDE9026723FA04F305
:10F3900003F0FF0001F0FF01FDE80445A0EB0100D0
:10F3A000704724BAB4FA84F424F0070426FA04F16E
:10F3B000DDE9026722FA04F202F0FF0001F0FF012A
:10F3C000FDE80445A0EB0100704714F0030F3CD1A9
:10F3D00010F0030428D150F8082B51F8083B82FAAA
:10F3E0004CF582EA0305A5FA8CF55DB950F8042CBA
:10F3F00051F8043C82FA4CF582EA0305A5FA8CF533
:10F40000002DE8D02DBAB5FA85F424F0070423FACC
:10F4100004F122FA04F202F0FF0001F0FF01FDE81E
:10F420000445A0EB010070474FEAC40420F003003C
:10F4300050F8082B21F0030151F8083B0CFA04F4B2
:10F4400062EA040263EA0403C9E710F003041AD075
:10F45000A1EB040120F00300E40750F8042B06D0D0
:10F460000FD28B785FFAA2F4E41A06D12BB1CB78D5
:10F470005FFAB2F4E41A00D11BB920465DF8104BD4
:10F48000704701F1040150F8042BCC0721F003016F
:10F4900051F8043B48D824D222F07F4482FA4CF53C
:10F4A00094EA1325A5FA8CF50AD165B951F8043B05
:10F4B00084EA0204B4EB036F0ED150F8042BEBE79F
:10F4C0004FEA132355E035F07F454DD10878FDE82C
:10F4D0000445C0F1000070474FEA126203F0FF03D9
:10F4E00047E002EA1C4482FA4CF594EA1345A5FA77
:10F4F0008CF50AD165B951F8043B84EA0204B4EBF7
:10F50000034F0CD150F8042BEBE74FEA134330E0E4
:10F5100015EA1C4528D10B884FEA124229E04FEA30
:10F52000124203EA1C4324E002F0FF0482FA4CF585
:10F5300094EA1365A5FA8CF50AD165B951F8043B34
:10F5400084EA0204B4EB032F09D150F8042BEBE753
:10F550004FEA13630DE015F0FF0F05D10B684FEA7A
:10F56000122223F07F4304E04FF00000FDE8044541
:10F57000704712BA1BBA82FA4CF482EA0304A4FA66
:10F580008CF5B5FA85F402FA04F203FA04F34FEAB3
:10F590001260FDE80445A0EB1360704780EA0102A9
:10F5A000844612F0030F4FD111F0030F32D14DF802
:10F5B000044D11F0040F51F8043B0BD0A3F10132BC
:10F5C0009A4312F0803F04BF4CF8043B51F8043BCF
:10F5D00016D100BF51F8044BA3F101329A4312F047
:10F5E000803FA4F101320BD14CF8043BA24312F04E
:10F5F000803F04BF51F8043B4CF8044BEAD023464B
:10F600000CF8013B13F0FF0F4FEA3323F8D15DF8FC
:10F61000044B704711F0010F06D011F8012B0CF8C4
:10F62000012B002A08BF704711F0020FBFD031F83C
:10F63000022B12F0FF0F16BF2CF8022B8CF80020C3
:10F6400012F47F4FB3D1704711F8012B0CF8012B46
:10F65000002AF9D1704700BF000000000000000040
:10F66000000000000000000000000000000000009A
:10F67000000000000000000000000000000000008A
:10F6800090F800F06DE9024520F007016FF0000CE2
:10F6900010F0070491F820F040F049804FF000048A
:10F6A0006FF00700D1E9002391F840F000F1080065
:10F6B00082FA4CF2A4FA8CF283FA4CF3A2FA8CF39D
:10F6C0004BBBD1E9022382FA4CF200F10800A4FA04
:10F6D0008CF283FA4CF3A2FA8CF3E3B9D1E9042358
:10F6E00082FA4CF200F10800A4FA8CF283FA4CF38F
:10F6F000A2FA8CF37BB9D1E9062301F1200182FA49
:10F700004CF200F10800A4FA8CF283FA4CF3A2FA4E
:10F710008CF3002BC6D0002A04BF04301A4612BA5C
:10F72000B2FA82F2FDE8024500EBD2007047D1E95F
:10F73000002304F00305C4F100004FEAC50514F0EE
:10F74000040F91F840F00CFA05F562EA05021CBFBF
:10F7500063EA050362464FF00004A9E7002A41D09E
:10F7600040EA010313F00303F0B425D1032A23D99F
:10F7700004680D68AC421FD1043A35D0A4F10135BC
:10F7800025EA040414F0803F31D1071D0D1D0DE062
:10F7900057F8043B0E68A3F10134B34224EA030492
:10F7A0000AD1043A20D014F0803F23D1032A2946FD
:10F7B000384605F10405EBD803780C789C4202F139
:10F7C000FF320CD182B114B916E06AB17BB110F8E6
:10F7D000013F11F8014FA34202F1FF32F5D0181B8F
:10F7E000F0BC7047104670471046F0BC7047184692
:10F7F000F0BC70470020F3E72046F1E72DE9F04F19
:10F80000474C83460E46D4F800E000E026463446D6
:10F8100014F8015B0EEB0500407800F0080000F0E2
:10F82000FF080028F2D12D2D5CD02B2D04BF757858
:10F83000B41C002B3ED0102B60D09A46B8F1000FBC
:10F840000CBF6FF000404FF000400027B0FBFAF90A
:10F85000BC460AFB19000CE0303DAB4219DD7E1CB2
:10F8600005D0CC4523D820D00AFB0C5C012714F826
:10F87000015B0EEB0506767816F0040FECD116F05E
:10F88000030606D0012E14BF57263726AD1BAB4208
:10F89000E5DC7B1C16D0B8F1000F10D16046002AC1
:10F8A00039D0DFB91160BDE8F08F8542DCDD4FF063
:10F8B000FF37DCE7302D1AD00A239A46BEE7CCF199
:10F8C000000CEBE7B8F1000F4FF022030CBF6FF014
:10F8D00000404FF00040CBF80030F2B1611E1160E3
:10F8E000BDE8F08FB41C75784FF00108A1E72378CC
:10F8F00003F0DF03582B08D008239EE7302D9CD15E
:10F90000207800F0DF00582897D14FF0100A657872
:10F910005346023492E7BDE8F08FBDE8F08F00BF98
:10F92000D002002010B4044C13460A460146206859
:10F9300010BCFFF763BF00BF6C0200202DE9F04F41
:10F94000494C82460E46D4F800E000E02646344694
:10F9500014F8015B0EEB0500407800F0080000F0A1
:10F96000FF0C0028F2D12D2D54D02B2D04BF75781B
:10F97000B41C5BB1102B5ED04FF0FF38B8FBF3F82E
:10F9800003FB08FB6FEA0B0B994607E0302D46D0CE
:10F990000A23DFF8D88099464FF0050B0027384638
:10F9A0000CE0303DAB4219DD7E1C05D0404522D82D
:10F9B0001FD009FB0050012714F8015B0EEB050670
:10F9C000767816F0040FECD116F0030606D0012E5F
:10F9D00014BF57263726AD1BAB42E5DC002F0FDBEB
:10F9E000BCF1000F00D0404242B17FB91160BDE8C8
:10F9F000F08F5D45DDDD4FF0FF37DDE7BDE8F08FCF
:10FA00002223CAF800304FF0FF305AB3611E116054
:10FA1000BDE8F08FB41C75784FF0010CA9E723788E
:10FA200003F0DF03582B0DD0082399464FF0070B46
:10FA30006FF06048B2E7302D0ED1207800F0DF0083
:10FA4000582809D14FF0100965784B464FF00F0B3D
:10FA500002346FF07048A1E74FF00F0B6FF0704861
:10FA600099469BE7BDE8F08FD0020020999999193B
:10FA700010B4044C13460A460146206810BCFFF738
:10FA80005DBF00BF6C020020F8B50E461446054667
:10FA900010B18369002B41D0254B9C4243D0254BAC
:10FAA0009C4242D0244B9C4208BFEC68A389A269C7
:10FAB000A2601A0721D52369FBB122686169D31AB4
:10FAC0008B42F7B221DA0133A168501C0139A160E1
:10FAD0002060167062699A4206D0A389DB0701D5BF
:10FAE0000A2F01D03846F8BD21462846FEF7B4FD5E
:10FAF0000028F7D04FF0FF37F4E72146284600F002
:10FB000025F80028F6D12369D7E721462846FEF7D5
:10FB1000A3FD0028EED122680123D5E7FEF7D6FE2B
:10FB2000034B9C42BBD16C68C0E7AC68BEE700BF2A
:10FB3000083C0108E83B0108C83B0108024B0A46A3
:10FB400001461868FFF7A0BF6C020020384B70B563
:10FB50001D6806460C4615B1AB69002B42D0354BEB
:10FB60009C4245D0344B9C4258D0344B9C4208BFF9
:10FB7000EC68B4F90C2093B219070CD52069A8B130
:10FB800013F001021ED0636900225B42A361A260F0
:10FB9000F0B1002070BDDD0642D558072AD4206997
:10FBA00042F00803A3819BB20028E9D103F420723C
:10FBB000B2F5007FE4D03046214600F06FF8A3890B
:10FBC0002069DDE7990758BF6269A2600028E0D18B
:10FBD000B4F90C301A06DDD543F04003A3814FF091
:10FBE000FF3070BD2846FEF771FE124B9C42B9D122
:10FBF0006C68BEE7616B51B104F14403994204D0D3
:10FC00003046FFF723F9B4F90C2000236363002387
:10FC10002069636022F024022060C1E7AC68A8E795
:10FC200042F04002092333604FF0FF30A28170BDE3
:10FC30006C020020083C0108E83B0108C83B0108B1
:10FC400070B50C46B1F90E10002990B015461E464D
:10FC500013DB01AAF0F7CEFA00280EDB029A02F4B9
:10FC60007042A2F50052B2FA82F252094FF4806358
:10FC7000002032602B6010B070BDA38900221B06EB
:10FC8000326004D5402300202B6010B070BD4FF4CB
:10FC9000806300202B6010B070BD00BF8A8992077E
:10FCA0000B4606D501F1470201211A601A6159611C
:10FCB0007047F0B583B001AB6A460C460546FFF7C6
:10FCC000BFFF009906462846FFF706F9B4F90C3045
:10FCD000D0B1019A124F0099AF6243F08003A38123
:10FCE0002060206161611AB93343A38103B0F0BD84
:10FCF0002846B4F90E10F0F782FAB4F90C30002857
:10FD0000F2D043F00103EFE79A05EFD404F1470284
:10FD100043F002030121A381226022616161E5E7D2
:10FD2000E5E600089368013B002B10B4936007DB05
:10FD3000CCB21368581C10601970204610BC704774
:10FD40009469A34202DBCCB20A2CF2D110BCFFF7BB
:10FD50009BBE00BF93B1F8B514460F460646D518B2
:10FD600001E0AC4208D03A4614F8011B3046FFF7D8
:10FD7000D9FF431CF5D1F8BD0020F8BD0020704725
:10FD8000936810B5144613B95360184610BD00F0BF
:10FD9000D1FB0023A360636010BD00BF2DE9F04FCD
:10FDA0009DB0884614460393814618B18369002BA1
:10FDB00000F00B818B4B984500F00D818A4B9845E4
:10FDC00000F00C81894B984508BFD9F80C80B8F831
:10FDD0000C301D0740F1EF80D8F81030002B00F0F8
:10FDE000EA8030238DF82A302378814DDFF804A291
:10FDF0000021202209918DF82920002B00F0858018
:10FE0000252B264603D117E0252B00F0868016F817
:10FE1000013F002BF8D1B6EB040B76D022465B46AF
:10FE200041464846FFF796FF01306ED0099B327875
:10FE30005B440993002A68D000234FF0FF31721C05
:10FE40000493079306938DF853301A930591012676
:10FE500004E0049906FA03F30B4304931446644840
:10FE60002178052200F0ECFC621C431B0028F0D135
:10FE7000049BD80644BF20228DF85320190721780F
:10FE800044BF2B228DF853202A2968D0A1F13002DB
:10FE9000092A0BD8079B14F8011F03EB830302EB1D
:10FEA0004303A1F13002092AF5D907932E293FD047
:10FEB0000322504800F0C4FC48B10499CAEB00008A
:10FEC000402202FA00F041EA000301340493217851
:10FED00049488DF828100622013400F0B1FC0028B2
:10FEE0005FD0464BEBB103AB00934246444B04A9B1
:10FEF0004846AFF3008007467A1C06D0099B3B4476
:10FF000009932378002B7FF47BAFB8F80C305B06A5
:10FF100058D409981DB0BDE8F08FB6EB040B8BD018
:10FF20007CE7039B073323F0070308330393E5E7DC
:10FF300061782A291DD0A1F130020023092A04F199
:10FF400001040593B4D814F8011F03EB830302EBFB
:10FF50004303A1F13002092AF5D90593A8E7039AD2
:10FF6000116804320029039215DB0791617801348E
:10FF70009CE7039B1A680592002A03F1040303938C
:10FF8000B8BF4FF0FF3204F10203AEBFA178A178F1
:10FF900005921C468CE7494243F002030791049303
:10FFA000E4E703AB00934246154B04A9484600F032
:10FFB000CDF80746A0E741464846FFF7C7FD0028B1
:10FFC0003FF40FAF4FF0FF30A4E7FEF77FFC054B87
:10FFD00098457FF4F3AED9F80480F8E6D9F80880A4
:10FFE000F5E600BF083C0108E83B0108C83B0108F2
:10FFF000343D01083C3D0108403D0108000000007F
:020000040801F1
:1000000055FD000810B4044C13460A46014620680A
:1000100010BCFFF7C3BE00BF6C0200202DE9F04703
:100020000C4691460969A268DDF820808A42B8BF73
:100030000A46C9F8002094F8431006461F4611B13D
:100040000132C9F80020236899065DD5D9F800204F
:100050000232C9F80020236813F0060F19461DD19B
:10006000E1688A1A002AD8BF194617DD04F1190A77
:10007000002505E0E368D9F800209B1AAB420CDDAF
:100080000123524639463046C047013005F101058B
:10009000F0D14FF0FF30BDE8F087216894F843308D
:1000A000003318BF01238A060AD5E1185A1C3020F4
:1000B00081F84300224494F8451082F8431002333B
:1000C00004F1430239463046C0470130E1D023688D
:1000D00003F00603042B29D0A36822699342C8BF0A
:1000E0004FF000092FDD9B1A99441A34002501E0D6
:1000F0004D4528D00123224639463046C0470130BD
:1001000005F10105F4D1C4E713F0060F08D1E16849
:10011000D9F800208A1A002AD8BF1946A6DCBDE704
:1001200094F84330003318BF0123C9E7D9F8000021
:10013000E168A3682269091A934221EAE179D2DCD5
:10014000B9F1000FD1D10020BDE8F0872DE9F043CF
:100150000C46097E85B06E29064617460C989846CF
:1001600004F1430C5AD01AD8632900F0128100F22E
:10017000D68000295CD0582940F0F58084F84510DD
:1001800022680368DFF864E2150603F104011ED457
:10019000550653BF1B6801601B88016019E0732975
:1001A00000F0CF807ED86F2900F0E480702940F005
:1001B000DA80226842F020022260782384F84530F9
:1001C0000368DFF82CE2150603F10401E0D51B6893
:1001D0000160D00744BF42F020022260002B40F0B3
:1001E0009080226822F0200222601021002284F8F0
:1001F00043206068A0600028C0F28880226822F056
:1002000004022260002B62D1002840F08180654604
:1002100008296AD0C5EB0C0323610CE023681A0699
:1002200040F1D58003686269191D01601B681A607E
:10023000002365462361CDF800803B4603AA214692
:100240003046FFF7EBFE013021D02A4623693946BC
:100250003046C04701301AD02368039813F0020FCC
:10026000E36819D01A1A002A16DD04F119090025CD
:1002700004E0E36803981A1AAA420DDD01234A46F6
:1002800039463046C047013005F10105F1D14FF044
:10029000FF3005B0BDE8F0839842B8BF184605B0FE
:1002A000BDE8F083752965D078295CD1226884E7A0
:1002B0006168A1602D200029C3F1000384F8430088
:1002C00021DB22F00402DFF824E122600A216546E6
:1002D000B3FBF1F201FB123013461EF8002005F8C3
:1002E000012D002BF4D1082994D12368D90791D589
:1002F000626823699A428DDC302305F8013C013D98
:1003000088E7102172E7DFF8E4E00A21002BDED154
:100310009EF8003084F8423004F1420578E7642901
:1003200001D069291FD122680368150603F1040171
:100330003AD51B680160002BBADBDFF8B0E00A2178
:1003400057E703686268191D01601D68002128468F
:1003500000F076FA002846D0401B60602061002340
:1003600084F8433067E7012384F84210236104F1E5
:100370004205F4E723681A061ED503681A1D1B6898
:100380000260227EDFF864E06F2A14BF0A21082190
:100390002CE703681A68191D0123016004F1420566
:1003A00084F842202361DAE7550653BF1B680160D9
:1003B000B3F900300160BEE713F0400F036803F1AA
:1003C000040215BF02601B681B880260D9E713F0A6
:1003D000400F0368626903F1040101601B6814BFE8
:1003E0001A801A6024E76068B8E700BF483D01083A
:1003F0005C3D0108838903F00903092B01D000202B
:100400007047FEF75BB900BFF8B50C46054610B162
:100410008369002B45D0424B9C4247D0414B9C42C4
:100420006FD0414B9C4208BFEC68B4F90C2093B2EA
:1004300000219F06616031D45E0722D5616B61B1F6
:1004400004F14403994202D02846FEF7FFFC236CD6
:10045000636000206063002B43D12369002B52D0DE
:10046000B4F90C70BEB2B30722D1226922602846CB
:100470006369656A216AA8470028606009DD002079
:10048000F8BDD80644D519072ED442F00402A28143
:10049000E3E7A3891DD143F02003A3814FF0FF3090
:1004A000F8BDFEF713FA1E4B9C42B7D16C68BCE74F
:1004B0001E4B1F4918680123A38106F00906FEF7A9
:1004C00025FA092EA781D0D121462846FEF72CF81F
:1004D000CBE7002243F04003A38162604FF0FF307E
:1004E000F8BDE36B2360F8BD21462846FEF7B4F85B
:1004F0000028D3D1B4F90C20A060A06122F008023A
:10050000C3E7AC6891E721462846FFF7C7FBA7E79A
:1005100042F0400209232B604FF0FF30A281F8BD6A
:10052000083C0108E83B0108C83B0108283C0108D9
:10053000F50301089368002B76D02DE9F04F8B89E5
:1005400085B00C4619070190164629D522693AB3A1
:1005500003F002081FFA88F0356800282FD04FF00A
:100560000009B44FC846B246B84543464A4628BF7C
:100570003B460198B8F1000F50D0216AA66AB047F7
:10058000002871DDDAF808301B1A8144C0EB080836
:10059000CAF80830002BE7D1002005B0BDE8F08F85
:1005A00021460198FFF7D2FA002840F03A81A3894A
:1005B000356803F002081FFA88F00028CFD113F045
:1005C00001095BD14F4602961FB39A05D4F8088003
:1005D0002CD54745C246C0F0A48013F4906F40F07C
:1005E000B18020685246494600F07AF9A068236835
:1005F000C8EB00005344A06023603846029A936819
:100600001B1A81443F1A9360002BC5D0A389002F89
:10061000DBD1D5F800906F680835D5E7D5F80090A4
:10062000D5F8048008359FE70020704720682369CB
:10063000984203D861698F4280F0B780B84528BFDF
:10064000B8464246494600F04BF9A3682268C8EB19
:1006500003034244A3602260002B49D12146019844
:10066000FDF7FAFF002843D0B4F90C3043F0400303
:100670004FF0FF30A38105B0BDE8F08F80460290B7
:1006800082468146B9F1000F2AD0029B002B4CD044
:10069000206823696269C845C34628BFCB46984293
:1006A0005F4604D9A36813449B4500F390809345AB
:1006B00020DB1346A76A216A01985246B847071EF5
:1006C000D2DDB8EB070823D0B368DB1BBA44C7EB15
:1006D0000909B360002B3FF45FAFB9F1000FD4D12B
:1006E0000023D5F800A0D5F8049002930835C9E797
:1006F000404683E75A46514600F0F2F8A268236864
:10070000CBEB02025B44B8EB0708A2602360DBD1AD
:1007100021460198FDF7A0FF0028A5D1CDF808805B
:10072000D2E72068B846BA465CE74A460A215046F6
:1007300000F086F800286FD001300123CAEB0008D2
:100740000293A5E762692068216902EB4208C1EBC8
:10075000000A08EBD8780AF101004FEA680838442B
:100760004045424684BF804642465B0542D511461D
:100770000198FEF7B1FB8346002855D05246216907
:10078000FEF77CFAA38923F4906343F08003A381EE
:10079000CAEB08030BEB0A00C4F81480C4F810B0CD
:1007A0002060A360B846BA461CE76FF00043BB4226
:1007B00028BF3B464A4693FBF1F30198A66A01FB2A
:1007C00003F3216AB04700283FF718AF4CE71A46F9
:1007D0005146039300F084F82268039B01981A4461
:1007E00022602146FDF738FF039B00287FF43CAFD1
:1007F0001F4666E7019800F0D7F883460028C7D166
:10080000019D21692846FEF721FBB4F90C300C222A
:1008100023F080032A6029E7012309F101080293EC
:1008200036E74FF0FF30B8E6019A0C231360B4F9B5
:100830000C301BE700FCFF7F000000000000000000
:1008400001F0FF01102A2BDB10F0070F08D010F881
:10085000013B013A8B422DD010F0070F42B3F6D185
:10086000F0B441EA012141EA014122F007047FF09E
:1008700000070023F0E80256083C85EA010586EAF5
:10088000010685FA47F5A3FA87F586FA47F6A5FA31
:1008900087F68EB9EED1F0BC01F0FF0102F007023D
:1008A00032B110F8013B013A83EA010313B1F8D1E8
:1008B0000020704701387047002D06BF35460338C9
:1008C000073815F0010F07D1013015F4807F02BF02
:1008D000013015F4C03F0130F0BC0138704700BF53
:1008E0008842F0B50DD98B1898420AD28118002A97
:1008F00051D09A1A13F8014D01F8014D9342F9D1E4
:10090000F0BD0F2A48D941EA00039B0746D100F108
:10091000100401F11003154653F8106C44F8106CE4
:1009200053F80C6C44F80C6C53F8086C44F8086CE1
:10093000103D53F8046C44F8046C0F2D03F11003C0
:1009400004F11004E8D8A2F1100323F00F0302F021
:100950000F0E1033BEF1030F1944034421D91E1F9B
:100960000D467446043C55F8047B46F8047F032C7E
:10097000F8D8AEF1040424F00304043423442144E1
:1009800002F0030262B1013B0A4411F8014B03F883
:10099000014F8A42F9D1F0BD0346F3E70346F2E77F
:1009A000F0BD7246EEE700BFF9B1F8B50646154650
:1009B000B2B10C4600F01CF8854201D82046F8BDC3
:1009C00029463046FEF788FA074668B12A4621468E
:1009D000FEF754F930462146FEF738FA3846F8BD9E
:1009E000FEF734FA2846F8BDF8BD1146FEF774BA92
:1009F00051F8040C0028BEBF091851F8043CC01877
:100A0000043870474E4D492048414E444C455200F1
:100A10004D454D204D414E4147452048414E444CA7
:100A2000455200425553204641554C542048414EB2
:100A3000444C4552005553414745204641554C547E
:100A40002048414E444C4552004445425547204DB4
:100A50004F4E2048414E444C45520044554D4D594F
:100A60002048414E444C4552000A49535220737469
:100A700061636B206F766572666C6F776564005397
:100A80007461636B20706F696E74657220636F723E
:100A90007275707465642C20726573657420746F50
:100AA00020746F70206F6620737461636B000A435B
:100AB0006F6E74657874206265666F726520686118
:100AC00072646661756C743A0020202072303A209E
:100AD00030782530386C780A20202072313A203066
:100AE000782530386C780A20202072323A2030780D
:100AF0002530386C780A20202072333A203078254F
:100B000030386C780A0020207231323A2030782553
:100B100030386C780A2020206C723A2030782530EA
:100B2000386C780A20202070633A203078253038DD
:100B30006C780A20207073723A2030782530386C37
:100B4000780A0A004653522F4641523A0020434643
:100B500053523A2030782530386C780A00204846C5
:100B600053523A2030782530386C780A00204446B9
:100B700053523A2030782530386C780A00204146AC
:100B800053523A2030782530386C780A002042469B
:100B900041523A2030782530386C780A004D4D4665
:100BA00041523A2030782530386C780A004D69730C
:100BB00063004558435F5245543A20307825303819
:100BC0006C780A00417474656D7074696E67207486
:100BD0006F207265636F6E737472756374207374C3
:100BE00061746520666F7220646562756767696EFF
:100BF000672E2E2E00496E204744423A0A20207369
:100C00006574202470633D3078256C780A20206656
:100C100072616D6520300A202062740A000A49530F
:100C20005220737461636B206F766572666C6F77A8
:100C30006564206279206174206C6561737420257D
:100C4000642062797465732E0A004841524420463C
:100C500041554C542048414E444C45520046414970
:100C60004C454420415353455254494F4E2E002584
:100C7000700A002A2A2A2052494F54206B65726E4E
:100C8000656C2070616E69633A0A25730A0A002A4E
:100C90002A2A2068616C7465642E0A0A006D6169F5
:100CA0006E28293A20546869732069732052494F8D
:100CB0005421202856657273696F6E3A20554E4B49
:100CC0004E4F574E20286275696C646469723A20F1
:100CD0002F686F6D652F656C6F7065732F5046457B
:100CE00031352F52494F5429290A0069646C650037
:100CF0006D61696E005F5100210E0108290E010827
:100D0000320E01083B0E0108410E0108490E010890
:100D1000520E01085B0E0108640E01086C0E0108FA
:100D2000740E01087374617465006E616D6500096D
:100D3000706964207C20252D3231737C20252D396B
:100D40007351207C20707269207C20737461636B06
:100D5000202028207573656429207C2062617365DA
:100D6000206164647220207C2063757272656E74E9
:100D700020202020200A000920202D207C206973BB
:100D8000725F737461636B2020202020202020205C
:100D90002020207C202D20202020202020202D20DD
:100DA0007C2020202D207C202536692028253569AF
:100DB00029207C2025313070207C20253130700A9C
:100DC000000925336869207C20252D323073207C72
:100DD00020252D387320252E3173207C2025336962
:100DE000207C20253669202825356929207C20256E
:100DF000313070207C2025313070200A007C005377
:100E0000554D000925357320252D3231737C253150
:100E10003373253673202536692028253569290A3C
:100E20000073746F7070656400736C656570696ED3
:100E30006700626C206D7574657800626C20727852
:100E400000626C2073656E6400626C207265706C69
:100E50007900626C20616E79666C00626C20616C56
:100E60006C666C00626C206D626F780072756E6EDD
:100E7000696E670070656E64696E670000440040CB
:100E800000000200030002400200024007070026A3
:100E90000048004000000400090C0240080C024019
:100EA00007070027070604020107070503020000E1
:100EB00000300140070002400600024005000240E9
:100EC00004000240050000000010000001000000C6
:100ED000003800400F0402400E0402400D0402409E
:100EE0000C0402400500000000400000000000006B
:100EF00000000040FFFFFFFF01000000001C000099
:100F0000000C0040FFFFFFFF08000000003200005F
:100F100002020000000000000000000000000000CD
:100F20004572726F72206372656174696E672055D5
:100F3000445020736F636B004572726F722073654B
:100F40006E64696E67207265706C790057616974B0
:100F5000696E67207061636B65742E2E2E00676F5B
:100F6000004572726F722073656E64696E67206DE2
:100F70006573736167650054696D65646F757400AE
:100F80004572726F7220726563656976696E67205B
:100F90006D65737361676500525454203D20256967
:100FA000206D730A006572726F723A20636F756C00
:100FB00064206E6F742061646420444F4441472074
:100FC0002825732920746F20696E7374616E6365C0
:100FD00020282564290A0073756363657373667539
:100FE0006C6C792061646465642061206E65772093
:100FF00052504C20444F4441470A0052494F54201C
:101000006E6574776F726B20737461636B206578A3
:10101000616D706C65206170706C69636174696F7B
:101020006E00736F636B5F636C69656E745F746889
:101030007265616400736F636B5F7365727665726E
:101040005F746872656164006E6577206E6F6465B9
:10105000203F00416C6C2075702C2072756E6E699B
:101060006E6720746865207368656C6C206E6F779E
:10107000000000000100000003000000060C024018
:1010800002100240070C02400A0C02405B617574BA
:101090006F5F696E69745F6E657469665D20657205
:1010A000726F7220696E697469616C697A696E67C2
:1010B0002061743836726632787820726164696FA4
:1010C000202325750A0061743836726632787800FC
:1010D0006970763600293A11676E72635F6E6574C7
:1010E0006465763A20706F737369626C79206C6FF7
:1010F000737420696E746572727570742E00FF02CD
:10110000000000000000000000000000001A525023
:101110004C0001020000366C6F00FF7F3F1F0F077D
:10112000030175647000FFFFFE80000000000000F6
:1011300000000000000000000000000000000000AF
:101140000000000000000000FF010000000000009F
:101150000000000000000001FF020000000000008D
:101160000000000000000001FF020000000000007D
:1011700000000001FF000000FF020000000000006E
:10118000000000000000000200000000000000005D
:1011900000000000000000013031323334353637B2
:1011A0003839616263646566007368656C6C3A2007
:1011B000696E636F72726563742071756F74696EA6
:1011C000670068656C700044657363726970746968
:1011D0006F6E00436F6D6D616E6400252D3230734C
:1011E0002025730A007368656C6C3A20636F6D6D1F
:1011F000616E64206E6F7420666F756E643A202590
:10120000730A007265626F6F74005265626F6F746B
:1012100020746865206E6F64650070730050726999
:101220006E747320696E666F726D6174696F6E2083
:1012300061626F75742072756E6E696E6720746876
:1012400072656164732E0070696E67360050696E56
:1012500067207669612049434D5076360072616E91
:10126000646F6D5F696E697400696E697469616C41
:10127000697A6573207468652050524E4700726128
:101280006E646F6D5F6765740072657475726E73FE
:1012900020333220626974206F6620707365756434
:1012A0006F2072616E646F6D6E6573730069666343
:1012B0006F6E66696700436F6E6669677572652059
:1012C0006E6574776F726B20696E746572666163A8
:1012D000657300666962726F757465004D616E6951
:1012E00070756C61746520746865204649422028D9
:1012F000696E666F3A2027666962726F7574652041
:101300005B6164647C64656C5D2729006E63616366
:101310006865006D616E616765206E65696768620A
:101320006F722063616368652062792068616E6412
:1013300000726F757465727300495076362064656B
:101340006661756C7420726F75746572206C697358
:10135000740072706C0072706C20636F6E666967E7
:1013600075726174696F6E20746F6F6C20282772BC
:10137000706C2068656C702720666F72206D6F72CC
:101380006520696E666F726D6174696F6E29006E9B
:101390007470646174650073796E6368726F6E69EE
:1013A0007A6573207769746820612072656D6F7447
:1013B000652074696D652073657276657200000042
:1013C000031201080A120108E99100081A12010823
:1013D0001D120108F3910008471201084D1201087F
:1013E00061AC00085D12010869120108FD91000856
:1013F0007E1201088912010835920008AD12010819
:10140000B6120108219B0008D3120108DC12010862
:1014100091A500080C1301081313010879A800080E
:10142000311301083913010875AA00085213010885
:10143000561301084DB500088F13010897130108D2
:1014400061B700080000000000000000000000007C
:1014500050524E4720696E697469616C697A65649F
:1014600020746F2063757272656E742074696D6587
:101470003A2025640A0050524E4720696E6974690B
:10148000616C697A656420676976656E2076616C47
:1014900075653A2025640A004F464600534C454581
:1014A00050005354414E4442590049444C45005267
:1014B00058005458005245534554002530387800A0
:1014C0002873686F72742920616464726573730095
:1014D0006C6F6E67206164647265737300736F75FF
:1014E0007263652061646472657373206C656E67F6
:1014F0007468006368616E6E656C0070616765009A
:101500006E6574776F726B206964656E7469666965
:10151000657200545820706F776572205B696E2089
:1015200064426D5D006D61782E2072657472616E2B
:10153000736D697373696F6E730043534D4120720D
:101540006574726965730043434120746872657302
:10155000686F6C64205B696E2064426D5D00656E2F
:101560006372797074696F6E00656E6372797074FE
:10157000696F6E206B65790075736167653A202528
:1015800073203C69665F69643E20736574203C6B20
:1015900065793E203C76616C75653E0A002020200E
:1015A0002020205365747320616E20686172647717
:1015B0006172652073706563696669632073706525
:1015C00063696669632076616C75650A2020202056
:1015D00020203C6B65793E206D6179206265206F2B
:1015E0006E65206F662074686520666F6C6C6F771F
:1015F000696E670A202020202020202A2022616492
:10160000647222202D2073657473202873686F72B2
:10161000742920616464726573730A20202020207D
:1016200020202A2022616464725F6C6F6E67222022
:101630002D2073657473206C6F6E67206164647213
:101640006573730A202020202020202A2022616434
:1016500064725F73686F727422202D20616C6961FF
:101660007320666F72202261646472220A20202037
:10167000202020202A20226368616E6E656C222063
:101680002D207365747320746865206672657175AA
:10169000656E6379206368616E6E656C0A20202038
:1016A000202020202A20226368616E22202D2061C4
:1016B0006C69617320666F7220226368616E6E656B
:1016C0006C220A202020202020202A202263736DF3
:1016D000615F7265747269657322202D2073657471
:1016E000206D61782E206E756D626572206F6620A8
:1016F0006368616E6E656C206163636573732061FE
:101700007474656D7074730A202020202020202AB4
:1017100020226363615F7468726573686F6C642212
:10172000202D2073657420454420746872657368A9
:101730006F6C6420647572696E6720434341206951
:101740006E2064426D0A202020202020202A2022A2
:101750006E696422202D207365747320746865207F
:101760006E6574776F726B206964656E7469666903
:10177000657220286F72207468652050414E2049A0
:1017800044290A202020202020202A20227061675E
:101790006522202D2073657420746865206368615C
:1017A0006E6E656C2070616765202849454545204F
:1017B0003830322E31352E34290A202020202020A6
:1017C000202A202270616E22202D20616C696173B5
:1017D00020666F7220226E6964220A202020202059
:1017E00020202A202270616E5F696422202D2061F2
:1017F0006C69617320666F7220226E6964220A2010
:101800002020202020202A2022706F77657222203D
:101810002D20545820706F77657220696E206442C5
:101820006D0A202020202020202A20227265747238
:10183000616E7322202D206D61782E206E756D6291
:101840006572206F662072657472616E736D697364
:1018500073696F6E730A202020202020202A202206
:101860007372635F6C656E22202D20736574732024
:1018700074686520736F7572636520616464726556
:101880007373206C656E67746820696E206279746A
:10189000650A202020202020202A202273746174D1
:1018A0006522202D20736574207468652064657638
:1018B0006963652073746174650A202020202020EC
:1018C000202A2022656E637279707422202D207385
:1018D00065742074686520656E6372797074696FD1
:1018E0006E206F6E2D6F66660A202020202020203B
:1018F0002A20226B657922202D207365742074685C
:101900006520656E6372797074696F6E206B65799E
:1019100020696E2068657861646563696D616C201B
:10192000666F726D61740A00756E006572726F7217
:101930003A20756E61626C6520746F207365742047
:101940006F7074696F6E00737563636573733A20AB
:101950002573736574206F7074696F6E0A00657209
:10196000726F723A20756E61626C6520746F2070C0
:101970006172736520616464726573732E0A4D75BC
:101980007374206265206F6620666F726D617420CB
:101990005B302D39612D66412D465D7B327D283AC5
:1019A0005B302D39612D66412D465D7B327D292AC4
:1019B0000A286865782070616972732064656C69B3
:1019C0006D6974656420627920636F6C6F6E732932
:1019D000006572726F723A20756E61626C65207478
:1019E0006F207365742000737563636573733A20A9
:1019F0007365742000206F6E20696E746572666175
:101A000063652025686920746F2025730A00206FA4
:101A10006E20696E74657266616365202568692051
:101A2000746F2025690A006572726F723A20756EB4
:101A300061626C6520746F207061727365207661DD
:101A40006C75652E0A4D75737420626520612031B6
:101A5000362D62697420756E7369676E65642069DE
:101A60006E74656765722028646563206F722068F4
:101A70006578290A00206F6E20696E746572666150
:101A800063652025686920746F2000307825303424
:101A9000780A004C61796572203200495076360030
:101AA000616C6C00556E6B6E6F776E00202020208D
:101AB0002020202020202050726F746F636F6C20D4
:101AC0006F722064657669636520646F65736E2745
:101AD000742070726F7669646520737461746973C1
:101AE000746963732E005265736574207374617436
:101AF00069737469637320666F72206D6F64756CAF
:101B000065202573210A002020202020202020206D
:101B100020205374617469737469637320666F72F3
:101B20002025730A20202020202020202020202073
:101B30005258207061636B65747320257520206294
:101B4000797465732025750A20202020202020200C
:101B5000202020205458207061636B657473202509
:101B60007520284D756C7469636173743A2025750E
:101B700029202062797465732025750A2020202091
:101B80002020202020202020545820737563636576
:101B900065646564202575206572726F72732025F7
:101BA000750A00776972656400776972656C6573A0
:101BB000730049666163652025326420200020435C
:101BC00068616E6E656C3A20256875200020506152
:101BD00067653A202568752000204E49443A203038
:101BE00078256878004C6F6E67204857616464728E
:101BF0003A2000257320000A2020202020202020C9
